:020000040800F2
:1000000000040020E5010008150F0008190F000882
:100010006D0F0008190F0008410F0008E7010008E4
:10002000E7010008E7010008E7010008C52800080B
:10003000E7010008E7010008E7010008E701000800
:10004000E7010008E7010008E7010008E7010008F0
:10005000E7010008E7010008153A0008413A0008E6
:100060006D3A0008993A0008C53A0008E70100080F
:10007000E7010008E7010008E7010008E7010008C0
:10008000E7010008E7010008E7010008E7010008B0
:10009000E7010008E7010008E7010008F13A00085D
:1000A000E7010008E7010008E7010008E701000890
:1000B00031380008E7010008E7010008E7010008FF
:1000C000E7010008E7010008E7010008E701000870
:1000D000E70100083D110008E70100085111000880
:1000E000593B0008E7010008E7010008E7010008A4
:1000F000E7010008E7010008E7010008E701000840
:10010000E7010008E7010008E7010008E70100082F
:100110006511000879110008E7010008E7010008EF
:10012000E7010008E7010008E7010008E70100080F
:10013000E7010008E7010008E7010008E7010008FF
:10014000E7010008E7010008E7010008B12F0008F7
:10015000E7010008E7010008E70100088D11000829
:10016000E7010008E7010008E7010008E7010008CF
:10017000E7010008E7010008E7010008E7010008BF
:10018000E7010008E7010008E7010008E7010008AF
:10019000E7010008E7010008E7010008E70100089F
:1001A000E7010008E7010008E7010008E70100088F
:1001B000E7010008E7010008E7010008E70100087F
:1001C000E7010008E7010008E7010008E70100086F
:1001D000E7010008E7010008E7010008E70100085F
:1001E000DD0E000802E000F000F8FEE772B63948C4
:1001F00080F30888384880F3098838484EF608515B
:10020000CEF20001086040F20000CCF200004EF691
:100210003471CEF200010860BFF34F8FBFF36F8FD0
:1002200040F20000C0F2F0004EF68851CEF200011C
:100230000860BFF34F8FBFF36F8F4FF00000E1EE08
:10024000100A4EF63C71CEF200010860062080F3E1
:100250001488BFF36F8F02F073FB03F07FFA4FF047
:1002600055301F491B4A91423CBF41F8040BFAE745
:100270001C49194A91423CBF41F8040BFAE71A495C
:100280001A4A1B4B9A423EBF51F8040B42F8040B2A
:10029000F8E700201749184A91423CBF41F8040B87
:1002A000FAE702F051FB03F0B5FA144C144DAC42DE
:1002B00003DA54F8041B8847F9E700F03FF8114CC3
:1002C000114DAC4203DA54F8041B8847F9E702F0F9
:1002D00039BB0000000400200024002000000008BA
:1002E0000000002000040020C83F00080024002077
:1002F000282400202824002060460020E001000877
:10030000E4010008E4010008E40100082DE9F04FD1
:100310002DED108AC1F80CD0C3689D46BDEC108A43
:10032000BDE8F08F002383F311882846A047002002
:1003300001F04CFF01F0FCFE00DFFEE71A4B7F22CC
:1003400070B500241A700F225C709C70DC701C71F8
:100350005C719C71DC711C725C729A72DC7202F0CE
:1003600083FA064602F0A8FA054650B90F4B9E42A2
:1003700017D001339E4241F2883412BF0546002453
:100380000125002002F07AFA0DB100F0B5F800F076
:1003900047FD00F019FC204600F00CF900F0ACF825
:1003A000F9E70446EDE700BF28240020010007B06C
:1003B00008B500F087FBA0F120035842584108BD62
:1003C00007B5054B02211B88ADF8043001A800F0E9
:1003D000E5FB03B05DF804FB403C0008064991F8DA
:1003E000243033B100230822086A81F8243000F059
:1003F0000DBC0120704700BF482400202DE9F84FB4
:10040000234C94F824300546884617468BBB2E466D
:10041000DFF87C90002F38D094F824A0BAF1000FB8
:1004200005D12022FF214846266200F0E7FCCAF1F0
:100430000805BD4228BF3D465FFA85FBAD00414639
:100440002A4604EB8A0000F0AFFC94F82430A7EBB6
:100450000B079B445FFA8BFBBBF1080F2E44A844AB
:10046000FFB284F824B0D5D1FFF7B8FF0028D1D16E
:1004700008E0266A06EB8306B042C9D0FFF7AEFF5C
:100480000028C4D10020BDE8F88F0120BDE8F88F16
:100490004824002010B5202383F311881248C36834
:1004A0000BB101F019FF0023104A0F484FF47A7185
:1004B00001F0D6FE002383F311880D4C236813B19D
:1004C0002368013B2360636813B16368013B636089
:1004D000084B1B7833B9636823B9022000F052FC43
:1004E0003223636010BD00BF34240020950400084F
:1004F000782500207024002010B5254B254953F89D
:10050000042F013200D110BD8B42F8D1224C234B75
:1005100022689A423AD9224B9B6803F1006303F5A3
:1005200080339A4232D2002000F068FB1D4B02203B
:10053000187000F019FC1C4B1A6C00221A64196E1A
:100540001A66196E596C5A64596E5A665A6E5A690F
:1005500042F080025A615A6922F080025A615A6957
:100560001A6942F000521A611A6922F000521A61A7
:100570001B6972B60D4A0E4B13601B68226820215E
:1005800081F311889D4683F30888104710BD00BF92
:10059000FCFF00081C00010804000108FFFF000820
:1005A00028240020702400200038024008ED00E0DC
:1005B000000001082DE9F04F99B0B34C01902022C2
:1005C000FF2110A8A66800F019FCB04A1378A346D2
:1005D000A3B9AF480121C3601170202383F31188B0
:1005E000C3680BB101F078FE0023AA4AA8484FF473
:1005F0007A7101F035FE002383F31188019B13B15A
:10060000A54B019A1A60A54AA349019F02920023B3
:1006100013704B6099461C461D469846012000F019
:10062000A3FB002F00F012829B4B1B68002B40F0B5
:100630000D8219B0BDE8F08F0220FFF7B9FE002847
:1006400040F0FB81019BB9F1000F08BF1F46944B9E
:100650001B88ADF82C3002210BA800F09FFADDE7D3
:100660004FF47A7000F02EFA031E0393EADB0220A7
:10067000FFF79EFE82460028E4D0039B581E042804
:1006800000F2DD81DFE800F0030E1114170018A856
:10069000052340F8343D042100F080FA54464FF021
:1006A000000856E004217848F6E704217D48F3E786
:1006B00004217D48F0E71C24204600F0A1FA043410
:1006C0000B9004210BA800F069FA2C2CF4D1E5E77B
:1006D000002DB7D0002CB5D00220FFF769FE0546EB
:1006E000002800F0AF8101206C4C00F087FA022056
:1006F000207000F039FB4FF000095FFA89FA50468C
:1007000000F08CFA074658B1504600F097FA09F10C
:1007100001090028F1D12C46A9460027634B97E731
:1007200001230220237000F011FB3E46DBF8083065
:100730009E4206D2304600F063FA0130EBD1043617
:10074000F4E7029B00261E70534BA9465E602C46C0
:10075000374600F05BFB15B1002C18BF0027FFF7F0
:100760002FFE5BE7002D3FF46DAF002C3FF46AAF26
:10077000029B0220187000F0F7FA322000F0A2F974
:10078000B0F1000AC0F25E811AF0030540F05A8110
:10079000DBF8082006EB0A03934200F25381BAF516
:1007A000807F00F24F8155450DDA4FF47A7000F0EA
:1007B00089F90490049B002BC0F244813C4A049BBD
:1007C000AB540135EFE7C820FFF7F2FD05460028DE
:1007D00000F038811F2E11D8C6F12004544528BFDF
:1007E000544610AB26F0030022463149184400F06D
:1007F000DBFA2246FF212E4800F000FB4FEAAA0A4E
:100800005FFA8AF22A493046FFF7F8FD04460028CD
:1008100000F01A8106EB8A0605469AE70220FFF7E8
:10082000C7FD00283FF40EAFFFF7D8FD00283FF4C6
:1008300009AF4FF0000A5346DBF8082092451CD25E
:10084000BAF11F0F12D8109A01320FD02AF003020A
:1008500018A90A4452F8202C0B92184604220BA91E
:1008600000F098FB0AF1040A0346E5E750460393BB
:1008700000F0C6F9039B0B90EFE718A8042140F89D
:100880004C3D00F08BF964E72824002074250020FB
:1008900034240020950400087825002070240020CE
:1008A000423C00082C24002030240020443C000856
:1008B0007424002018A8002340F8343D642100F07F
:1008C00039F900287FF4BEAE0220FFF771FD002841
:1008D0003FF4B8AE0B9800F0C3F918AB43F8480DDD
:1008E00004211846CDE718A8002340F8343D6421C0
:1008F00000F020F900287FF4A5AE0220FFF758FD94
:1009000000283FF49FAE0B9800F0B8F918AB43F8FD
:10091000440DE5E70220FFF74BFD00283FF492AEBF
:1009200000F0B2F918AB43F8400DD9E70220FFF709
:100930003FFD00283FF486AE0BA9142000F0AAF971
:10094000824618A8042140F83CAD00F027F9514632
:100950000BA896E7322000F0B5F8B0F1000AFFF6D8
:1009600071AE1AF0030F7FF46DAEDBF808200AEBCE
:10097000080393423FF666AE0220FFF719FD0028F8
:100980003FF460AE2AF0030AC244D0453FF4E1AE22
:10099000404600F035F904210A900AA800F0FEF85C
:1009A00008F10408F1E74FF47A70FFF701FD002821
:1009B0003FF448AEFFF712FD00283FF4AFAE109BA6
:1009C00001330CD0082210A90020FFF717FD0028E2
:1009D0003FF4A4AE2022FF2110A800F00FFAFFF789
:1009E000EFFC374801F0F8FB23E6002D3FF42AAE78
:1009F000002C3FF427AE18A8002340F8343D6421B2
:100A000000F098F8824600287FF41CAE0220FFF721
:100A1000CFFC00283FF416AE0390FFF7D1FC41F263
:100A2000883001F0D9FB0B9800F038FA00F0EEF9AD
:100A3000039B57461C461D46F0E5054689E64FF0E8
:100A40000008FFE52546FDE52C4667E6002000F09E
:100A500039F80490049B002BFFF6E3AD012000F071
:100A600075F9049B213B122B3FF6D8AD01A252F839
:100A700023F000BF3906000861060008D10600080F
:100A80001D0600081D0600081D0600086507000871
:100A9000550900081D080008B5080008E708000807
:100AA000150900081D0600082D0900081D0600088C
:100AB000A7090008530700081D060008EB090008F5
:100AC000A08601002DE9F34702AE00244FF47A75A9
:100AD00006F8014D144FDFF85880454397F9003070
:100AE0005A1C5FFA84F901D0A34212D158F82400AD
:100AF00003680122D3F820A031462B46D0470128B5
:100B000007D10A4B9DF8070083F8009002B0BDE8BA
:100B1000F0870134062CE1D14FF4FA7001F05CFB50
:100B20004FF0FF30F2E700BF00240020982500209E
:100B3000843C00082DE9F0474FF47A75144FDFF834
:100B4000588006464D43002497F900305A1C5FFA3E
:100B500084F901D0A34210D158F82400036804227C
:100B6000D3F820A031462B46D047042805D1094BA5
:100B700083F800900020BDE8F0870134062CE3D113
:100B80004FF4FA7001F028FB4FF0FF30BDE8F0871A
:100B90000024002098250020843C000830B4074B36
:100BA0001A78074B53F822402368DD69054B0A4643
:100BB000AC460146204630BC604700BF9825002067
:100BC000843C0008A086010070B501F051FD094C7D
:100BD000094E2070002530682378834208D901F03F
:100BE00041FD336805440133B5F5803F3360F2D3EE
:100BF00070BD00BF992500208025002001F0E6BDD2
:100C000000F1006000F580300068704700F100607E
:100C1000920000F5803001F071BD0000054B1A68AC
:100C2000054B1B789B1A834202D9104401F01ABD70
:100C300000207047802500209925002038B5074DF9
:100C400004462868204401F015FD28B9286820448E
:100C5000BDE8384001F026BD38BD00BF802500202A
:100C600010F0030308D1B0F5007F05D800F1005063
:100C7000A0F508400068704700207047014BC0583D
:100C8000704700BF107AFF1F014B1868704700BF04
:100C9000002004E070B52A4B1C68C4F30B03240C3D
:100CA00063B140F21342934231D040F21942934271
:100CB0002FD040F2214293422DD10323214A0C250B
:100CC00005FB03235D6893F9082042F201039C426F
:100CD00024D0B4F5805F23D041F201039C4221D09F
:100CE00041F203039C421FD041F207039C4208BF1C
:100CF0003122441E0C44013D0B46A3421ED215F97D
:100D0000016F581C96B1034600F8016CF5E701230A
:100D1000D4E70223D2E73F220B4DD6E73322E3E7A5
:100D20004122E1E75A22E4E75922E2E72C258442F6
:100D30001D7001D9981C5A70401A70BD1846FBE707
:100D4000002004E0543C0008483C0008022804D17C
:100D50004FF08042034B9A6170470128FCD14FF05D
:100D60000052F7E700000240022804D14FF480420D
:100D7000034B9A6170470128FCD14FF40052F7E70A
:100D800000000240022805D1064A536983F48043DB
:100D9000536170470128FCD1024A536983F4005320
:100DA000F6E700BF0000024010B50023934203D0D5
:100DB000CC5CC4540133F9E710BD000030B5441ECB
:100DC00014F9010F0B4660B193F90050854201F10F
:100DD000010106D11AB993F90020801A30BD013AF9
:100DE000EEE7002AF7D1104630BD00000246034668
:100DF000981A13F9011B0029FAD1704702440346DF
:100E0000934202D003F8011BFAE77047024B1A78AD
:100E1000024B1A70704700BF982500200024002064
:100E2000F8B5184C1848194D194E174F00F01CFD15
:100E30002146154800F044FD24681648626DD2F83A
:100E4000043843F00203C2F8043801F0C5F9204623
:100E5000114900F041FE626DD2F8043823F002031C
:100E6000C2F804384FF4E1332B60002456F8240014
:100E7000B84202D0294600F055FC0134062CF5D1C9
:100E8000F8BD00BF743D0008943C0020842500207C
:100E9000843C000840420F009C3D000838B50B4BD5
:100EA0001A780B4B53F822400A4B9C4205460CD053
:100EB000094B002118461422FFF7A0FF05600146E8
:100EC0002046BDE8384000F02DBC38BD98250020F4
:100ED000843C0008943C00208425002070B50A4C16
:100EE0001826324600212046FFF788FF0125074BD0
:100EF0006360657032460021A019FFF77FFF044B45
:100F000025766576E36170BD9C2500200E000240C9
:100F10000D000240FEE7000000B59BB0EFF3098131
:100F200068226846FFF740FFEFF30583034B9A6B97
:100F30009A6A9A6A9A6A9A6A9B6AFEE700ED00E0EA
:100F400000B59BB0EFF3098168226846FFF72CFFDC
:100F5000EFF30583044B9A6B9A6A9A6A9A6A9A6AC3
:100F60009A6A9B6AFEE700BF00ED00E000B59BB007
:100F7000EFF3098168226846FFF716FFEFF3058358
:100F8000034B5A6B9A6A9A6A9A6A9A6A9B6AFEE754
:100F900000ED00E030B5084D0A4491420BD011F845
:100FA000013B09245840013CF7D040F300032B409B
:100FB00083EA5000F7E730BD2083B8ED00230449F1
:100FC0001A465A50C8180833802B4260F9D170472E
:100FD000CC250020026843681143016003B1184723
:100FE00070470000024AD36843F0C003D3607047E3
:100FF00000100140024AD36843F0C003D360704739
:1010000000480040024AD36843F0C003D3607047F1
:10101000004C0040024AD36843F0C003D3607047DD
:1010200000500040024AD36843F0C003D3607047C9
:10103000001401402DE9F041D0F85C64F768336892
:10104000DA0505469CB20DD5202383F311884FF4B1
:1010500000710430FFF7BEFF6FF48073336000232C
:1010600083F31188202383F3118805F1040814F019
:101070002F0333D183F31188380615D5210613D5F4
:10108000202383F3118805F1380000F0A9FA002825
:1010900046DA0821281DFFF79DFF4FF67F733B407E
:1010A000F360002383F311887A060ED563060CD50E
:1010B000202383F31188EA6C2B6D9A4202D12B6CAA
:1010C000002B2FD1002383F31188D5F86424D36833
:1010D000002B31D01069BDE8F0411847230713D029
:1010E00014F0080F0CBF00218021E00748BF41F039
:1010F0002001A20748BF41F04001630748BF41F407
:1011000080714046FFF766FFA406736805D595F821
:1011100060142846194000F013FB3468A4B2A6E717
:101120007060BEE727F040073F041021281D3F0CE8
:10113000FFF750FFF760C5E7BDE8F08108B5034849
:10114000FFF778FFBDE8084001F0CCBB4C2600203B
:1011500008B50348FFF76EFFBDE8084001F0C2BBC9
:10116000B42A002008B50348FFF764FFBDE8084033
:1011700001F0B8BB1C2F002008B50348FFF75AFF49
:10118000BDE8084001F0AEBB8433002008B5034839
:10119000FFF750FFBDE8084001F0A4BBEC3700208A
:1011A00010B5174C174A2046002100F099FA164B4B
:1011B000C4F85C34154C164A2046002100F090FA21
:1011C000144BC4F85C34144C144A2046002100F03F
:1011D00087FA134BC4F85C34124C134A20460021A2
:1011E00000F07EFA114BC4F85C34114C114A002116
:1011F000204600F075FA104BC4F85C3410BD00BFF7
:101200004C260020E50F000800100140B42A002001
:10121000F50F0008004800401C2F002005100008B2
:10122000004C00408433002015100008005000409E
:10123000EC370020251000080014014038B5494D56
:10124000037C002918BF0D46012B0446C0F86454E6
:1012500010D1454B984242D1444B5A6C42F0100297
:101260005A645A6E42F010025A665B6E0B212520BA
:1012700000F08EF83E4BD4F85C249A422B6802D0E2
:101280003C498A426BD13C4901EB5301B1FBF3F37A
:10129000A988080442BF23F0070003F0070343EACC
:1012A00040039360EB8843F040039BB213612B89AA
:1012B00043F001039BB2536141F4045343F02C0308
:1012C000D36001F4A05100231360B1F5806F13685F
:1012D00053680CBF7F23FF2384F8603438BD274B4D
:1012E00098420CD1214B1A6C42F480221A641A6E77
:1012F00042F480221A661B6E0B212720B8E7204B90
:1013000098420CD1194B1A6C42F400221A641A6EDE
:1013100042F400221A661B6E0B213420A8E7194BF9
:1013200098420CD1114B1A6C42F480121A641A6E56
:1013300042F480121A661B6E0B21352098E7124B7F
:10134000984297D1094B5A6C42F020025A645A6E67
:1013500042F020025A665B6E0B21472088E70B495A
:1013600092E700BFBC3C00084C2600200038024039
:10137000001001400014014000BD0105B42A002006
:101380001C2F002084330020EC37002080DE8002F8
:1013900000F1604300F01F02400903F561430901B9
:1013A0008000C9B200F1604083F8001300F561408D
:1013B00001239340C0F8803103607047F8B51546AB
:1013C00082680669AA420B46816938BF8568761A29
:1013D000B542044607D218462A46FFF7E5FCA36942
:1013E0002B44A3610DE011D932461846FFF7DCFC0F
:1013F000AF1B3A46E1683044FFF7D6FCE2683A4456
:10140000A261A3685B1BA3602846F8BD18462A4664
:10141000FFF7CAFCE368E4E783682DE9F04104467E
:1014200093421546266938BF85684069361AB54229
:101430000F4606D22A46FFF7B7FC63692B44636167
:101440000DE012D93246A5EB0608FFF7ADFC424687
:10145000B919E068FFF7A8FCE26842446261A3683A
:101460005B1BA3602846BDE8F0812A46FFF79CFC81
:10147000E368E4E710B50A440024C361029B0060FE
:1014800040608460C160816141610261036210BD9E
:1014900008B582694369934201D1826882B9826842
:1014A000013282605A1C42611970426903699A4292
:1014B00001D3C3684361002100F0AAFE002008BDEB
:1014C0004FF0FF3008BD000070B5202304460E46E3
:1014D00083F31188A568A5B1A368A269013BA36045
:1014E000531CA36115782269934224BFE368A3616A
:1014F000E3690BB120469847002383F311882846FF
:1015000070BD3146204600F073FE0028E2DA85F314
:10151000118870BD2DE9F74F05460F4690469A4653
:10152000D0F81C90202686F311884FF0000B14464B
:1015300064B1224639462846FFF740FF034668B9A2
:101540005146284600F054FE0028F1D0002383F3D2
:101550001188A8EB040003B0BDE8F08FB9F1000FCB
:1015600003D001902846C847019B8BF31188E41AE9
:101570001F4486F31188DBE7C16081614161C3616B
:101580001144009B0060406082600161036270470B
:10159000F8B504460E461746202383F31188A56844
:1015A000A5B1A368013BA36063695A1C62611E7008
:1015B000236962699A4224BFE3686361E3690BB1FE
:1015C00020469847002080F31188F8BD3946204610
:1015D00000F00EFE0028E2DA85F31188F8BD000065
:1015E000836942699A4210B501D182687AB98268EA
:1015F000013282605A1C82611C7803699A4201D3CD
:10160000C3688361002100F003FE204610BD4FF047
:10161000FF3010BD2DE9F74F05460F4690469A461C
:10162000D0F81C90202686F311884FF0000B14464A
:1016300064B1224639462846FFF7EEFE034668B9F4
:101640005146284600F0D4FD0028F1D0002383F352
:101650001188A8EB040003B0BDE8F08FB9F1000FCA
:1016600003D001902846C847019B8BF31188E41AE8
:101670001F4486F31188DBE7026843681143016069
:1016800003B11847704700001430FFF743BF000054
:101690004FF0FF331430FFF73DBF00003830FFF745
:1016A000B9BF00004FF0FF333830FFF7B3BF000081
:1016B0001430FFF709BF00004FF0FF311430FFF77F
:1016C00003BF00003830FFF763BF00004FF0FF3268
:1016D0003830FFF75DBF000000207047FFF760BDA6
:1016E00037B50F4B0360002343608360C360012361
:1016F00004460374154600900B464FF4007200F147
:101700005C011430FFF7B6FE00942B464FF40072D4
:1017100004F5177104F13800FFF72EFF03B030BD58
:10172000D03C000810B52023044683F31188FFF74E
:1017300085FD02232374002383F3118810BD00006C
:1017400038B5C36904460D461BB904210844FFF7A8
:1017500093FF294604F11400FFF79AFE002806DAE9
:10176000201D4FF48061BDE83840FFF785BF38BDCC
:10177000026843681143016003B1184770470000D5
:1017800013B5446BD4F894341A681178042915D130
:10179000217C022912D11979128901238B4013422D
:1017A0000CD101A904F14C0001F052FED4F894448C
:1017B000019B21790246206800F0DAF902B010BDE1
:1017C000143001F0D5BD00004FF0FF33143001F0AC
:1017D000CFBD00004C3001F0A7BE00004FF0FF333A
:1017E0004C3001F0A1BE0000143001F0A3BD000098
:1017F0004FF0FF31143001F09DBD00004C3001F07E
:1018000073BE00004FF0FF324C3001F06DBE00009F
:10181000D0F8942438B5136819780429054601D006
:10182000012038BD017C0229FAD112795C8901209E
:1018300090400440F4D105F1140001F035FD02465A
:101840000028EDD0D5F894544FF480732868697956
:1018500000F07CF9204638BD406BFFF7D9BF00008F
:1018600000207047704700007FB5124B03600023D3
:1018700043608360C360012502260F4B0574044654
:101880000290019300F18402294600964FF4807380
:10189000143001F0E5FC094B0193029400964FF4DB
:1018A000807304F52372294604F14C0001F0ACFD6D
:1018B00004B070BDF83C00085918000881170008F2
:1018C0000B68202282F311880A7903EB820290616F
:1018D0004A79093243F822008A7912B103EB820374
:1018E000986102230374C0F89414002383F31188D1
:1018F0007047000038B5037F044613B190F85430A8
:10190000ABB9201D01250221FFF732FF04F11400BD
:1019100025776FF0010100F087FC84F8545004F142
:101920004C006FF00101BDE8384000F07DBC38BDCF
:1019300010B5012104460430FFF71AFF0023237776
:1019400084F8543010BD000038B50446002514302A
:1019500001F09EFC04F14C00257701F06DFD201D87
:1019600084F854500121FFF703FF2046BDE83840BA
:10197000FFF74EBF90F8443003F06003202B19D1DD
:1019800090F84520212A0AD0222A4FF000030ED0D9
:10199000202A0FD1084A82630722C26304E0064B63
:1019A00083630723C36300230364012070478363B9
:1019B000C363F9E70020704701240020D0F8943475
:1019C00037B51A681178042904461AD1017C022916
:1019D00017D11979128901238B40134211D100F1DB
:1019E0004C05284601F0E8FD58B101A9284601F050
:1019F0002FFDD4F89444019B21790246206800F021
:101A0000B7F803B030BD000000EB8103F7B59C6967
:101A100005460E46F4B1202383F3118805EB8607B3
:101A2000201D0821FFF7A4FEFB685B691B684C348E
:101A300013B1204601F01AFD01A9204601F008FD6E
:101A4000024648B1019B3146284600F091F8002338
:101A500083F3118803B0F0BDFB685A691268002A4D
:101A6000F5D01B8A013B1340F1D105F14402EAE7AE
:101A7000093138B550F82140DCB1202383F31188B7
:101A8000D4F894241368527903EB8203DB689B69D2
:101A90005D6845B104216018FFF76AFE294604F12C
:101AA000140001F00BFC2046FFF7B2FE002383F385
:101AB000118838BD7047000000F0CCBF01230370CF
:101AC00000234360C36183620362C36243620363B2
:101AD000038143817047000038B50446202383F317
:101AE000118800254160C56005614561856100F090
:101AF000C1FF0223237085F3118838BD70B500EB58
:101B0000810305465069DA600E46144618B110226A
:101B10000021FFF773F9A06918B110220021FFF727
:101B20006DF931462846BDE8704001F06DB80000FF
:101B3000028902F001020281428902F0010242811F
:101B4000002202614261826101F0F2B8F0B400EB60
:101B500081044789E4680125A4698D403D4345819E
:101B600023600023A2606360F0BC01F00DB90000A7
:101B7000F0B400EB81040789E468012564698D40B5
:101B80003D43058123600023A2606360F0BC01F047
:101B900087B9000070B50223002504460370A0F841
:101BA0004C5080F84E5080F84F5005814581C560FB
:101BB00005614561856180F8345000F0C1FF6368BC
:101BC0001B6823B129462046BDE87040184770BD08
:101BD000436802781B6880F85020052202700BB120
:101BE0000421184770470000436890F850201B6894
:101BF00002700BB1052118477047000090F834308F
:101C000070B5044613B1002380F8343004F1440267
:101C1000204601F0AFF863689B6863BB94F84450BA
:101C200015F0600615D194F8453005F07F0545EABA
:101C3000032540F202339D4200F00E815BD8022D55
:101C400000F0DC803FD8002D00F08780012D00F0EF
:101C5000CF800021204601F0E5FA0021204601F066
:101C6000D7FA63681B6813B10621204698470623FC
:101C700084F8343070BD204698470028CED094F8C0
:101C80004B2094F84A3043EA0223E26B934238BF78
:101C9000E36394F94430E56B002B4FF0200380F2AE
:101CA000FD80002D00F0EC80092284F8342083F3BD
:101CB00011880021E36BA26B2046FFF759FF002338
:101CC00083F3118870BDB5F5817F00F0B180B5F563
:101CD000407F49D0B5F5807FBBD194F84630012BC9
:101CE000B7D1B4F84C3023F00203A4F84C30A6630B
:101CF000E6632664C3E740F201639D421ED8B5F552
:101D0000C06F3BD2B5F5A06FA3D1B4F84430B3F5A2
:101D1000A06F0ED194F8463084F84E30204600F083
:101D200067FF63681B6813B10121204698470323AE
:101D300023700023A363E3632364A0E7B5F5106F6A
:101D400032D040F602439D4252D0B5F5006F80D1AB
:101D500004F14F03A363012324E004F14C03A363C4
:101D60000223E36325648AE794F84630012B7FF46D
:101D700070AFB4F84C3043F00203B6E794F8492052
:101D8000616894F848304D6894F8471043EA02239C
:101D9000204694F84620A84700283FF45AAF4368ED
:101DA000A3630368E363A4E72378042B10D1202303
:101DB00083F311882046FFF7BBFE86F31188636822
:101DC00084F84F601B68032121700BB120469847AF
:101DD00094F84630002BACD084F84F3004232370A5
:101DE00063681B68002BA4D0022120469847A0E717
:101DF000374BA3630223E36300239DE794F8481065
:101E000011F0800F204601F00F010ED000F0A4FF6A
:101E1000012806D002287FF41CAF2E4BA363E06399
:101E200067E72D4BA363E56363E700F087FFEFE708
:101E300094F84630002B7FF40CAF94F8483013F040
:101E40000F013FF476AF1A06204602D501F0FEF9E5
:101E50006FE701F0F1F96CE794F84630002B7FF45E
:101E6000F8AE94F8483013F00F013FF462AF1B0650
:101E7000204602D501F0D6F95BE701F0C9F958E731
:101E8000142284F8342083F311882B462A462946ED
:101E90002046FFF75BFE85F3118870BD5DB115220A
:101EA00084F8342083F311880021E36BA26B204671
:101EB000FFF74CFE03E70B2284F8342083F31188EC
:101EC0002B462A4629462046FFF752FEE3E700BF8D
:101ED000283D0008203D0008243D000838B590F852
:101EE00034300446152B29D8DFE803F03E28282893
:101EF00028283E28280B2939282828282828282857
:101F00003E3E90F84B1090F84A20C36B42EA012203
:101F10009A4214D9C268128AB3FBF2F502FB153556
:101F20006DB9202383F311882B462A462946FFF7F3
:101F30001FFE85F311880A2384F8343038BD14233A
:101F400084F83430202383F3118800231A4619467D
:101F50002046FFF7FBFD002383F3118838BD036C97
:101F600003B198470023E7E7002101F05BF9002166
:101F7000204601F04DF963681B6813B10621204625
:101F800098470623D8E7000090F83420152A38B582
:101F9000044622D80123934040F6416213421DD1EA
:101FA00013F480150FD19B0217D50B2380F8343022
:101FB000202383F311882B462A462946FFF7D8FDB4
:101FC00085F3118838BDC3689B695B682BB9036CC6
:101FD00003B19847002384F8343038BD002101F064
:101FE00021F90021204601F013F963681B6813B141
:101FF0000621204698470623EDE70000024B002209
:102000001B605B609A607047543C0020002303749F
:102010008268054B1B6899689142FBD25A6803603D
:102020004260106058607047543C002008B520237F
:1020300083F31188037C032B05D0042B0DD02BB91F
:1020400083F3118808BD436900221A604FF0FF3303
:102050004361FFF7DBFF0023F2E790E80C001A6012
:1020600002685360F2E70000002303748268054BA6
:102070001B6899689142FBD85A68036042601060FF
:1020800058607047543C0020054B19690874186863
:1020900002681A605360186101230374FEF736B9B1
:1020A000543C002030B54B1C87B005460A4C10D07C
:1020B00023690A4A01A800F0D3F82846FFF7E4FF95
:1020C000049B13B101A800F007F92369586907B010
:1020D00030BDFFF7D9FFF8E7543C00202D20000861
:1020E00038B50C4D41612B6981689A68914204466C
:1020F00003D8BDE83840FFF789BF1846FFF786FFD1
:1021000001232C61014623742046BDE83840FEF7C8
:10211000FDB800BF543C0020044B1A681B6990684E
:102120009B68984294BF002001207047543C0020D7
:1021300010B5084C236820691A6822605460012297
:1021400023611A74FFF790FF01462069BDE8104033
:10215000FEF7DCB8543C00208260022202740022A8
:10216000427470478368A3F17C0243F80C2C026927
:1021700043F83C2C426943F8382C074A43F81C2C9E
:10218000C26843F8102C022203F8082C002203F83E
:10219000072CA3F1180070472503000810B5202371
:1021A00083F31188FFF7DEFF00210446FFF798FF55
:1021B000002383F31188204610BD0000024B1B69E9
:1021C00058610F20FFF760BF543C0020202383F3A9
:1021D0001188FFF7F3BF000008B50146202383F301
:1021E00011880820FFF75EFF002383F3118808BDE4
:1021F00049B1064B42681B6918605A60136043601E
:102200000420FFF74FBF4FF0FF307047543C0020D1
:102210000368984206D01A680260506059611846F7
:10222000FFF7F4BE7047000038B504460D4620683D
:10223000844200D138BD036823605C604561FFF7CC
:10224000E5FEF4E7054B03F114025A619A614FF081
:10225000FF32DA6100221A62704700BF543C00204E
:10226000F8B503614FF08043C2605C6A194B1A46AF
:10227000022952F8145F38BF0221954206461F46D4
:102280000AD1586198611C62056045608160081937
:10229000BDE8F84001F0B2B9186AAB68241A0C190D
:1022A00002D3E41A2D6804E09C4202D2204401F0DB
:1022B000B3F9AB689C42F4D86B68736035601E60FC
:1022C0006E60B460A9684FF0FF33091BA960FB6121
:1022D000F8BD00BF543C002010B41B4C234653F8FB
:1022E000141F814210D0416802680A600268516080
:1022F0009A424FF00001C16003D0936881680B449B
:1023000093605DF8044B70470A68626100209A424E
:102310005360C86003D15DF8044B01F077B993684E
:102320008868034493604FF08042206A526A121A10
:102330009342E6D9991A012998BF931C18445DF875
:10234000044B01F069B900BF543C002000207047E5
:10235000FEE70000704700004FF0FF3070470000BC
:10236000022906D0032906D00129064818BF0020FB
:10237000704705487047032A9ABF044800EBC20023
:1023800000207047F83D0008AC3D000808240020FC
:1023900070B59AB001AD064608462946144600F0CD
:1023A00095F82846FEF722FDC0B2431C5B0086E884
:1023B0001800237003236370002302341946DAB235
:1023C000904204F1020401D81AB070BDEA5C04F82E
:1023D000022C04F8011C0133F1E7000008B52023AA
:1023E00083F311880348FFF7E9FA002383F3118888
:1023F00008BD00BF943C002010B50446052916D83E
:10240000DFE801F016150316161D202383F311884B
:102410000E4A0121FFF772FB20460D4A0221FFF709
:102420006DFB0C48FFF790FA002383F3118810BD71
:10243000202383F311880748FFF75CFAF4E7202391
:1024400083F311880348FFF773FAEDE72C3D00088A
:10245000503D0008943C002038B50C4D0C4C0D4903
:102460002A4604F10800FFF793FF05F1CA0204F1C0
:1024700010000949FFF78CFF05F5CA7204F1180036
:102480000649BDE83840FFF783BF00BF5C4100202C
:10249000082400207C3D0008863D0008913D00088E
:1024A00070B5044608460D46FEF7A0FCC6B22046AD
:1024B000013403780BB9184670BD32462946FEF741
:1024C0007DFC0028F3D1012070BD00002DE9F0470C
:1024D00004460D46FEF78AFC2C49C6B22046FFF79B
:1024E000DFFF08B10736F6B229492046FFF7D8FFCB
:1024F00008B11036F6B2632E0BD8DFF89080DFF803
:102500009090244FDFF898A0267846B92E70BDE849
:10251000F08721462846BDE8F04701F089BB252E0B
:102520002FD1072241462046FEF748FC70B91A4BCE
:102530002A4603F10C0153F8040B42F8040B8B42BA
:10254000F9D11B88138007340E35DDE70822494690
:102550002046FEF733FCA0B9104BAA1C13F8011F4C
:1025600009095345C95D02F8021C197801F00F01F1
:1025700002F10202C95D02F8031CEFD118350834DC
:10258000C2E72E7001340135BEE700BF183E0008D7
:10259000913D00082F3E0008203E00080F7AFF1FE3
:1025A0001B7AFF1FBFF34F8F024AD368DB03FCD4B3
:1025B000704700BF003C024008B5094B1B7873B957
:1025C000FFF7F0FF074B1A69002ABFBF064A5A609F
:1025D00002F188325A601A6822F480621A6008BDDB
:1025E000BA430020003C02402301674508B50B4B6D
:1025F0001B7893B9FFF7D6FF094B1A6942F00042E6
:102600001A611A6842F480521A601A6822F48052E1
:102610001A601A6842F480621A6008BDBA4300204A
:10262000003C02400B2870B513D80B4A0B4C1378B2
:1026300063B90B4E4FF0006144F8231056F8235055
:1026400001330C2B2944F7D10123137054F82000D7
:1026500070BD002070BD00BFEC430020BC430020D3
:10266000403E0008014B53F820007047403E0008F0
:102670000C2070470B2810B5044601D9002010BD6E
:10268000FFF7D0FF064B53F824301844C21A0BB999
:10269000012010BD12680132F0D1043BF6E700BF03
:1026A000403E00080B2810B5044621D8FFF77AFFFA
:1026B000FFF782FF0F4AF323D360C300DBB243F47A
:1026C000007343F002031361136943F48033136111
:1026D000FFF768FFFFF7A6FF074B53F8241000F041
:1026E000DDF8FFF783FF2046BDE81040FFF7C2BFCB
:1026F000002010BD003C0240403E00082DE9F84398
:1027000012F00103154640D18218B2F1016F3CD29C
:102710002C4B1B6813F0010337D02B4CFFF74CFFF9
:10272000F323E360FFF73EFF40F20127032D01D9B9
:10273000830713D0244C0F46401A40F20118EB1BBC
:102740000B44012B00EB0706236924D823F0010377
:102750002361FFF74BFF0120BDE8F883236923F4D1
:102760004073236123693B43236151F8046B066086
:10277000BFF34F8FFFF716FF03689E4208D023690F
:1027800023F001032361FFF731FF0020BDE8F88348
:10279000043D0430CAE723F440732361236943EA0C
:1027A00008032361B94637F8023B3380BFF34F8FEC
:1027B000FFF7F8FE3688B9F80030B6B2B342BED0A3
:1027C000DDE700BF00380240003C0240084908B580
:1027D0000B7828B153B9FFF7EFFE01230B7008BD4A
:1027E00023B1BDE808400870FFF700BF08BD00BF77
:1027F000BA43002010B50244064B0439D2B29042CD
:1028000000D110BD441C00B253F8200041F8040F61
:10281000E0B2F4E750280040104B30B51C6F2404A0
:1028200007D41C6F44F400741C671C6F44F400440C
:102830001C670B4C236843F4807323600244094BEC
:102840000439D2B2904200D130BD441C00B251F8DC
:10285000045F43F82050E0B2F4E700BF00380240C4
:10286000007000405028004007B5012201A9002057
:10287000FFF7C0FF019803B05DF804FB13B50446F1
:10288000FFF7F2FFA04206D002A9012241F8044D51
:102890000020FFF7C1FF02B010BD0000704700002C
:1028A000034B1B689B0042BF024B01221A7070470A
:1028B00074380240ED430020014B1878704700BF88
:1028C000ED430020064A536823F001035360EFF301
:1028D0000983683383F30988002383F311887047E1
:1028E00030EF00E010B5202383F31188104B5B68B4
:1028F00013F4006318D0F1EE103AEFF309844FF0AF
:10290000807344F84C3C0B4BDB6844F8083CA4F162
:10291000680383F30988FFF7FFFB18B1064B44F8FF
:10292000503C10BD054BFAE783F3118810BD00BF82
:1029300000ED00E030EF00E0350300083803000848
:1029400070470000FEE70000084A094B09498B4226
:1029500004D3094A0021934205D3704752F8040F6B
:1029600043F8040BF3E743F8041BF4E7EC3F0008DB
:10297000604600206046002060460020836D30B530
:1029800000229D68446D11464FF0FF3004EB421366
:1029900001329542C3F80019C3F81019C3F80809A9
:1029A000C3F8001BC3F8101BC3F8080BEED24FF09E
:1029B0000113C4F81C3830BD890141F020010161C8
:1029C00003699B06FCD4122000F0AEBE204B03EB43
:1029D00080022DE9F047D2F80CE05D6DDEF814209E
:1029E000461CD2F800C005EB063605EB40185168CE
:1029F00061450BD3D5F83428012303FA00F022EA0D
:102A00000000C5F834081846BDE8F087BEF810404D
:102A1000ACEB0103A34228BF2346D8F81849A4B25F
:102A2000B3EB840F10D894681F46A4F1040959F839
:102A300004AFC6F800A0042F01D9043FF7E71C44F7
:102A40000B4494605360D2E70020BDE8F08700BFDC
:102A5000F043002010B5054C2046FFF72FF84FF04B
:102A6000A0436365024BA36510BD00BFF043002087
:102A7000943E00080378012B70B5054650D12A4BCF
:102A8000446D98421BD1294B5A6B42F080025A6325
:102A90005A6D42F080025A655A6D5A6942F08002BE
:102AA0005A615A6922F080025A610E2143205B6903
:102AB000FEF76EFC1E4BE3601E4BC4F8003800238B
:102AC000C4F8003EC02323606E6D4FF40413A3636B
:102AD0003369002BFCDA012333610C2000F024FE63
:102AE0003369DB07FCD4122000F01EFE3369002B93
:102AF000FCDA0026A6602846FFF740FF6B68C4F8A2
:102B00001068DB68C4F81468C4F81C684BB90A4B39
:102B1000A3614FF0FF336361A36843F00103A36037
:102B200070BD064BF4E700BFF043002000380240C0
:102B30004014004003002002003C30C0083C30C07C
:102B4000F8B5446D054600212046FFF735FFA96D15
:102B500000234FF001128F68C4F834384FF000663C
:102B6000C4F81C284FF0FF3004EB431201339F429E
:102B7000C2F80069C2F8006BC2F80809C2F8080B75
:102B8000F2D20B686A6DEB656362102313611669FC
:102B900016F01006FBD1122000F0C6FDD4F8003864
:102BA00023F4FE63C4F80038A36943F4402343F0E0
:102BB0001003A3610923C4F81038C4F814380A4B71
:102BC000EB604FF0C043C4F8103B084BC4F8003B27
:102BD000C4F81069C4F80039EB6D03F1100243F436
:102BE0008013EA65A362F8BD703E000840800010C3
:102BF000426D90F84E10D2F8003823F4FE6343EA99
:102C00000113C2F8003870472DE9F0410EB200EB15
:102C100086080D46D8F80C100F6807F00303022B46
:102C200050D0032B50D03D4A3D4F012B18BF1746C3
:102C3000446D4FEA451E04EB0E030022C3F8102B2F
:102C40008A6905F1100C002A40D04A8A05F1580320
:102C50005B013A43E2500123D4F81C2803FA0CF339
:102C60001343A6444A69C4F81C380023CEF810392F
:102C700005F13F03002A39D00A8A898B920801297D
:102C800088BF4A43C16D04EB8303561841EA0242F0
:102C9000C66529465A602046FFF78EFED8F80C30EC
:102CA0001B8A43EA85531F4305F148035B01E75044
:102CB0000123D4F81C2803FA05F51543C4F81C5861
:102CC000BDE8F081174FB3E7174FB1E704EB4613A8
:102CD000D3F8002B22F40042C3F8002BD4F81C28B0
:102CE000012303FA0CF322EA0303BAE704EB83039C
:102CF0000E4A5A6004EB461629462046FFF75CFE52
:102D0000D6F8003923F40043C6F80039D4F81C384B
:102D1000012202FA05F523EA0505CFE7008000103D
:102D2000008004100080081000800C1000040002D5
:102D3000826D1268C265FFF721BE00005831436DF5
:102D400049015B5813F4004004D013F4001F14BF72
:102D500001200220704700004831436D49015B5853
:102D600013F4004004D013F4001F14BF012002200C
:102D70007047000000EB8101CB68196A0B68136093
:102D80004B6853607047000000EB810330B5DD688D
:102D9000AA691368D36019B9402B84BF402313601C
:102DA0006B8A1468426D1C44013CB4FBF3F463432A
:102DB000033323F0030302EB411043EAC44343F01F
:102DC000C043C0F8103B2B6803F00303012B09B28A
:102DD0000ED1D2F8083802EB411013F4807FD0F8FE
:102DE000003B14BF43F0805343F00053C0F8003B56
:102DF00002EB4112D2F8003B43F00443C2F8003B1F
:102E000030BD00002DE9F041244D6E6D06EB4013FE
:102E10000446D3F8087BC3F8087B38070AD5D6F8F0
:102E20001438190706D505EB84032146DB682846CC
:102E30005B689847FA072FD5D6F81438DB072BD5EF
:102E400005EB8403D968CCB98B69488A5E68B6FB08
:102E5000F0F200FB12628AB91868DA6890420DD26B
:102E6000121A83E81400202383F311880B482146AB
:102E7000FFF78AFF84F31188BDE8F081012303FA8C
:102E800004F26B8923EA02036B81CB6823B12146EC
:102E90000248BDE8F0411847BDE8F081F04300204A
:102EA00000EB810370B5DD68436D6C692668E660F0
:102EB0004A0156BB1A444FF40020C2F810092A6890
:102EC00002F00302012A0AB20ED1D3F8080803EB7C
:102ED000421410F4807FD4F8000914BF40F08050F1
:102EE00040F00050C4F8000903EB4212D2F8000988
:102EF00040F00440C2F80009D3F83408012202FA75
:102F000001F10143C3F8341870BD19B9402E84BFD4
:102F10004020206020682E8A841940F00050013C37
:102F20001A44B4FBF6F440EAC440C6E7F8B50446D8
:102F30001E48456D05EB4413D3F80869C3F80869CA
:102F4000F10717D5D5F81038DA0713D500EB84034D
:102F5000D9684B691F68DA68974218D2D21B0027DC
:102F60001A605F60202383F311882146FFF798FFE2
:102F700087F31188330617D5D5F834280123A340E9
:102F8000134211D02046BDE8F840FFF71FBD0123D2
:102F900003FA04F2038923EA020303818B68002BFE
:102FA000E8D021469847E5E7F8BD00BFF043002090
:102FB00096482DE9F84F456D6E69AB691E4016F4D1
:102FC000805F6E61044605D0FEF7E4FDBDE8F84F72
:102FD000FFF788BC002E12DAD5F8003E8B489B071D
:102FE0001EBFD5F8003E23F00303C5F8003ED5F818
:102FF000043823F00103C5F80438FEF7F5FD370562
:1030000002D58248FEF7E4FDB0040CD5D5F80838A7
:1030100013F0060FEB6823F470530CBF43F4105306
:1030200043F4A053EB60310704D56368DB680BB150
:1030300076489847F2025AD4B3020CD5D4F854809B
:10304000DFF8C8A100274FF00109A36D9B68F9B212
:103050008B4280F08780F70619D5616D0A6AC2F34A
:103060000A1702F00F0302F4F012B2F5802F00F0FD
:10307000A180B2F5402F0AD104EB830301F5805102
:10308000DB68186A00231A469F4240F087803003AD
:10309000D5F8184813D5E10302D50020FFF7B2FE9A
:1030A000A20302D50120FFF7ADFE630302D5022083
:1030B000FFF7A8FE270302D50320FFF7A3FE750341
:1030C00084D5E00702D50020FFF730FFA10702D525
:1030D0000120FFF72BFF620702D50220FFF726FF32
:1030E00023077FF573AF0320FFF720FF6EE7D4F8C7
:1030F0005480DFF818A100274FF00109A36D9B68E9
:103100005FFA87FB5B4597D308EB4B13D3F8002995
:1031100002F44022B2F5802F22D1D3F80029002AF0
:103120001EDAD3F8002942F09042C3F80029D3F800
:103130000029002AFBDB5946606DFFF73DFC228920
:1031400009FA0BF322EA0303238104EB8B03DB6808
:103150009B6813B15946504698475846FFF736FCCE
:103160000137CBE708EB4112D2F8003B03F44023D0
:10317000B3F5802F10D1D2F8003B002B0CDA628916
:1031800009FA01F322EA0303638104EB8103DB689C
:10319000DB680BB150469847013756E79C0708BFDC
:1031A0000A68072B98BF027003F101039CBF120A43
:1031B000013069E7023304EB830201F58051526864
:1031C00090690268D0F808C04068A2EB000E0022A7
:1031D000104697420AD104EB830463689B699A689E
:1031E0003A449A605A6817445F6050E712F0030F40
:1031F00008BF0868964588BF8CF8000002F10102FC
:1032000084BF000A0CF1010CE3E700BFF04300208B
:10321000436D03EB4111D1F8003B43F40013C1F8B7
:10322000003B7047436D03EB4111D1F8003943F483
:103230000013C1F800397047436D03EB4111D1F819
:10324000003B23F40013C1F8003B7047436D03EBD0
:103250004111D1F8003923F40013C1F80039704747
:1032600030B5039C0172043304FB0325C361049B46
:1032700003630021059B00604060C1604261026100
:103280008561046242628162C162436330BD0000B5
:103290000022416A41610161C2608262C2626FF0D4
:1032A0000101FEF7C1BF000003694269934203D1E7
:1032B000C2680AB100207047181D70470369196081
:1032C000C2680132C260C2691344826903619342D9
:1032D00024BF436A03610021FEF79ABF38B5044654
:1032E0000D46E3683BB16269131D1268A362134483
:1032F000E362002038BD237A33B929462046FEF721
:1033000077FF0028EDDA38BD6FF00100FBE7000021
:10331000C368C269013BC360436913448269436166
:10332000934224BF436A436100238362036B03B16A
:103330001847704770B52023044683F31188866AC6
:103340003EB9FFF7CBFF054618B186F31188284632
:1033500070BDA36AE26A13F8015BA362934202D3D1
:103360002046FFF7D5FF002383F31188EFE7000025
:103370002DE9F84F04460E4690469946202787F3DC
:1033800011880025AA46D4F828B0BBF1000F09D156
:1033900049462046FFF7A2FF20B18BF3118828464B
:1033A000BDE8F88FA16AE36AA8EB050B5B1A9B45A1
:1033B00028BF9B46BBF1400F1BD9334601F14002A9
:1033C00051F8040B43F8040B9142F9D1A36A40333E
:1033D0004036A3624035A26AE36A9A4202D320468D
:1033E000FFF796FF8AF311884545D8D287F31188F5
:1033F000C9E730465A46FDF7D7FCA36A5B445E44F2
:10340000A3625D44E7E7000010B5029C017204333B
:1034100003FB0421C36100238362C362039B036334
:10342000049B00604060C46042610261816104628B
:103430004262436310BD0000026AC260426A426198
:10344000026100228262C2626FF00101FEF7ECBEEF
:10345000436902699A4203D1C2680AB100207047E9
:10346000184650F8043B0B6070470000C368C269FF
:103470000133C3604369134482694361934224BFAB
:10348000436A43610021FEF7C3BE000038B504461D
:103490000D46E3683BB123691A1DA262E269134439
:1034A000E362002038BD237A33B929462046FEF76F
:1034B0009FFE0028EDDA38BD6FF00100FBE7000049
:1034C00003691960C268013AC260C2691344826923
:1034D0000361934224BF436A036100238362036B49
:1034E00003B118477047000070B5202304460E460C
:1034F00083F31188856A35B91146FFF7C7FF10B10C
:1035000085F3118870BDA36A1E70A36AE26A013355
:103510009342A36204D3E16920460439FFF7D0FF48
:10352000002080F3118870BD2DE9F84F04460D4648
:1035300091469A464FF0200888F311880026B3463A
:10354000A76A4FB951462046FFF7A0FF20B187F385
:1035500011883046BDE8F88FA06AE76AA9EB060338
:103560003F1A9F4228BF1F46402F1BD905F1400339
:1035700055F8042B40F8042B9D42F9D1A36A40333F
:10358000A3624036A26AE36A9A4204D3E169204604
:103590000439FFF795FF8BF311884E45D9D288F394
:1035A0001188CDE729463A46FDF7FEFBA36A3B4466
:1035B0003D44A3623E44E5E7026943699A4203D170
:1035C000C3681BB9184670470023FBE7836A002BCA
:1035D000F8D0043B9B1AF5D01360C368013BC3606D
:1035E000C3691A44836902619A4224BF436A036132
:1035F000002383620123E5E700F02EB94FF08043FA
:10360000002258631A610222DA6070474FF080434B
:103610000022DA60704700004FF080435863704723
:10362000FEE7000010B5174CFEF7E8FCFEF70AFEB7
:10363000802215492046FEF78FFD012344F8180C1F
:103640000374124B124AD96821F4E0610904090C91
:103650000A431049DA60CA6842F08072CA600E49B3
:103660000A6842F001020A601022DA77202283F809
:103670002220002383F3118862B60848BDE8104079
:10368000FEF78CBD7C3C0020A03E000800ED00E071
:103690000003FA05F0ED00E0001000E0A83E00088D
:1036A0002DE9F84F1F4C4FF00008656904F114072D
:1036B000C1464FF08043266A5B6AAA689E1B964209
:1036C0001DD34FF0200AAA68236AD5F80CB0134422
:1036D00023622B68BB425F60A6EB02066361C5F8FC
:1036E0000C8001D1FFF792FF89F311882869D84730
:1036F0008AF311886569AB689E42E4D2D9E76269B2
:10370000BA420CD0916823628E1B9660A86802288A
:103710002CBF1818981CBDE8F84FFFF77DBFBDE817
:10372000F88F00BF543C0020034B59685A68521A66
:103730009042FBD8704700BF001000E04B68436028
:103740008B688360CB68C3600B6943614B6903621C
:103750008B6943620B6803607047000008B5224B19
:1037600022481A6940F2FF110A431A611A6922F4C9
:10377000FF7222F001021A611A691A6B0A431A6376
:103780001A6D0A431A651A4A1B6D1146FFF7D6FFD8
:10379000184802F11C01FFF7D1FF174802F1380168
:1037A000FFF7CCFF154802F15401FFF7C7FF14489B
:1037B00002F17001FFF7C2FF124802F18C01FFF71E
:1037C000BDFF114802F1A801FFF7B8FF0F4802F151
:1037D000C401FFF7B3FF0E4802F1E001FFF7AEFFAF
:1037E000BDE8084000F0A2B80038024000000240E6
:1037F000C83E00080004024000080240000C0240DD
:10380000001002400014024000180240001C024058
:103810000020024008B500F0F9F9FFF703FFFFF7B9
:103820003FF8BDE80840FEF717BE000070470000F3
:103830004FF0804310B51A69920708D500241C6127
:10384000202383F31188FFF72BFF84F31188BDE851
:103850001040FFF747B80000104B1A6C42F001020D
:103860001A641A6E42F001021A660D4A1B6E9368C2
:1038700043F0010393604FF0804353229A624FF06C
:10388000FF32DA6200229A615A63DA605A600122DA
:103890005A6108211A601C20FDF77ABD00380240E9
:1038A000002004E01F4B1A696FEAC2526FEAD2523D
:1038B0001A611A69C2F308021A614FF0FF301A69DF
:1038C0005A69586100215A6959615A691A6A62F045
:1038D00080521A621A6A02F080521A621A6A5A6A8E
:1038E00058625A6A59625A6A1A6C42F080521A64D3
:1038F0001A6E42F080521A661A6E0B4A106840F433
:1039000080701060186F00F44070B0F5007F1EBF2B
:103910004FF4803018671967536823F400735360BD
:1039200000F054B90038024000700040304B4FF0B6
:1039300080521A642F4A4FF4404111601A6842F0D5
:1039400001021A601A689207FCD59A6822F00302F5
:103950009A60274B19469A6812F00C02FBD118683E
:1039600000F0F90018609A601A6842F480321A6018
:103970000B689B03FCD54B6F43F001034B671C4B5B
:103980005A6F9007FCD51C4A5A601A6842F0807240
:103990001A60184A53685904FCD5154B1A689201ED
:1039A000FCD5164A9A60164B1A68164B9A42164B6B
:1039B0001BD1164A1168164A914216D140F20512DF
:1039C0001A600B4B9A6842F002029A609A6802F001
:1039D0000C02082AFAD15A6C42F480425A645A6E98
:1039E00042F480425A665B6E704740F20572E7E728
:1039F00000380240007000400854400700948838A6
:103A0000002004E011640020003C024000ED00E0D2
:103A100041C20F41084A08B5536911680B4003F0D1
:103A20000103536123B1054A13680BB150689847ED
:103A3000BDE80840FEF756BF003C0140CC25002001
:103A4000084A08B5536911680B4003F0020353613B
:103A500023B1054A93680BB1D0689847BDE8084088
:103A6000FEF740BF003C0140CC250020084A08B5C5
:103A7000536911680B4003F00403536123B1054AF5
:103A800013690BB150699847BDE80840FEF72ABF9B
:103A9000003C0140CC250020084A08B55369116854
:103AA0000B4003F00803536123B1054A93690BB13E
:103AB000D0699847BDE80840FEF714BF003C0140BC
:103AC000CC250020084A08B5536911680B4003F063
:103AD0001003536123B1054A136A0BB1506A98472A
:103AE000BDE80840FEF7FEBE003C0140CC250020AA
:103AF000174B10B55C691A68144004F478725A6167
:103B0000A30604D5134A936A0BB1D06A984760069E
:103B100004D5104A136B0BB1506B9847210604D59E
:103B20000C4A936B0BB1D06B9847E20504D5094A58
:103B3000136C0BB1506C9847A30504D5054A936CE0
:103B40000BB1D06C9847BDE81040FEF7CBBE00BF6C
:103B5000003C0140CC2500201A4B10B55C691A6866
:103B6000144004F47C425A61620504D5164A136D70
:103B70000BB1506D9847230504D5134A936D0BB1D3
:103B8000D06D9847E00404D50F4A136E0BB1506E08
:103B90009847A10404D50C4A936E0BB1D06E984798
:103BA000620404D5084A136F0BB1506F9847230481
:103BB00004D5054A936F0BB1D06F9847BDE810400C
:103BC000FEF790BE003C0140CC250020062108B540
:103BD0000846FDF7DDFB06210720FDF7D9FB06218E
:103BE0000820FDF7D5FB06210920FDF7D1FB0621B2
:103BF0000A20FDF7CDFB06211720FDF7C9FB0621A2
:103C00002820BDE80840FDF7C3BB000008B5FFF75A
:103C100049FEFDF7D3F9FDF761FDFDF74DFFFDF717
:103C200021FEFFF703FEBDE80840FFF7E5BC0000FA
:103C3000034611F8012B03F8012B002AF9D1704734
:103C4000121012131211000053544D3332463F3FED
:103C50003F00000000000000483C00083F0000005A
:103C6000130400009C3C00083F0000001904000001
:103C7000A63C00083F00000021040000B03C000802
:103C80003F000000943C00204C260020B42A002075
:103C90001C2F002084330020EC37002053544D3378
:103CA00032463430780053544D3332463432780043
:103CB00053544D3332463434365858000096000081
:103CC00000000000000000000000000000000000F4
:103CD00000000000A516000891160008CD16000887
:103CE000B9160008C5160008B11600089D16000890
:103CF00089160008D916000800000000DD1700082A
:103D0000C917000805180008F1170008FD1700087A
:103D1000E9170008D5170008C11700086118000846
:103D20000000000001000000000000000200000090
:103D300000000000091A0008711A00084000400045
:103D40002C4100203C410020020000000000000047
:103D50000300000000000000B51A00080000000089
:103D6000100000004C410020000000000100000095
:103D700000000000F0430020010102004172647560
:103D800050696C6F740025424F415244252D424CBE
:103D9000002553455249414C25000000F9230008F5
:103DA0006123000875190008DD23000843000000A6
:103DB000B43D000809024300020100C032090400BA
:103DC0000001020201000524001001052401000188
:103DD000042402020524060001070582030800FFEF
:103DE00009040100020A000000070501024000006A
:103DF000070581024000000012000000003E00089C
:103E00001201100102000040091241570002010294
:103E1000030100000403090425424F4152442500D8
:103E20004D6174656B463430352D57696E670030CF
:103E30003132333435363738394142434445460010
:103E40000040000000400000004000000040000072
:103E5000000001000000020000000200000002005B
:103E6000000002000000020000000200000002004A
:103E700000000000FD1B0008DD1E0008891F00086F
:103E80004000400050440020504400200100000049
:103E9000604400208000000040010000030000009A
:103EA0006D61696E00000000C03E0008684400209B
:103EB00060460020010000002136000800000000DC
:103EC00069646C65000000000A01A816000000008B
:103ED000AAAAAAAA05011400FF9F000088000000FA
:103EE00070A70A000000000100000000AAAAAAAA08
:103EF00000000001FFFF00000000000000000000C3
:103F000000A0A01200000000AAAAAAAA0050501106
:103F1000FFFF00000000008800770800200000007C
:103F200000000000AAAAAAAA10000000FFFF0000DB
:103F30000008000000000000000000000000000079
:103F4000AAAAAAAA00000000FFFF000000000000CB
:103F5000000000000000000000000000AAAAAAAAB9
:103F600000000000FFFF0000000000000000000053
:103F70000000000000000000AAAAAAAA0000000099
:103F8000FFFF000000000000000000000000000033
:103F9000000000000A000000000000000300000014
:103FA0000000000000000000000000000000000011
:103FB0000000000000000000000000000000000001
:103FC0000000000000000000FF0096000000000854
:103FD00004000000143E0008000000000000000083
:103FE00000000000000000000000000000000000D1
:103FF000FFFFFFFFFFFFFFFFFFFFFFFFFFFFFFFFD1
:10400000FFFFFFFFFFFFFFFFFFFFFFFFFFFFFFFFC0
:10401000FFFFFFFFFFFFFFFFFFFFFFFFFFFFFFFFB0
:020000040801F1
:100000000006002099120108DD560A0839560A0830
:10001000A5560A0839560A0871560A089B120108A3
:100020009B1201089B1201089B12010875C80C085D
:100030009B1201089B1201089B1201089B120108E8
:100040009B1201089B1201089B1201089B120108D8
:100050009B1201089B1201080DD40C0835D40C0822
:100060005DD40C0885D40C08ADD40C08F5760C08CA
:100070001D770C0849770C0875770C08A1770C08D8
:10008000C9770C08F5770C0879760C089B120108E3
:100090009B1201089B1201089B120108D5D40C0881
:1000A00021D60C0835D60C0849D60C084DD60C08BC
:1000B00051D60C0865D60C0879D60C084D800C0872
:1000C00061800C0885800C0899800C089B1201083F
:1000D0009B120108A9D50C08BDD50C08D1D50C0878
:1000E00039D50C089B1201089B1201089DD60C08FB
:1000F000A1D60C08B5D60C08B9D60C0821780C0886
:100100009B1201089B1201088DD60C089B12010856
:10011000E5D50C08F9D50C089B1201089B120108C3
:100120004D780C0875780C08A1780C08CD780C086F
:10013000F9780C089B1201089B1201089B12010818
:100140009B1201089B1201089B120108A1CF0C0809
:1001500021790C084D790C0879790C080DD60C081A
:100160009B1201089B1201089B1201089B120108B7
:100170009B1201089B1201089B1201089B120108A7
:100180009B1201089B1201089B1201089B12010897
:100190009B1201089B1201089B1201089B12010887
:1001A0009B1201089B1201089B1201089B12010877
:1001B0009B1201089B1201089B1201089B12010867
:1001C0009B1201089B1201089B1201089B12010857
:1001D0009B1201089B1201089B1201089B12010847
:1001E000496501089D2F0308ADA80408512F060892
:1001F000753506081DB50608591907081D21070899
:1002000055240708CD84070841A90708C93A0808FA
:10021000218E0808799B080879480A085D4D0A086C
:10022000C9460B0861B30B08C5D90B0831E50B08AB
:10023000BD140C08E91A0C080000000000000000C2
:1002400081F0004102E000BF83F0004330B54FEA87
:1002500041044FEA430594EA050F08BF90EA020FF4
:100260001FBF54EA000C55EA020C7FEA645C7FEA87
:10027000655C00F0E2804FEA5454D4EB5555B8BFAA
:100280006D420CDD2C4480EA020281EA030382EA1B
:10029000000083EA010180EA020281EA0303362DAD
:1002A00088BF30BD11F0004F4FEA01314FF4801C80
:1002B0004CEA113102D0404261EB410113F0004F92
:1002C0004FEA03334CEA133302D0524263EB430349
:1002D00094EA050F00F0A780A4F10104D5F1200EE7
:1002E0000DDB02FA0EFC22FA05F2801841F1000142
:1002F00003FA0EF2801843FA05F359410EE0A5F116
:1003000020050EF1200E012A03FA0EFC28BF4CF046
:10031000020C43FA05F3C01851EBE37101F00045FC
:1003200007D54FF0000EDCF1000C7EEB00006EEB09
:100330000101B1F5801F1BD3B1F5001F0CD3490893
:100340005FEA30004FEA3C0C04F101044FEA4452EA
:1003500012F5800F80F09A80BCF1004F08BF5FEA71
:10036000500C50F1000041EB045141EA050130BD51
:100370005FEA4C0C404141EB0101013C28BFB1F563
:10038000801FE9D291F0000F04BF01460020B1FAAE
:1003900081F308BF2033A3F10B03B3F120020CDA81
:1003A0000C3208DD02F1140CC2F10C0201FA0CF05F
:1003B00021FA02F10CE002F11402D8BFC2F1200CC4
:1003C00001FA02F120FA0CFCDCBF41EA0C0190407A
:1003D000E41AA2BF01EB0451294330BD6FEA0404C3
:1003E0001F3C1CDA0C340EDC04F11404C4F12002AE
:1003F00020FA04F001FA02F340EA030021FA04F3C0
:1004000045EA030130BDC4F10C04C4F1200220FA16
:1004100002F001FA04F340EA0300294630BD21FA54
:1004200004F0294630BD94F0000F83F4801306BF1A
:1004300081F480110134013D4EE77FEA645C18BF0E
:100440007FEA655C29D094EA050F08BF90EA020FA5
:1004500005D054EA000C04BF1946104630BD91EA9D
:10046000030F1EBF0021002030BD5FEA545C05D1A0
:100470004000494128BF41F0004130BD14F58004DF
:100480003CBF01F5801130BD01F0004545F0FE4153
:1004900041F470014FF0000030BD7FEA645C1ABF88
:1004A000194610467FEA655C1CBF0B46024650EABF
:1004B000013406BF52EA033591EA030F41F40021EB
:1004C00030BD00BF90F0000F04BF0021704730B571
:1004D0004FF4806404F132044FF000054FF0000146
:1004E00050E700BF90F0000F04BF0021704730B507
:1004F0004FF4806404F1320410F0004548BF4042DC
:100500004FF000013EE700BF42004FEAE2014FEA30
:1005100031014FEA02701FBF12F07F4393F07F4F0B
:1005200081F06051704732F07F4208BF704793F00E
:100530007F4F04BF41F40021704730B54FF4607421
:1005400001F0004521F000411CE700BF50EA010224
:1005500008BF704730B54FF000050AE050EA0102CD
:1005600008BF704730B511F0004502D5404261EB3D
:1005700041014FF4806404F132045FEA915C3FF47E
:10058000D8AE4FF003025FEADC0C18BF03325FEA1B
:10059000DC0C18BF033202EBDC02C2F1200300FACC
:1005A00003FC20FA02F001FA03FE40EA0E0021FAF1
:1005B00002F11444BDE600BF70B54FF0FF0C4CF4DF
:1005C000E06C1CEA11541DBF1CEA135594EA0C0F91
:1005D00095EA0C0F00F0DEF82C4481EA030621EACC
:1005E0004C5123EA4C5350EA013518BF52EA033507
:1005F00041F4801143F4801338D0A0FB02CE4FF0B9
:100600000005E1FB02E506F00042E0FB03E54FF0E8
:100610000006E1FB03569CF0000F18BF4EF0010EE0
:10062000A4F1FF04B6F5007F64F5407404D25FEADC
:100630004E0E6D4146EB060642EAC62141EA55518F
:100640004FEAC52040EA5E504FEACE2EB4F1FD0CD1
:1006500088BFBCF5E06F1ED8BEF1004F08BF5FEA4F
:10066000500E50F1000041EB045170BD06F0004601
:1006700046EA010140EA020081EA0301B4EB5C04AE
:10068000C2BFD4EB0C0541EA045170BD41F48011A6
:100690004FF0000E013C00F3AB8014F1360FDEBFCB
:1006A000002001F0004170BDC4F10004203C35DAA7
:1006B0000C341BDC04F11404C4F1200500FA05F32A
:1006C00020FA04F001FA05F240EA020001F00042CB
:1006D00021F0004110EBD37021FA04F642EB060141
:1006E0005EEA430E08BF20EAD37070BDC4F10C046B
:1006F000C4F1200500FA04F320FA05F001FA04F22F
:1007000040EA020001F0004110EBD37041F100011A
:100710005EEA430E08BF20EAD37070BDC4F1200525
:1007200000FA05F24EEA020E20FA04F301FA05F28D
:1007300043EA020321FA04F001F0004121FA04F235
:1007400020EA020000EBD3705EEA430E08BF20EA05
:10075000D37070BD94F0000F0FD101F0004640003F
:1007600041EB010111F4801F08BF013CF7D041EAC1
:10077000060195F0000F18BF704703F000465200C5
:1007800043EB030313F4801F08BF013DF7D043EA96
:100790000603704794EA0C0F0CEA135518BF95EA4C
:1007A0000C0F0CD050EA410618BF52EA4306D1D1D3
:1007B00081EA030101F000414FF0000070BD50EAF2
:1007C000410606BF1046194652EA430619D094EA7C
:1007D0000C0F02D150EA013613D195EA0C0F05D166
:1007E00052EA03361CBF104619460AD181EA0301BA
:1007F00001F0004141F0FE4141F470014FF0000072
:1008000070BD41F0FE4141F4780170BD70B54FF00C
:10081000FF0C4CF4E06C1CEA11541DBF1CEA13558C
:1008200094EA0C0F95EA0C0F00F0A7F8A4EB05046E
:1008300081EA030E52EA03354FEA013100F0888065
:100840004FEA03334FF0805545EA131343EA12632E
:100850004FEA022245EA111545EA10654FEA0026E3
:100860000EF000419D4208BF964244F1FD0404F59C
:10087000407402D25B084FEA3202B61A65EB0305F8
:100880005B084FEA32024FF480104FF4002CB6EBB5
:10089000020E75EB030E22BFB61A754640EA0C0035
:1008A0005B084FEA3202B6EB020E75EB030E22BF75
:1008B000B61A754640EA5C005B084FEA3202B6EBB6
:1008C000020E75EB030E22BFB61A754640EA9C0075
:1008D0005B084FEA3202B6EB020E75EB030E22BF45
:1008E000B61A754640EADC0055EA060E18D04FEA03
:1008F000051545EA16754FEA06164FEAC30343EAA3
:1009000052734FEAC2025FEA1C1CC0D111F4801F6F
:100910000BD141EA00014FF000004FF0004CB6E768
:1009200011F4801F04BF01430020B4F1FD0C88BF07
:10093000BCF5E06F3FF6AFAEB5EB030C04BFB6EB12
:10094000020C5FEA500C50F1000041EB045170BD05
:100950000EF0004E4EEA113114EB5C04C2BFD4EB32
:100960000C0541EA045170BD41F480114FF0000EB6
:10097000013C90E645EA060E8DE60CEA135594EA32
:100980000C0F08BF95EA0C0F3FF43BAF94EA0C0F35
:100990000AD150EA01347FF434AF95EA0C0F7FF4AA
:1009A00025AF104619462CE795EA0C0F06D152EAFE
:1009B00003353FF4FDAE1046194622E750EA4106E2
:1009C00018BF52EA43067FF4C5AE50EA41047FF4F3
:1009D0000DAF52EA43057FF4EBAE12E74FF0FF3C58
:1009E00006E000BF4FF0010C02E000BF4FF0010C29
:1009F0004DF804CD4FEA410C7FEA6C5C4FEA430CA2
:100A000018BF7FEA6C5C1BD001B050EA410C0CBFF0
:100A100052EA430C91EA030F02BF90EA020F002052
:100A2000704710F1000F91EA030F58BF994208BFB9
:100A300090422CBFD8176FEAE37040F00100704776
:100A40004FEA410C7FEA6C5C02D150EA013C07D1CD
:100A50004FEA430C7FEA6C5CD6D152EA033CD3D018
:100A60005DF8040B704700BF8446104662468C4612
:100A70001946634600E000BF01B5FFF7B7FF002845
:100A800048BF10F1000F01BD4DF808EDFFF7F4FF6E
:100A90000CBF012000205DF808FB00BF4DF808EDF9
:100AA000FFF7EAFF34BF012000205DF808FB00BF1C
:100AB0004DF808EDFFF7E0FF94BF012000205DF83E
:100AC00008FB00BF4DF808EDFFF7CEFF94BF0120F3
:100AD00000205DF808FB00BF4DF808EDFFF7C4FFEC
:100AE00034BF012000205DF808FB00BF4FEA410C35
:100AF0007FEA6C5C02D150EA013C0AD14FEA430C18
:100B00007FEA6C5C02D152EA033C02D14FF0000054
:100B100070474FF0010070474FEA410212F5001292
:100B200015D211D56FF47873B3EB625212D94FEA34
:100B3000C12343F0004343EA505311F0004F23FA1E
:100B400002F018BF404270474FF00000704750EA73
:100B5000013005D111F0004008BF6FF00040704730
:100B60004FF00000704700BF4A0011D212F500128A
:100B700011D20DD56FF47873B3EB62520ED44FEAF5
:100B8000C12343F0004343EA505323FA02F0704775
:100B90004FF00000704750EA013002D14FF0FF30B3
:100BA00070474FF0000070474FEA4102B2F1E04356
:100BB00024BFB3F5001CDCF1FE5C0DD901F0004C44
:100BC0004FEAC0024CEA5070B2F1004F40EB830094
:100BD00008BF20F00100704711F0804F21D113F1C0
:100BE0003872BCBF01F00040704741F480114FEAF9
:100BF0005252C2F11802C2F1200C10FA0CF320FA82
:100C000002F018BF40F001004FEAC1234FEAD3239E
:100C100003FA0CFC40EA0C0023FA02F34FEA430308
:100C2000CCE77FEA625307D150EA01331EBF4FF091
:100C3000FE4040F44000704701F0004040F0FE40AC
:100C400040F40000704700BF80F0004002E000BFA9
:100C500081F0004142001FBF5FEA410392EA030FA7
:100C60007FEA226C7FEA236C6AD04FEA1262D2EBF1
:100C70001363C1BFD218414048404140B8BF5B42F6
:100C8000192B88BF704710F0004F40F4000020F08F
:100C90007F4018BF404211F0004F41F4000121F0A5
:100CA0007F4118BF494292EA030F3FD0A2F10102EF
:100CB00041FA03FC10EB0C00C3F1200301FA03F12D
:100CC00000F0004302D5494260EB4000B0F5000F50
:100CD00013D3B0F1807F06D340084FEA310102F10F
:100CE0000102FE2A51D2B1F1004F40EBC25008BFC1
:100CF00020F0010040EA03007047490040EB00008B
:100D0000013A28BFB0F5000FEDD2B0FA80FCACF18B
:100D1000080CB2EB0C0200FA0CF0AABF00EBC250B8
:100D200052421843BCBFD0401843704792F0000FA6
:100D300081F4000106BF80F400000132013BB5E7F9
:100D40004FEA41037FEA226C18BF7FEA236C21D06F
:100D500092EA030F04D092F0000F08BF08467047D4
:100D600090EA010F1CBF0020704712F07F4F04D1A2
:100D7000400028BF40F00040704712F100723CBFB5
:100D800000F50000704700F0004343F0FE4040F4DF
:100D9000000070477FEA226216BF08467FEA23639D
:100DA0000146420206BF5FEA412390EA010F40F488
:100DB000800070474FF0000304E000BF10F00043D4
:100DC00048BF40425FEA000C08BF704743F09643BB
:100DD00001464FF000001CE050EA010208BF7047D6
:100DE0004FF000030AE000BF50EA010208BF70475D
:100DF00011F0004302D5404261EB41015FEA010C72
:100E000002BF84460146002043F0B64308BFA3F169
:100E10008053A3F50003BCFA8CF2083AA3EBC2534B
:100E200010DB01FA02FC634400FA02FCC2F120026A
:100E3000BCF1004F20FA02F243EB020008BF20F0A1
:100E40000100704702F1200201FA02FCC2F1200207
:100E500050EA4C0021FA02F243EB020008BF20EAFC
:100E6000DC7070477BB972B90029BEBF00204FF01B
:100E7000004106E008BF00281CBF6FF000414FF0A2
:100E8000FF3000F007BAADF1080C6DE904CE00297F
:100E900009DB002B1ADB00F095F8DDF804E0DDE952
:100EA000022304B07047404261EB4101002B1BDB81
:100EB00000F088F8DDF804E0DDE9022304B04042E8
:100EC00061EB4101524263EB43037047524263EBD3
:100ED000430300F077F8DDF804E0DDE9022304B015
:100EE000404261EB41017047524263EB430300F023
:100EF00069F8DDF804E0DDE9022304B0524263EB57
:100F00004303704753B94AB9002908BF00281CBFE2
:100F10004FF0FF314FF0FF3000F0BCB9ADF1080CDD
:100F20006DE904CE00F04EF8DDF804E0DDE90223BF
:100F300004B07047430803F05533C01A830803F028
:100F4000333300F03330184400EB101000F00F3052
:100F500000EB002000EB0040000E704707EE900A07
:100F6000F5EEC07AF1EE10FA01D400F00BB8F1EE14
:100F7000677A08B517EE900A00F004F8404261EB7A
:100F8000410108BDD0B5FFF7BFFA0C4B0022064661
:100F90000F46FFF711FBFFF7E7FD0446FFF792FA54
:100FA000074B0022FFF708FB02460B463046394646
:100FB000FFF74AF9FFF7D8FD2146D0BD0000F03D0C
:100FC0000000F0412DE9F047089D04468E46002BB5
:100FD0004DD18A42944669D9B2FA82F252B101FAED
:100FE00002F3C2F1200120FA01F10CFA02FC41EAFD
:100FF000030E94404FEA1C48210CBEFBF8F61FFA82
:101000008CF708FB16E341EA034306FB07F199421C
:101010000AD91CEB030306F1FF3080F01F819942CF
:1010200040F21C81023E63445B1AA4B2B3FBF8F0A9
:1010300008FB103344EA034400FB07F7A7420AD930
:101040001CEB040400F1FF3380F00A81A74240F258
:1010500007816444023840EA0640E41B00261DB1C3
:10106000D4400023C5E900433146BDE8F0878B42F8
:1010700009D9002D00F0EF800026C5E900013046B7
:101080003146BDE8F087B3FA83F6002E4AD18B4291
:1010900002D3824200F2F980841A61EB030301203B
:1010A0009E46002DE0D0C5E9004EDDE702B9FFDE27
:1010B000B2FA82F2002A40F09280A1EB0C014FEAD2
:1010C0001C471FFA8CFE0126200CB1FBF7F307FB2F
:1010D000131140EA01410EFB03F0884208D91CEBD2
:1010E000010103F1FF3802D2884200F2CB8043466F
:1010F000091AA4B2B1FBF7F007FB101144EA01444E
:101100000EFB00FEA64508D91CEB040400F1FF31DC
:1011100002D2A64500F2BB800846A4EB0E0440EACA
:1011200003409CE7C6F12007B34022FA07FC4CEAD3
:10113000030C20FA07F401FA06F31C43F9404FEAC6
:101140001C4900FA06F3B1FBF9F8200C1FFA8CFEDB
:1011500009FB181140EA014108FB0EF0884202FA2F
:1011600006F20BD91CEB010108F1FF3A80F08880F0
:10117000884240F28580A8F102086144091AA4B2AD
:10118000B1FBF9F009FB101144EA014100FB0EFE2E
:101190008E4508D91CEB010100F1FF346CD28E455D
:1011A0006AD90238614440EA0840A0FB0294A1EBEE
:1011B0000E01A142C846A64656D353D05DB1B3EB4B
:1011C000080261EB0E0101FA07F722FA06F3F1407B
:1011D0001F43C5E9007100263146BDE8F087C2F122
:1011E0002003D8400CFA02FC21FA03F3914001439A
:1011F0004FEA1C471FFA8CFEB3FBF7F007FB1036D3
:101200000B0C43EA064300FB0EF69E4204FA02F47E
:1012100008D91CEB030300F1FF382FD29E422DD9D1
:10122000023863449B1B89B2B3FBF7F607FB163306
:1012300041EA034106FB0EF38B4208D91CEB010186
:1012400006F1FF3816D28B4214D9023E6144C91A06
:1012500046EA004638E72E46284605E70646E3E616
:101260001846F8E64B45A9D2B9EB020864EB0C0E20
:101270000138A3E74646EAE7204694E74046D1E72F
:10128000D0467BE7023B614432E7304609E76444DD
:10129000023842E7704700BF02E000F000F8FEE7C6
:1012A00072B6374880F30888364880F30988364894
:1012B0003649086040F20000CCF200004EF634716E
:1012C000CEF200010860BFF34F8FBFF36F8F40F283
:1012D0000000C0F2F0004EF68851CEF20001086026
:1012E000BFF34F8FBFF36F8F4FF00000E1EE100A96
:1012F0004EF63C71CEF200010860062080F314889F
:10130000BFF36F8FBBF014FBBAF07CFB4FF055308E
:101310001F491B4A91423CBF41F8040BFAE71D49A3
:10132000184A91423CBF41F8040BFAE71A491B4A9C
:101330001B4B9A423EBF51F8040B42F8040BF8E7EE
:1013400000201849184A91423CBF41F8040BFAE7C3
:10135000BBF0F2FABAF0AAFB144C154DAC4203DA1A
:1013600054F8041B8847F9E701F092FB114C124D29
:10137000AC4203DA54F8041B8847F9E7BBF0DABA49
:1013800000060020002200200000010808ED00E017
:101390000000002000060020E0740F08002200205A
:1013A000382B0020382B0020305F0120E00101089D
:1013B0003802010838020108380201082DE9F04F0F
:1013C0002DED108AC1F80CD0C3689D46BDEC108A83
:1013D000BDE8F08F002383F311882846A047002042
:1013E000BAF096F8FEE7B9F0F3FE00DFFEE7000082
:1013F00001F0FF01102A2BDB10F0070F08D010F8C6
:10140000013B013A8B422DD010F0070F42B3F6D1C9
:10141000F0B441EA012141EA014122F007047FF0E2
:1014200000070023F0E80256083C85EA010586EA39
:10143000010685FA47F5A3FA87F586FA47F6A5FA75
:1014400087F68EB9EED1F0BC01F0FF0102F0070281
:1014500032B110F8013B013A83EA010313B1F8D12C
:101460000020704701387047002D06BF354603380D
:10147000073815F0010F07D1013015F4807F02BF46
:10148000013015F4C03F0130F0BC0138704700BF97
:1014900010F8012B11F8013B012A28BF9A42F7D01E
:1014A000D01A7047034613F8012B002AFBD1181AF3
:1014B0000138704738B50022002304460D46FFF777
:1014C000EDFA28B920462946BDE8384000F00AB8B0
:1014D000204605F1004100F005F8404261EB410172
:1014E00038BD00BFD0B50C4B002206460F46FFF7B3
:1014F00063F8FFF739FB0446FEF7E4FF074B0022D1
:10150000FFF75AF802460B4630463946FEF79CFE76
:10151000FFF72AFB2146D0BD0000F03D0000F0415E
:10152000036800221B68184710B503685B6804460F
:10153000984708B194F84D0010BD00002DE9F04126
:10154000664B03F5C04490B094F9042206460F465A
:10155000002A00F0C08094F84C5235B9604A82F0FD
:101560005DFA284610B0BDE8F081B3F9A4201AB99D
:10157000B3F8A220A3F8A420B3F8A430632B05D8B5
:10158000584A3946304682F049FA002500212E2279
:1015900004A80391BFF026F9D4F86401036803AAF4
:1015A0001B6832219847804630B94F4A03AB394611
:1015B000304682F033FA4546B4F84031A3F57A73E9
:1015C0009BB241F65832934206D9484B3A46202105
:1015D000304682F01BF8002594F97433002B69DD46
:1015E00094F92C33002B59DD414B3A4620213046EB
:1015F00082F00CF800253F49D4F87001322303AA89
:101600008DF0ECF9804640B903AB00933A463A4B73
:101610002021304681F0FAFF45463849D4F86C0164
:10162000322303AA8AF00CFA804640B903AB009338
:101630003A46314B2021304681F0E8FF45462021D3
:10164000304681F0DBFFB8B1D4ED707A9FED2C7A93
:10165000F0EEE77AF4EEC77AF1EE10FA0CD594F9D1
:101660007433002B02DD94F8D8332BB9254A394660
:10167000304682F0D3F9002594F97433002B7FF7BC
:1016800070AF94F93132002B3FF46BAF1E4B3A46EA
:101690002021304681F0BAFF002562E794F8D88314
:1016A000B8F1000F06D1194B3A462021304681F09F
:1016B000ADFF454694F92C33002B9CDD94F85D83F7
:1016C000B8F1000F97D1124B3A462021304681F0F5
:1016D0009DFF45468FE7012543E700BF482B0020CB
:1016E0004C4C0D086E4C0D08954C0D08A04C0D0887
:1016F000B24C0D08234D0D08274D0D08394D0D082E
:10170000000000343D4D0D08574D0D08D84C0D0814
:10171000FE4C0D0838B5044681F054FF114B93F888
:101720001013114B1D68EB6A1A68002908BF0146A7
:101730001268184690475BF05DFEEB6A93F89C10C8
:101740005AF044FE94F837305BB193F0FDFFEB6A3A
:10175000D3F8A030C01AB0F5FA6F24BF002384F884
:10176000373038BD488B0020442B002008B5FFF7E8
:10177000D1FF054B05481B68DB6A93F89C10BDE858
:10178000084011F075B900BF442B0020808C002068
:1017900070B50E46054667F0B9F867F07BF810B9EA
:1017A0000124204670BD0A4B93F98A32012BF7D1F0
:1017B00067F0ACF8437A002BF2D167F0A7F8847A8F
:1017C000002CEDD1034A3146284682F027F9E8E79C
:1017D000484B0020704D0D08034BD3F8F4320BB981
:1017E00081F0A6BE01207047484B00202DE9F0474C
:1017F0002DED028BC47F90B006460F468CB990F950
:101800000430002B00F00581834B1D68A86A036833
:101810005B6B9847044650B9804A3946304682F09F
:10182000FDF8204610B0BDEC028BBDE8F087B36830
:101830004BB933685B6B3946304610B0BDEC028B58
:10184000BDE8F0471847E86AFFF76EFE0446002837
:10185000E7D13946304682F05FFFDFF8F481054674
:101860003946304682F002F998EDA77AD8EDA67A8B
:10187000B4EEE77A2840F1EE10FAC5B209D598F92E
:101880009432032B05D0664A3946304682F0C6F8BA
:101890002546D8ED8F7AB0EE088AF4EEC87AF1EEDC
:1018A00010FA0BD517EE900AFEF72EFE5D4ACDE931
:1018B00000013946304682F0B1F80025D8ED907A23
:1018C000F4EEC87AF1EE10FA0BD517EE900AFEF797
:1018D0001BFE554ACDE900013946304682F09EF89C
:1018E0000025D8ED917AB8EE087AF4EEC77AF1EED9
:1018F00010FA0BDD17EE900AFEF706FE4B4ACDE913
:1019000000013946304682F089F80025B8F92832BE
:10191000042B07DC052200923946454A304682F006
:101920007DF80025D8F8B00C67F04CF880B198F934
:101930008A326BB1D8F8B03CB8F98C22B3F90E30CA
:101940009A4205DA3B4A3946304682F067F800256C
:1019500039463046FFF71CFFDFF8F8A081463946CC
:101960003046FFF7EBFD9AF8B53F002B4AD109EA64
:10197000050500EA050430484FF4806101F06AF87B
:1019800078B1D8F8B03CB3F90C30A3F2E24292B28D
:10199000B2F5FA7F05D9294A3946304682F03EF839
:1019A0000024274890F808365BB100F5C06037F096
:1019B000FDFF054628B9234A3946304682F02EF805
:1019C0002C4600212E2204A80DF10C080391BEF034
:1019D00009FFDAF8A00F4246322109F027FD05463B
:1019E00000287FF41EAFDAF8A00F03689B689847C1
:1019F000154ACDF8008003463946304682F00EF88D
:101A00002C460EE7114A3946304682F007F800248A
:101A1000B1E7012405E700BF442B0020804D0D08ED
:101A2000974D0D08BA4D0D08DA4D0D08FC4D0D0807
:101A30001E4E0D083D4E0D08482B0020784E0D0817
:101A4000487B0020A04E0D08101B0E08634E0D08A9
:101A5000484B0020486B002070B505460E46FFF746
:101A600097FE31460446284682F014FD2040C0B25D
:101A700070BD0000F0B591B005460E4682F0ACF89E
:101A80000446D8B11021284681F0B8FDB0B100213C
:101A90002E2204A803AF0391BEF0A4FE1BF030FF7A
:101AA00032233A4601211BF0EBF9044630B9054BCD
:101AB000009732461021284681F0A8FD204611B03B
:101AC000F0BD00BFB44E0D0870B505460E46B1B965
:101AD00090F910408CB1164813F0FAFEDFED157A3C
:101AE000B0EEC00AB4EEE70AF1EE10FA07D4124ADB
:101AF0000121284681F092FF3446204670BDAB6834
:101B00009BB10E4B1B68D86AFFF70EFD044630B13F
:101B100065F050FC0A4A04215EF0C4FDEDE7314651
:101B20002846BDE8704082F023BB0124E5E700BFF2
:101B3000482B002000000034C04E0D08442B00202C
:101B4000D24E0D0838B5044682F096FE0546A8B17F
:101B50000B4806F061FB38B10A490B481BF0E8FA64
:101B600010B1074800F048FF2046FFF7FFFD0123B2
:101B7000064984F83730204682F09EFD284638BD5D
:101B8000482B0020AC8B0020703E0020F44E0D0846
:101B9000F8B505460E461746C2B1232901D00129E2
:101BA00014D8254808F006FF044668B100242046F2
:101BB000F8BD95F91030022B08D065F0FBFB1F4AE9
:101BC00006215EF06FFDF2E7002EF2D03A46314674
:101BD000284682F007FF04460028E7D0184ED6F8C2
:101BE000A02F06F550639A4203D006F5B05038F0A6
:101BF00013FBD6F8A00F134F03689B6B984787F829
:101C0000D80507F58057D7F88831012B07D166F042
:101C10007DFE542167F0D4FD08B9C7F88801284635
:101C2000FFF7A4FD4FF0FF330749C6F8D83F284619
:101C300082F042FDBBE700BF482B0020044F0D0897
:101C4000486B0020487B00201C4F0D082DE9F04F09
:101C50002DED028BDFF8489191B00746884681F060
:101C600079FD99F95F520446D5B9BD2109F558505F
:101C700038F068FA38B1434B42464FF48041384659
:101C800081F0C4FC2C464048BC2138F05BFA38B1E6
:101C90003E4B42464FF48041384681F0B7FC002469
:101CA0003B4E96F84C32002B66D0A6F580531C2292
:101CB000002102A8B3F834A6DFED368ABEF092FD0B
:101CC00004A820F03FFDA6F5206B0125A6F5C0462F
:101CD000554551D20BA820F035FD09AA2946584692
:101CE00035F0D0FE002847D0BDF82610304607F06A
:101CF0007DFF80B3BDF80A30102B2CD104A90BA8AE
:101D000021F082F809F6C853B0EE408A93ED000A3C
:101D10002148B4EEE80AF1EE10FAB8BF99ED8B0A4B
:101D200020EE000A0EF0BAFFF6EE087A60EE277A8F
:101D3000B4EEE78AF1EE10FA0DD517EE900AFEF731
:101D4000E3FB164BCDE9000142464FF48041384693
:101D500081F05CFC00240DF1240CBCE80F000DF1B7
:101D6000080EAEE80F009CE80700AEE8030001355E
:101D70008EF80020ADB2ABE7204611B0BDEC028B6F
:101D8000BDE8F08F304F0D08488100205C4F0D08F2
:101D9000488B002000000034808C00208F4F0D08FD
:101DA000484B002000207047014800F0A5BD00BF4F
:101DB000482B002003685B681847000066F0F4BCFD
:101DC0002FF058BB5AF084BC08F046BF58F088BDCD
:101DD0000DF0EABB14F0E6BF03F00CBB57F01CB9E2
:101DE0001FF014BD69F010BB15F042B813F0EEBD42
:101DF0001FF06AB86BF0CEBA66F0F0B964F0AABB17
:101E000008F0D8B805F07EB90CF0AEBE0DF02EBBD0
:101E100014F002BE15F0DAB813F00ABC14F03CBF9F
:101E200001F0B8BB00F2545021F056BD08F052BC8E
:101E300090F8C432B02202FB030390F8082393F811
:101E4000A13012B1012B28BF0123184670470000B2
:101E500090F814310BB190F84131184670470000EA
:101E6000034808602921117008221A60704700BFDA
:101E7000C0520D08F8B5044604F5995600F5C14066
:101E800070300836FFF746FC002130461BF0AAFCF4
:101E90008021204615F00CFB18B131F06FF92EF0BF
:101EA00003FF04F50055D5ED8F7A9FED317A67EE8B
:101EB000877A05F6C447FDEEE77A04F5C64017EECB
:101EC000903AC5F8C03CD5F844323B60703015F00C
:101ED000F1FCF8B9D5F8C03C07EE903A04F5805310
:101EE00003F2745292ED007AF8EEE77A03F5AE63EE
:101EF00067EE877AFDEEE77A17EE902AC5F8C02CD8
:101F0000D3ED007A97ED007AF0EEE77A67EE877A04
:101F1000C7ED007A04F5B35106F5457035F030F899
:101F200004F5AA4594ED467AD5ED167AE7EE007AE7
:101F3000C5ED167AB0EE670A31F08EFE04F5C240A8
:101F400085ED160A38300DF0B7FF04F5C2400021C8
:101F5000443086F087FC4FF40011204615F0A8FAB3
:101F600020B13046BDE8F84019F05CBDF8BD00BFB7
:101F70000000C842FFF77EBF70B500F580430546FC
:101F8000D3F8A00F03689B6B984705F5C24438341B
:101F90000646204610F02EFD05F5A043002893F8D4
:101FA000973518BF00262BB926B105F535501830E6
:101FB00086F0BCFB204610F0B3F918B92046FFF7B5
:101FC00047FF20B12046BDE8704010F061BF70BDF2
:101FD000FFF7D2BF38B54FF48011054615F068FA07
:101FE000044620B90121284615F062FA0446022170
:101FF000284615F05DFA50B114B9284603F01EF9D1
:1020000005F599500830BDE8384019F009BC002C9E
:10201000F6D138BDFFF7DEBF38B54FF48011044666
:1020200015F046FA01210546204615F041FA18B18F
:1020300015B9204603F002F91021204615F038FAB0
:1020400060B1204603F0EEF94FF48001204615F010
:102050002FFA18B931F092F82EF022FF20212046F5
:1020600015F026FA28B1204603F052FA204603F074
:102070006BFB4FF40051204615F01AFA10B12046C0
:1020800003F04AFB8021204615F012FA28B131F006
:1020900075F8BDE838402EF02BBE38BDFFF7BCBF49
:1020A00010B5044621F008FD90F921308BB190F86D
:1020B000403373B194F978355BB1064B1B68DB6A2A
:1020C00093F89C302BB904F25450BDE8104021F035
:1020D0001BBA10BD442B0020FFF7E2BF2DE9F843E7
:1020E000434B1B68DB6A93F89C300446002B7CD082
:1020F00000F5805797F83136002B76D008F05AFC5F
:10210000002872D004F5FB5507F58059083599F879
:10211000B610284618F028FF002866D004F59076FF
:102120003046FFF785FE02285FD994F8E4334FF07C
:10213000B00808FB034393ED777AF1EE007AB4EE32
:10214000E77AF1EE10FA50D499F8B610284619F053
:10215000BBF904F50053B3F9282207EE902AB8EE34
:10216000E77AB4EEC07AF1EE10FA0CDD94F8E423CD
:1021700008FB0242F8EE677A92ED777AF4EEC77ABE
:10218000F1EE10FA31DCD7F82025D3F8C01C002A74
:10219000B8BF52428A4228DC07F22452D2ED007ABC
:1021A000D3ED906A9FED136AF8EEE77A66EE866AE1
:1021B000F4EEE67AF1EE10FA17DC03F6C44292ED83
:1021C000007A27EE067AF4EEC77AF1EE10FA0CD414
:1021D00094F8E413B02202FB01612846B3F92A22E5
:1021E000D431BDE8F84318F03DBDBDE8F88300BF29
:1021F000442B00200000C842FFF770BF2DE9F041DA
:1022000090F8E4332B4D00EB03132F68D3F894813F
:1022100000F5907604463046FFF70AFE474512D097
:10222000022812D904F58047C5F8008097F8D03FFE
:10223000012B13D815D104F5C045EB6EDBB92B6F1C
:10224000CBB905230BE0022810D804F5804393F89E
:10225000D02F5AB1052283F8D02F07E0013B87F831
:10226000D03F04F5BB5004301CF0FEFC2046BDE816
:10227000F0410CF063BE104B1B68D86A03685B68C2
:10228000984780460028ECD194F8E413B02303FB70
:102290000161AC31204606F031F82B6D0FCB05F112
:1022A0005406743586E80F0085E80F0087F8D08F54
:1022B000D7E700BF382B0020442B0020FFF79EBF3C
:1022C00070B500F5C043044693F84C3200F58056D3
:1022D000BBB100F5C640703015F0F2FD18B1012316
:1022E00086F8313670BD04F5C2453835284610F001
:1022F00017F808B10023F3E72846FFF7A9FD0028E7
:10230000F8D104F5A04393F89725002AF2D1D3F829
:10231000DC35042BE3D104F5BF4014308FF042FCD0
:1023200086F83106DEE7000010B500F5804400F5C0
:102330009A43D4F8A01F994200F5A04308D000F5B5
:102340009D42083291421CBF4FF0FF32C3F8502526
:1023500003F5A8620749116003F24453064A1A6064
:10236000FFF7AEFFD4F8A00F0368BDE810401B696B
:10237000184700BF0000C8420000C8C2FFF7D4BF22
:10238000F7B500F5A0470446D7F8DC358B420D467B
:1023900024D00B1F00F5BF46594206F114065941DF
:1023A000304601918FF0EEFA019930468FF0EAFA4B
:1023B000072D0BD104F55150D7F860256423052172
:1023C00092FBF3F32830064A5EF06CF92046C7F81A
:1023D000DC5503B0BDE8F04003F004B903B0F0BD34
:1023E00020500D0870B500F580460446D6F8A00FC1
:1023F00003689B6B9847B0B104F5A04595F8D835B4
:102400008BB9D6F8A02F04F59A439A424ED104F521
:10241000C246383630460FF09FF960B995F89035CE
:102420007BB9012108E004F5C245383528460FF094
:1024300077FF002840D002212046BDE87040FFF71A
:102440009FBFB5F83E36152B29D195F8981F11F08E
:10245000010122D1D5F8DC35072B1ED004F5C0438D
:1024600093F90E300BB90421E6E7204613F030FA59
:10247000DFED127AB4EEE70AF1EE10FAF3DB04F5C1
:10248000BF4014308FF0CEFA0028ECD004F5515044
:102490000B4A062128305EF005F90721CCE73046CB
:1024A000FFF7D6FC0028C6D10321C5E704F59D43FC
:1024B00008339A42F8D170BD2846F1E70000B442D3
:1024C00044500D0838B5314CD4F8A02F04F55063B2
:1024D0009A422DED028B0546B0EE408A03D00020D3
:1024E000BDEC028B38BD2A480FF036F940B1BDEC87
:1024F000028B05F5C2403830BDE8384010F048BACC
:1025000004F58055D5F8DC35042B35D194F8D13F4E
:1025100033B12049A1F6642038F0F6F80028DFD165
:102520001D4C94F84C325BB104F59C700FF014F91B
:102530000028D4D104F59C700FF0CEF80028CED13D
:102540009FED167AF0EEC87AF4EEC77AF1EE10FA43
:1025500009D49FED130A28EE008ABDEEC88A18EE52
:10256000103AC5F860350F488FF05CFA0028B6D0F5
:10257000002385F89335B3E7B5F83E16A4F58040FF
:1025800007F034FB0028C1D1A9E700BF486B002049
:10259000808C0020AC8B0020488B00200000003491
:1025A0000000C842DC8A002010B52DED028B00F53A
:1025B000A0430446D3F8DC35042B0BD105F01CF8FE
:1025C0002046B0EE408A05F03BF938EE400ABDECFB
:1025D000028B10BD00F5C04494ED280AF7E7000017
:1025E0002DE9F0412DED028B00F586658AB0044699
:1025F00028461DF03BFD04F59950002307A908303B
:102600000793089309931AF079FF002800F08B8054
:102610009DED090ADFED5B7A04F5A04505F5AE6393
:1026200093ED007A20EE270ADFED577AA7EE270A0E
:1026300004F58046204683ED000AFFF7D3FED6F866
:10264000A00F03689B6B9847074604F5C2403830DB
:1026500010F0D0F995F89735002818BF0027002B07
:102660005CD1002F5AD095F8D835002B56D1D5F82B
:10267000DC35042B6ED09FED458A204605F002F92B
:1026800004F5C04204F59A43C2F89C04D6F8A01F92
:102690002C3399421AD192F8E830BBB904F50053B3
:1026A000B3F98C3C002B04DC3949D1F86C1CC90609
:1026B0000CD5176D916D7F680A33C91B64277B4366
:1026C0008142ACBF5B181B18C2F89C34D5F8DC35CE
:1026D000D2F89C14D6F8D42F059120460492039387
:1026E00016F0ECFBB6F9E26F07462046FFF75CFFF9
:1026F000CDE9007604F50050D0EDB11A059905F545
:10270000BF6504F53550F0EE400ADDE9033295ED82
:10271000001AB0EE480A183085F0ACFC0AB0BDECE7
:10272000028BBDE8F08104F59070FFF781FB022871
:102730000AD994F8E433B02202FB034393F8102241
:1027400012B193ED7F0A65E728461DF029FBB1EE33
:10275000400A5FE704F5C04704F5C048643708F154
:10276000740804F5C04142465431384620F0B8FAA6
:10277000002880D04146384620F046FBB0EE408A23
:102780007BE700BFCDCC4C3ECDCC4C3F00000000E1
:10279000484B0020FFF724BFF8B500F5804200F554
:1027A0009B43D2F8A02F20339A4204460E4623D0F2
:1027B00000F5C247383738460FF0B2FD0546A8B1DC
:1027C00038460EF033FA70B104F5C044D4F8740101
:1027D00003689B689847DFED097A20EE270A86EDAB
:1027E000000A2846F8BD9FED060AF8E704F5AA445A
:1027F0000125A36F3360F4E70025F2E70AD7233CF5
:1028000000000000F8B500F5804200F59B43D2F8C7
:10281000A02F20339A4204460E4630D000F5C2471E
:10282000383738460FF07CFD0546A8B138460EF023
:10283000FDF970B104F5C044D4F874010368DB6895
:10284000984707EE900AF8EEE77AC6ED007A284638
:10285000F8BDDFED0C7AF8E704F540540125D4F813
:10286000840603681B69984707EE900A9FED067A75
:10287000F8EEE77A67EE877AC6ED007AE7E700259B
:10288000E5E700BF000000000AD7233CF8B500F5DB
:10289000804200F59B43D2F8A02F20339A42044691
:1028A0000E4624D000F5C247383738460FF038FDC1
:1028B000054688B138460EF0B9F950B104F5C04468
:1028C000D4F8743118698AF0F3FF86ED000A2846BF
:1028D000F8BD9FED080AF8E704F540540125D4F847
:1028E000840603685B69984786ED000AEFE70025D8
:1028F000EDE700BF0000000030B505460FC985B008
:102900006C4684E80F0040F279322146284605F0F3
:102910008FFB0C4B03F66452D3F8A03F93420ED1C9
:102920009DF8001011F0040102D120461FF0D4FFE1
:102930000548214605F030FC012005B030BD0020DF
:10294000FBE700BF486B0020482B002010B5044671
:1029500006480FF019FB40B904F58044D4F8A00FE5
:102960000368BDE810409B6C184710BD808C0020A8
:1029700010B5044606480EF05DFF40B904F58044EA
:10298000D4F8A00F0368BDE81040DB6C184710BDF9
:10299000808C002070B5044600F5C24038300E46E9
:1029A00015460EF0A5FA50B104F5C044D4F8EC3346
:1029B0009B682B60D4F8EC335B68336070BD04F522
:1029C000805303F5A66203F22C5312682A601B6839
:1029D000336004F50054D4F86C3C9B05EED4D4ED80
:1029E000B16AD5ED007A9FED037AE6EEC77AC5EDC0
:1029F000007AE3E735FA8E3C38B50D4D044629469A
:102A00000C481AF0A7FC04F5804305F13C0183F85B
:102A1000D10F04F59950083004F5C0441AF032FB88
:102A2000D4ED287AF1EE677AC4ED287A38BD00BF7C
:102A3000AC8B0020703E002010B5044600F590706D
:102A400029F0BCFB2046BDE81040FFF7D5BF0000D1
:102A5000FFF7F2BF00F50050D0F86C3C194214BFEC
:102A6000012000207047000010B500F580430446A7
:102A7000D3F8A00F03689B6D9847014604F59D406D
:102A80006030BDE8104091F03BBA0000FFF7ECBFAA
:102A900038B5054B1C6823680A461D68034B014680
:102AA0002046A847002038BD442B0020482B00209A
:102AB00070B52DED028B0446036804F500559B6D3F
:102AC0009847D5F86C3C1B0618D5B5F92832B5F9EE
:102AD0002A12CA1A0B4402EBD27203EBD3735210C0
:102AE0005B1000EE902A00EE103A04F59950F8EED3
:102AF000E00AB8EEC00A08301AF04AF85F4BB5F8A1
:102B00005A221A7004F5C14567F014FF703567F05A
:102B1000A3FB00212846FEF769FE594E0123B07140
:102B20002846F37180F04EFD28B9284681F0D8FD83
:102B3000B0FA80F0400930710421204614F0B8FC4E
:102B400020B104F5AD40783057F07CFF284680F086
:102B500039FD04F5C045D8B994F8E43304EB031308
:102B600041F28832D3F89461D5F8EC30F31A9342ED
:102B70000ED904F59070FFF75BF9022808D9C5F863
:102B8000EC60204605F048FB04F5BF4300225A6183
:102B9000B4F9A4301BB9B4F8A230A4F8A430B4F846
:102BA000A430DFED388A07EE903AF8EEE77AB7EE18
:102BB000008A88EE270AD4ED2B7AF0EEE77AF4EE5D
:102BC000E87AF1EE10FA09D5B4F9A23007EE903A9E
:102BD000F8EEE77A88EE277A84ED2B7AD4ED2B0A8B
:102BE00030F03CFF70BB58F0F3FD40F27D124FF423
:102BF000801158F0A5FD56F0C5FA55F02DFF95F857
:102C00004C32B0EE408A23B1D5F86C0103681B6FDB
:102C1000984704F54050B0EE480A143078F0CCFCE8
:102C200004F54550B0EE480A303078F0C5FCB0EEFF
:102C3000480ABDEC028B04F54A502430BDE87040D0
:102C400078F0BABCD4ED2B7A94ED460AF0EEE77A30
:102C5000F4EEE87AF1EE10FA09D5B4F9A23007EEF5
:102C6000903AF8EEE77A88EE277A84ED2B7AD4ED65
:102C70002B0A30F0F3FE0028B5D0BCE7502300202B
:102C80009590002000000034FFF712BF70B500F5EA
:102C9000C046044696F90C30002B2ADD07F08AFE68
:102CA00038BB04F5C1457035284681F019FD00B3E5
:102CB000284680F087FCE0B192F046FD04F5A04381
:102CC0004FF47A72D3F88035C01A96F90C3053431A
:102CD00098420ED301221C212846FEF759FF40B12D
:102CE00004F55150034ABDE87040062128305DF0DC
:102CF000D9BC70BD64500D0800B52DED028B9FED61
:102D00000B8AD0ED4E7A67EE887A83B0C0ED4E7AAA
:102D10003830019078F0AEFC019820EE080A03B03C
:102D2000BDEC028B5DF804EB78F0BCBD52B87E3F81
:102D300000B52DED028B9FED0B8AD0ED4F7A67EE3B
:102D4000887A83B0C0ED4F7A3C30019078F092FCE5
:102D5000019820EE080A03B0BDEC028B5DF804EB8D
:102D600078F0A0BD52B87E3F30B52DED048B0446FF
:102D700083B000F5995001A908301AF091FB0028A2
:102D800000F0B98004F5AA4595ED1A7ADDED017AD7
:102D9000B4EEE77AF1EE10FA05F1680507D504F50F
:102DA000C140703080F018FC08B1019B2B6004F525
:102DB000005595ED9F7AB5F92832DFED606A052B55
:102DC000B8BF052307EE903AB5F92A32F8EEE78A44
:102DD00007EE903AF8EEE77AB6EE009A77EEA77A29
:102DE0001820C7EE270ADFED567A68EEA77AF4EED0
:102DF000490A87EE271AF0EE007AF1EE10FAB4EEE7
:102E0000671AC8BFF0EE490AF1EE10FA48BFB0EEFB
:102E1000671ADDED017AF4EEE67AF1EE10FACCBF36
:102E200087EE270AB0EE410A30F02AFF04F5C240CF
:102E30003830B0EE408A0FF073FA38B904F5C04369
:102E400093F84C22D2B393F87932BBB304F5C14066
:102E5000703080F0C1FB88B328EE892A9DED011AFD
:102E6000B4EEC21AF1EE10FA28D5D5ED9F0ADFEDC7
:102E7000351A9FED350AC0EE820A30F033FE04F5B4
:102E80003F501C30B4EE408AF0EE408AF1EE10FA6A
:102E900048BFF0EE488AFFF72FFF04F54450343066
:102EA00004F54054FFF744FFD4EDF97A9FED277AFB
:102EB00067EE877AB0EE688AC4EDF97A244819F093
:102EC0009DFA90B923484021FFF7C4FD68B1224B19
:102ED000D3F8DC35012B08D1F7EE007AB4EEE78A9F
:102EE000F1EE10FA58BFB0EE678AB0EE480A03B0B0
:102EF000BDEC048B30BD04F5C140703080F06CFB3C
:102F0000B7EE008A0028D9D0462066F0BBFFB4EEA9
:102F1000C80ADFED127AF1EE10FAD8BFB0EE480A17
:102F200087EE800ABBF0AEFB2F209FED0D1ADFED80
:102F30000D0A30F0A5FEB0EE408ABFE717B7D138D2
:102F40003333333F000000006F12833A52B87E3FA4
:102F5000703E0020482B0020487B002000003442B7
:102F60008FC2D53F9A99193FF8B5044665F0CEFC5B
:102F70000368DB689847054610B900252846F8BD68
:102F800004F58046204607F093FBD6F8A02F04F501
:102F90009C4330339A42074605D104F5C04393F869
:102FA0000C33022BE9D804F5C24038300FF0DEFBB9
:102FB0000028E2D1D6F8A00F03689B6B984758B958
:102FC00096F8B43F002BD9D004F5005494F99452EC
:102FD000023D18BF0125D1E7084BD3F8A00F0368C5
:102FE0005B6B98470028EBD004F5005494F9D1327C
:102FF000002BC2D0032BC0D03D46BFE7486B00205A
:1030000070B52DED028B044600F5804600F5C240F8
:1030100006F57F6382B0383093ED008A0FF0BAFA7C
:1030200004F53F551C35002846D104F5C046D6F8B6
:103030006C0103689B689847D6F8FC335B0225D582
:10304000D6F86C3193ED437AD3ED097A67EE877A3F
:103050009FED327AF4EEC77AF1EE10FA16DB04F542
:10306000005404F57E6393ED007A67EE877AF7EEFD
:10307000006A86EEA77A04F6DC74B4EE667AF1EEA6
:1030800010FAC8BFB0EE667A84ED497ADFED247A93
:1030900090ED250AF0EE480A20EE270A284682F035
:1030A000B9F928468DED010AFFF726FE9DED010ACC
:1030B00002B0BDEC028B70BDD6F8A02F04F598438A
:1030C00010339A4228D104F50053D3F8A83CB3F941
:1030D0000860003E18BF012604F5A04204F58054A4
:1030E000D2F8F035D4F820451C1B92F8EC353BB1F2
:1030F0000C484FF40061FFF7ADFC80F00100C3B253
:103100003246B0EE480A2146284602B0BDEC028B9A
:10311000BDE8704082F082B90026DDE7000000348F
:10312000E02E6542482B002010B5044606F084FED0
:1031300098B104F5A042D2F8F03503F58C41503136
:10314000C2F8F01504F58051D1F820150029BEBF52
:10315000A3F58C43503BC2F8F0352046FFF750FFF3
:10316000BDE81040042066F079BE00002DE9F0476C
:1031700000F5C2442DED048B00F580493834054636
:1031800009F57F632046D3ED008A0FF003FA05F5B9
:1031900044563436002844D105F5C044D4F86C01B7
:1031A0000368DB689847D4F8FC335B0221D5D4F878
:1031B0006C3193ED447AD3ED0B7A67EE877A9FED0D
:1031C000537AF4EEC77AF1EE10FA12DB05F54055AA
:1031D00095ED4E7A67EE877AF7EE006A86EEA77A6B
:1031E000B4EE667AF1EE10FAC8BFB0EE667A85EDFD
:1031F000977A90ED250ADFED467AF0EE680A20EE28
:10320000270A304681F060FD3046B0EE408AFFF775
:103210008FFDBDEEC80ABDEC048BB8EEC00ABDE858
:10322000F087204605F500580DF02EFD9FED399AE8
:1032300098EDB18A28EE098A05F5A047BDEEC88A47
:10324000D7F8F43518EE102A1A4408EE102A8246F0
:10325000462066F017FEB8EEC88AD8ED9B7AD9F8FA
:10326000A00FA0EE278A05F5984310339842FDEE93
:10327000C87A17EE904A45D1D8F8AC3CB3F908802B
:10328000B8F1000818BF4FF00108BAF1000F1ED1C5
:1032900003685B699847D0B9D9F8A00F03689B6BA6
:1032A0009847A0B905F5C043D3F89434022B0ED14A
:1032B000284612F055F950B107F6EC73D3ED007AB9
:1032C00067EE897AFDEEE77A17EE903A1CB205F5C3
:1032D0008055D5F82435E41A97F8EC353BB10E4803
:1032E0004FF40061FFF7B6FB80F00100C3B2B0EE0F
:1032F000680ABDEC048B424621463046BDE8F047E3
:1033000081F0C8BD4FF00008BFE700BF00000034E7
:10331000E02E65420000C842482B002010B504464C
:1033200015F014FF68B100B200EB4000C0EB0013D1
:1033300000EE103AB8EEC00ABDE81040132066F067
:103340008DBD2046FFF712FFF6E7000010B51048CC
:10335000FFF70AFED0B10F480FF042FBB0B10E4CA0
:10336000042066F08FFDD4F8A80C65F03FFD042022
:1033700066F074FD132066F085FDD4F8AC0C65F0A2
:1033800035FDBDE81040132066F068BD10BD00BFDC
:10339000482B0020808C0020484B0020F8B52DEDF4
:1033A000028B0446FFF7E0FD002800F0AB8004F537
:1033B000804704F59842D7F8A03F4832934200F086
:1033C000A18004F599420432934200F09B8004F5F9
:1033D00099426432934200F0958004F5994220327C
:1033E000934200F08F8004F599423C32934200F002
:1033F000898004F59B423C32934200F0838004F5BF
:103400009B42583293427DD004F59B4274329342E2
:1034100078D004F59C421432934273D004F59C4258
:10342000503293426ED004F5C24038300FF0D8FAD3
:10343000002867D0D7F8A02F04F598432C339A4280
:1034400060D004F50055F6EE008AD5F8A80C65F0BA
:103450008DFBB4EEE80AF1EE10FA40DDB0EE087A2A
:10346000FFEE007AE0EE077AB0EE670AD5F8C02CDE
:1034700004F5A04607EE902AD6F8F035B8EEE77AC4
:1034800007EE903AF8EEE77A5142E7EE007AFDEE69
:10349000E77A17EE900AC6F8F00530F091FCC6F80E
:1034A000F005D7F8A02F04F59A4348339A4222D06A
:1034B000D5F8AC0C65F05AFBB4EEE80AF1EE10FA60
:1034C000B0EE408A21DCFEEE007AB4EEE70AF1EEBF
:1034D00010FA22D5B0EE087AF7EE007A19E0FEEE87
:1034E000007AB4EEE70AF1EE10FABFD5B0EE087A32
:1034F000F7EE007AB6E725484FF48051FFF7AAFAB5
:103500000028D5D0BDEC028BF8BDB0EE087AFFEEF6
:10351000007AE8EE077AB0EE678A204606F08CFC67
:1035200008B1B1EE488AD6F8F435D5ED906A9FED32
:10353000186A05F6C44595ED007AB5EEC08A07EE27
:10354000903AF1EE10FACCBF28EE268A27EE488A90
:10355000F8EEE77A66EE866AE8EE067A27EE067AF5
:10356000FDEEE77AFDEEE66A17EE903ABDEEC77A19
:1035700016EE902A17EE101A17EE900AC6F8F435D8
:1035800030F01EFCC6F8F405BCE700BF482B002055
:103590000000C842F8B5044604F5C04792F0D4F8DC
:1035A00097F84C32064653B1D7F87402036804F515
:1035B000AB4204F5AB411B6A70327431984704F595
:1035C0008045D5F8B03FF31AB3F5FA6F03D9D5F8B3
:1035D000A00F07F045FF2C4BC5F8B06FD3F8A00F34
:1035E0000268136898470021204612F071F9DFED58
:1035F000277AB0EEC00AB4EEE70AF1EE10FA42D52F
:10360000D7ED287AB1EE047AF0EEE77AF4EEC77AD5
:10361000F1EE10FA37D504F586601CF0C1FBF6EE2A
:10362000007AB0EEC00AB4EEE70AF1EE10FA2AD53D
:1036300004F5B95595ED037AF0EE087AB4EEE77A21
:10364000F1EE10FA05F10C051DD504F53F501C30C4
:1036500081F054FF04F54450343081F0CBFC04F584
:103660004A500C3082F0F8FB95ED007AF7EE007AC4
:10367000B4EEE77AF1EE10FA05D504F55050BDE846
:10368000F84082F03FB9F8BD486B002000000034DC
:1036900000F5005090F91F32012BC3BF00F65850BF
:1036A00090ED290ADFED047A9FED040AC8BF20EEF1
:1036B000270A462066F0D2BB0000C8420000000086
:1036C0002DE9F8432DED028B00F5804909F57F6364
:1036D000D3ED008A054611F047FD8046D9F8A00FCA
:1036E00003681B6A984705F54A560C3698B14F4C4B
:1036F000D4F8BC35002B0EDD92F026F8D4F8BC359A
:10370000C01A40F6B733984205D8B4F9B0453046F0
:1037100082F0AEFB7AE005F5C04305F5005793F85B
:10372000893443B1B7F9B032002B04DD05F54053BD
:1037300093F9A23203BBD9F8A03F05F5984510359F
:10374000AB426DD00021B0EE680A304682F028F915
:103750000546042066F096FB2BB207EE903A97EDF3
:10376000997AF8EEE77AE0EE077AFDEEE77A17EE5F
:10377000904A444424B2CAE72846012111F0E6FEEB
:103780009FED2B7AB7F9B032C0EE077A05F5A04568
:1037900005F2FC5508EE103A55F80C3C9FED250A51
:1037A000B8EEC88A28EE278A07EE903AF8EEE77A54
:1037B00067EE807A9FED200A27EE800ABAF086FD38
:1037C000B7F92832DFED1D7A95ED007A20EE270A51
:1037D00007EE903AF8EEE77A0021B4EEE77AF1EEE0
:1037E00010FA58BFF0EE477A80EE277A3046DFEDC8
:1037F000147AB0EE480AA7EE270AF0EE680A82F0C3
:103800002BFABDEEC00A10EE103A1CB2BDEC028BD2
:1038100020460C49BDE8F84341F2941230F0E0BA7A
:10382000B8F1000118BF01218DE700BF487B0020DF
:1038300000A08C450AD7233C35FA8E3C0AE81C418F
:10384000E02E65426CEEFFFF38B500F540530546AB
:10385000D3F884060368DB689847014605F55050A5
:1038600082F032F804B22846FFF77EFB70B107EE13
:10387000904A05F50055B8EEE70AD5F8B40C65F0A6
:10388000B5FABDEEC00A10EE103A1CB2204603494C
:10389000BDE8384041F2941230F0A2BA6CEEFFFF5E
:1038A00038B590F8E433B02202FB030393ED777A46
:1038B000F7EE007AB4EEE77AF1EE10FA054600F57D
:1038C000A0441DD5002112F003F8DFED417AB0EEDF
:1038D000C00AB4EEE70AF1EE10FA11D5D4F8DC35DF
:1038E000012B0DD0072B0BD0002384F8543504F5A1
:1038F000AB64002323602846BDE8384011F034BC97
:1039000091F022FFD4F85C35C4F85C05C31AB3F516
:103910007A7F84BF002384F85435284611F024FCB4
:10392000D4F8DC35012B07EE100A2CD0072B2AD057
:10393000B8EEC77ADFED276AC7EE267A05F50052A2
:10394000B2F9742200EE102AB8EEC00A27EE800AFF
:10395000DFED1F7AB0EEC07AB4EEE77AF1EE10FA3E
:1039600013D4002384F8543594F8543505F5505099
:10397000DBB981F091FEBDE83840174900B241F251
:10398000941230F02DBA9FED150A94F85425002AB0
:10399000EAD10122934284F85425E5D0072B1EBFBB
:1039A00004F5AB6300221A60DEE704F5AB6494ED26
:1039B000007ADFED0B7A67EEC77A9FED0A7A67EE41
:1039C000877AFDEEE77A17EE901A81F07DFFD2E755
:1039D0000000003400A08C456CEEFFFF00000000EA
:1039E000E02E65420000C84270B52DED028B00F557
:1039F000BF46143682B0044630468DF043FF05467C
:103A0000D8B904F50053D3F8A82CB2F9082072B93C
:103A100004F5C042D2ED287A93ED9C7AF0EEE77A75
:103A2000F4EEC77AF1EE10FA4CBF012500253046BE
:103A30008DF03CFF002808BF002530468DF022FFA6
:103A400050BB04F5A043D3F8503501331ED01DBB45
:103A50009FED1C8A2046FFF733FE07EE900AB8EE72
:103A6000E70A8DED010AFDB9152066F0F7F99DED25
:103A7000010A1A2066F0F2F904F5C340403002B0A2
:103A8000BDEC028BBDE8704003F00EBB002DDFD013
:103A90002046FFF705FF02E02046FFF7D5FE07EEC0
:103AA000900AB8EEE78AD5E71A2066F083FC9DED10
:103AB000010A08B9B0EE480A152066F0CFF9B0EE59
:103AC000480AD6E70000000010B500F5005303F6E1
:103AD000C442D3ED906ADFED127A92ED007A9FED49
:103AE000116A03F6585366EEA76A27EE277AD3EDDC
:103AF0002A7A67EE867AFDEEE66ABDEEC77AFDEEBB
:103B0000E77A044616EE902A17EE101A17EE900A7E
:103B100030F056F904F5A044C4F8F40510BD00BF18
:103B20000000C842A00CB34510B5044613F0C4FC15
:103B3000031E2ADB04F5005191F91F229A4224DD6D
:103B400004F5A040D0F8DC45022C1ED0D1ED9E7AC1
:103B5000DFED0E6AD31A66EEE76A07EE102A07EE6B
:103B6000903AB8EEC77AF8EEE77AD0F8F43587EEF7
:103B7000876A07EE903AF8EEE77AE6EE867AFDEE8F
:103B8000E77A17EE903AC0F8F43510BD0000C8424D
:103B900070B52DED028B00F5A0459FED550AD5F8C7
:103BA000F0359FED547A07EE903AF8EEE77A044646
:103BB00067EE807A9FED500AF0EEE76AF4EE476A0E
:103BC000F1EE10FAC8BFF0EE477A27EE800ABAF09D
:103BD000EDF92FF077FFB7EE008AC8EE007A05F511
:103BE000BF6304F50056C3ED007A04F5C04393F8B3
:103BF0004C229AB1D3F87402036804F533515B6A1E
:103C0000984758B1D6F8C02CD5F8F005514230F09D
:103C1000D7F8C5F8F005BDEC028B70BD96F95032AF
:103C2000002BF8D0204606F007F90028F3D104F560
:103C3000C640703013F03EFE0028ECD1B6F92832B1
:103C4000012BB8BF012307EE903A05F2FC52F8EEC3
:103C5000E77AD2ED006A86EEA77AB4EEC87AF1EE82
:103C600010FA13D840F6C4122449D5F8F00530F004
:103C7000A7F8C5F8F005D6F8C02C40F6C4139A4250
:103C8000D4BFC6F8C02CC6F8C03CC4E705F5BF6376
:103C9000D3ED007AF4EEC77AF1EE10FABBDD88EED0
:103CA000070A20EE000ABAF03BFBDFED157AD5F8E3
:103CB000F00520EE270ADFED137A20EE270A40F602
:103CC000C413FDEEC07A17EE904A9C42B8BF1C4662
:103CD0002246614230F074F8C5F8F005D6F8C03CD1
:103CE000A342D4BFC6F8C03CC6F8C04C93E700BF9F
:103CF0000AD7233C0000AA4235FA8E3C3CF6FFFF6F
:103D0000E02E65420000C84210B500F5405304465D
:103D1000D3F8840603681B68984704F50053D3F86A
:103D2000C02C514230F04CF804F5A043C3F8F00524
:103D30002046BDE81040FFF72BBF00007047000091
:103D4000012070470820704701207047014B93F80D
:103D50005C027047484B0020034B93F9600A00381F
:103D600018BF0120704700BF484B0020014B93F95A
:103D70005E027047484B002013B5064BD3F8A00FE6
:103D80004B690468009308310EC9646CA04702B007
:103D900010BD00BF486B0020704700007047000056
:103DA00038B5264DD5F8A00F03685B6898471928E9
:103DB0003CD8DFE800F00D39370D0D373737373B8A
:103DC0003939393939393B37373737393B0D393993
:103DD00040241B4B93F8612412B193F860340BB963
:103DE00044F01004174BD5F8A02F9A42A3F11C03FE
:103DF00003D09A4218BF44F01004134991F9D1023C
:103E0000B0B19A4216D0032803D101F534518A4249
:103E100001D144F040040D487FF0D4FB50B144F090
:103E2000800407E01024D4E71824D2E70124D0E767
:103E30009A42F0D144F0010038BD00BF486B002029
:103E4000485B0020E8780020484B0020388C002098
:103E500008B5044806F0AEFD00280CBF0120022082
:103E600008BD00BF482B0020F0B52DED028B8BB0B4
:103E7000054619F045FD4FF48071D0F8047290EDBD
:103E8000828AD0F80C6204461948FEF7E3FD30B987
:103E9000184BDFED197A93EDB17AA7EE678A1748D0
:103EA0000DF026F830B1164BD3F8EC335F6893ED84
:103EB000028ADE682D7C91F047FCD4F81823D4F8F0
:103EC0001C33D4F814130892099327221C23CDE93C
:103ED00000320390079103AA1E21284604978DED16
:103EE000058A06965DF0FCFB0BB0BDEC028BF0BDC5
:103EF000482B0020484B002035FA8E3C808C002057
:103F0000488B002038B5C5780B46352D044628BFB0
:103F10003525352200211846BCF064FC2A4604F100
:103F20000C01BDE83840BCF013BC000008B50248E5
:103F300013F0C2FA00B208BD482B002037B50D4679
:103F4000134840F2EF2204F073F82C7814F00404C4
:103F50000AD0696803220F481EF0FAFB0C4803B030
:103F6000BDE8304003F0B8B901AA214628461EF04A
:103F7000C3FC0028F2D0DDED017A9FED077A67EEF1
:103F8000877A2246FDEEE77A17EE901AE3E700BF44
:103F9000482B0020BC8B00200000C84210B5054C07
:103FA000012384F863345FF01DF8002384F8633440
:103FB00010BD00BF485B002062F07AB92DE9F041E6
:103FC0002DED028B4FF0000882B0CDE900281E4F86
:103FD0009FED1E8A0C461546B0EE480AB1F9022044
:103FE000D7F8A81C4FF47A73064662F03BFC012315
:103FF000CDE90053B4F90020D7F8AC1CB0EE480A64
:1040000030464FF47A7362F02DFCB4F90420D7F8EF
:10401000B01C9FED0F0A43463046CDE9005862F0D0
:1040200021FCCDE90058B4F90620D7F8B41CB0EE55
:10403000480A4FF47A73304662F014FC02B0BDECCB
:10404000028BBDE8F08100BF484B00200000FA441D
:1040500000007A4410B5074B93F9F82640F24D342E
:1040600040F24D13002A08BF1C465EF0B3FD20430A
:1040700010BD00BF487B002010B504461EF09CFF19
:10408000204610BD10B50B4C002384F893355FF02B
:10409000A3FC54F8602CA4F540739A4208D194F81C
:1040A00004362BB904F5C060BDE8104036F086BA7E
:1040B00010BD00BF487B002013B5124C94F8B61019
:1040C000A4F1980016F050FF78B194F8B610A4F15E
:1040D000980017F0B7F940B194F8B610A4F1980021
:1040E00002B0BDE8104017F0EFB919F009FC01A9C2
:1040F00019F0D6F918B19DED010A02B010BD9FED7F
:10410000020AFAE7484B002000000000044B93F835
:104110004C0220B1D3F8740203681B6B1847704738
:10412000488B002008B5084BD3F8502C002A03DC3C
:10413000BDE808405EF092BD03F537605BF014FE09
:1041400090ED000A08BD00BF484B002008B512489A
:10415000D0F8A02F00F684539A4216D0B0F9B83F99
:10416000ABB900F5805393F81D2582B990F8B52FAF
:104170006AB993F8C93563B9A0F5804006F01AFC16
:1041800000280CBF0320042008BD0220FCE7052006
:10419000FAE70620F8E700BF486B002010B5214B76
:1041A00003F55A62D3F8A03F934290B0044636D04C
:1041B00000231D4802931EF0B5FA014618B91A48AB
:1041C00002AA1EF0FBFA247C91F0BEFA174BDDED3B
:1041D000027A9FED177AD3E91F2305930023F8EEA7
:1041E000E77A0793089309930A930B930C930D9323
:1041F0000E934FF6F853ADF83C300023CDE903029F
:1042000067EE877A96228DF83E303323CDE900326F
:10421000572103AA2046CDED067A5DF061FA10B071
:1042200010BD00BF486B0020BC8B0020488B0020D5
:104230000AD7233CF0B58DB0044691F085FA184AB0
:10424000D2F87032C31A642B28D8D2F86C3102909D
:10425000D3F88C10D3F89020D3F88460D3F888502A
:10426000D3F8DC70D3F894E0D3F898C0D3F89C303E
:10427000099300238DF82C30069225231622CDE9D0
:1042800000320591207CCDF81CE002AA5321CDF824
:1042900020C00A97039604955DF022FA0DB0F0BD98
:1042A000488B002010B55EF0DFFE044678B909485F
:1042B00050F8602C80F89345A0F540739A4206D1DF
:1042C00090F804361BB900F5C06036F077F9204647
:1042D00010BD00BF487B00202DE9F0472DED088B75
:1042E0008B4CD4F8A02F04F55A639A4290B005463F
:1042F00000F0E7808748DFED888ADFED889A9FED40
:10430000889A0CF0F5FD002867D082480CF08EFCEE
:10431000002862D004F500589FED820AD8F86C019D
:104320006C3032F0B1FD08F5A270B0EE60AAB0EECC
:10433000418ACDED070A8DED081AF0EE40AA8DED09
:10434000060A84F0E3FAD8F870310146D3F85C230A
:10435000D3F85833059204A8049332F095FB09A8CA
:104360008DED090AB0EE680ACDED0A0A32F09CFB29
:1043700028EE288A02A8BDEEC88A95F81090CDEDE7
:10438000030A18EE103A8DED020A1EB232F000FC5C
:10439000DFED657A20EE270A02A8BDEEC00A6AEEBC
:1043A000A8AA10EE103A1FB232F03CFCB4EEE90AB3
:1043B000F1EE10FA58BFB0EE690ABCEEC00AD4F8AC
:1043C000A02F10EE103A9DB204F6BC539A422AEE8A
:1043D00028AA7BD1DFED558A7EE0DFF854A195F85D
:1043E0001090DAF884760AF500583846D8F8F03597
:1043F00007EE903AD8F8F435B8EEE7BA07EE903AFF
:104400003B689B68F8EEE7AA984707EE900AF8EE3B
:10441000E77A384667EEA87A08F5AF68FDEEE77AE6
:1044200004F6DC7417EE903A1EB23B681B6998479D
:1044300007EE900AF8EEE77A98ED00AA67EEA87A00
:10444000B4EEE9AAFDEEE77AF1EE10FA17EE903A33
:10445000DFED327AAAF5405058BFB0EE67AA1DB220
:1044600003F01EF83B68D4ED007A5B6908EE100A91
:10447000384627EE899A9847B8EEC88ABCEECAAA91
:104480002BEE28BA6AEEA8AA1AEE103A68EE288A2D
:104490008DED09BACDED0AAACDED0B8A8DED0C9A02
:1044A0008DED0D0AADF83860ADF83A50ADF83C30FE
:1044B000B7221A23CDE900323E2109AA48465DF011
:1044C0000FF910B0BDEC088BBDE8F087D8F870315B
:1044D000D3ED0F7A67EEA88AD8F8743104F6DC744D
:1044E000D4ED007A186927EE899A89F0E1F9CDEDCB
:1044F00009AA8DED0AAACDED0B8A8DED0C9A8DEDF2
:104500000D0AADF83860ADF83A70ADF83C50CFE721
:10451000486B0020808C00200AD7233C00FF7F4797
:104520000000C8429F0CB345E02E65420000000029
:10453000485B002001480CF08BBB00BF808C002042
:1045400008B5034BD3F8A00F03685B68984708BD14
:10455000486B002030B587B0054619F0D1F9044604
:104560002D7C91F0E5F8D4F88422D4F888320492B6
:10457000059300211023CD22CDE900320290039152
:1045800002AA42F60C3128465DF0AAF807B030BD09
:1045900030B52DED028B89B0054619F0B1F900F563
:1045A0005A7393E8070002AC84E80700DDED020AC5
:1045B0009DED030A2D7CF1EE600AB1EE400AB9F0E0
:1045C00017FF2046B0EE408A33F0E2F8DFED0B7AB9
:1045D000049B079328EE278A0C230122CDE90032A1
:1045E000A82105AA28468DED058A8DED060A5DF005
:1045F00077F809B0BDEC028B30BD00BFE02E6542FC
:10460000282938B5054623D007D824292BD02729B7
:1046100011D01B2908D1012413E0432937D008D831
:104620004029F8D0422928D02846BDE8384062F019
:104630004BBC5329EEE712215CF050FA044610B946
:104640000024204638BD297C134855F03BF9F8E793
:1046500016215CF043FA04460028F1D0297C0E486C
:1046600055F00AFAEDE70C215CF038FA0446002810
:10467000E6D02846FFF78CFFE3E710215CF02EFA26
:1046800004460028DCD02846FFF764FFD9E7017C08
:1046900002488DF0F5F8BEE740820020DC8A002059
:1046A000F0B52DED028B05468DB01646B0EE408A72
:1046B0000C46002930D0007C5CF0A8FF0746287C1F
:1046C0005DF0A8FE00F121039F4207D2287C0DB0C7
:1046D000BDEC028BBDE8F0405CF0EEB96369089375
:1046E000636A2269CDF82530236AA069E1680792E0
:1046F000CDF829306222212327680590CDE90032C8
:104700000691287C0397192303AAC2218DED048A00
:104710008DF824605CF0E4FF0DB0BDEC028BF0BDC1
:10472000F8B54B4CD4F8A02F04F55A639A420546CD
:1047300000F08C80A4F50056B6F80233DF0713D5DD
:1047400044480DF0EDFD002879D004F50054D4F86C
:104750006C0103689B68984700F1940191ED010A90
:1047600001222846FFF79CFFB6F802339C0712D5BA
:1047700038480DF0D5FD002864D0374BD3F86C01D4
:104780000368DB68984700F1940191ED010A022269
:104790002846FFF785FFB6F80233580712D52D4893
:1047A0000DF0BEFD00284FD02B4BD3F86C010368F1
:1047B0001B69984700F1940191ED010A03222846F4
:1047C000FFF76EFFB6F80233190708D523490B46E9
:1047D00093ED000A043905222846FFF761FFB6F879
:1047E0000233DA0616D51E4FD7F8DC35042B11D16B
:1047F00019F086F8044607F694708DF071F894ED80
:10480000C70ADFED187A014620EE270A062228465D
:10481000FFF746FFB6F802339B0617D50D480DF09B
:104820007FFD98B10C4BD3F87011284691EDAB0A7F
:10483000BDE8F840042201F52A71FFF731BFA4F664
:10484000FC618BE70849A0E70849B5E7F8BD00BF60
:10485000486B0020808C0020488B00207C5F00206B
:10486000487B0020E02E6542A85D00201C5F0020F0
:1048700070B504460E4627F0DFFC90F8C412B02352
:1048800003FB0101AC31204603F038FD0546C0B101
:104890003EB119F035F890F87C3243F0020380F80D
:1048A0007C3204F58043D3F8A00F04F59A432C33EF
:1048B000984204D004F59C443034A04201D106F063
:1048C000F3FC284670BD000073B5164601910446FE
:1048D00019F016F8019918F02BFC0546C0B13EB14D
:1048E00019F00EF890F87C3243F0020380F87C3225
:1048F00004F58043D3F8A00F04F59A432C33984273
:1049000004D004F59C443034A04201D106F0CCFC24
:10491000284602B070BD000030B5054685B00C4693
:10492000D1E9040130F0A6FA40B168461DF00AFF53
:104930006A462146284661F005FF08B9022067E073
:10494000344840F24F32694603F072FBD4ED037AEB
:10495000F4EE677AF1EE10FA22D69FED2F7AF0EEA0
:10496000E77AF4EEC77AF1EE10FA54BF0122002282
:104970009DF80030294962F3410368468DF8003004
:104980001EF04AF80028D9D1254869466DF01AFD75
:1049900040B958F02FFD0522162158F0E3FACDE773
:1049A0000022E5E7D4ED017AFDEEE77A17EE903AC2
:1049B000DB0706D41B4B03F66452D3F8A03F9342A7
:1049C00025D119491348022212F082FB9DF80010EC
:1049D00011F0040102D168461DF07EFF0D486946C2
:1049E00003F0DAFB94ED020AB4EE400AF1EE10FA9D
:1049F0000BD6B5EEC00AF1EE10FA06DD9DF80010F8
:104A00000948C1F3400107F03FFE002000E0042008
:104A100005B030BD482B002000000034AC8B0020D6
:104A2000684C0020486B0020AC78002010B52DEDBC
:104A3000028BD1ED017A91ED008AFCEEE77A8AB023
:104A4000CDED037A9DF80C1005AA044661F064FED2
:104A5000C8B1DFED0E7A059B009368EE277A00223D
:104A6000FDEEE77A114617EE903A06A81DF08AFE91
:104A700023682046D3F8C43006A9984700200AB01E
:104A8000BDEC028B10BD0220F9E700BF0000C84258
:104A900037B5124DD5F8A00F03681B6A0C4698472E
:104AA00040B9D5F8A02F05F550639A4202D00420F2
:104AB00003B030BDD4ED007AD4ED020A94ED010AC2
:104AC0000748FCEEE77ACDED017A9DF8041004F07A
:104AD000ABF80028EBD00020EAE700BF486B0020CD
:104AE000482B0020134610B524220C4618460021FE
:104AF000BBF078FEA27F8277E27FC277072280F840
:104B00002020A28B8283D4ED067AF1EE677AC0ED85
:104B1000067A10BD10B48C8B162C03D15DF8044BB3
:104B2000FFF7E0BF5DF8044B61F034B808B591F8C9
:104B30002030072B0ED1094890F84C3243B191ED4B
:104B4000060A00F59C70B1EE400A0DF0B1F918B9F3
:104B5000042008BD0220FCE70020FAE7488B002073
:104B600008B5D1ED007A9FED087A0848F0EEE77AB3
:104B7000F4EEC77AF1EE10FA54BF0121002105F0DE
:104B800055F9002008BD00BF00000034482B00206C
:104B90001FB5D1ED017AFCEEE77A0B46CDED027A36
:104BA000D1ED007A1A7C017C0192FCEEE77A0B4889
:104BB000CDED037AD3ED027AFCEEE77A17EE902A78
:104BC00092B2009293ED030A9DF80C209DF80830F4
:104BD00009F074FE05B05DF804FB00BF808C002076
:104BE00007B5D1ED007A0848FCEEE77ACDED017A01
:104BF0009DF804100BF032FC00280CBF04200020AC
:104C000003B05DF804FB00BF808C002070B58B8B77
:104C1000C02B05460C4633D8B12B0DD8142B00F011
:104C2000AA80162B53D0112B00F0A18021462846D4
:104C3000BDE8704062F0E0BFB23B0E2BF6D801A198
:104C400051F823F0BD4C01082D4C01082D4C0108F2
:104C50002D4C01082D4C01082D4C01082D4C01084C
:104C60002D4C0108B34C01082D4C0108E74C0108FC
:104C7000234D01082D4C0108D74C0108A94C01080F
:104C8000B3F5967F58D007D8D12B1CD0D42BCDD1DB
:104C9000BDE87040FFF764BF40F6B836B342C5D1F7
:104CA000BDE87040FFF79CBF2146BDE87040FFF7AC
:104CB00033BE2146BDE87040FFF7B8BE2146BDE8CF
:104CC0007040FFF7E5BEBDE87040FFF761BFBDE88B
:104CD0007040FFF72BBF94ED000A2948FDF7F2FB67
:104CE000E8B100201CE0274C94F8D13FBBB1264925
:104CF00004F5B05035F060FD88B104F58053012211
:104D000083F8392604F550610222A4F5804012F0A0
:104D1000DFF90028E5D11D4B002283F83926042055
:104D200070BD184C94F8D13F002BF8D0164904F50B
:104D3000B05035F0C5FCDFE7D1ED007A9FED147A75
:104D4000F0EEE77AF4EEC77AF1EE10FA16D5D1ED6F
:104D5000017AF0EEE77AF4EEC77AF1EE10FA0DD5AB
:104D60000C490222A1F59A4012F0B2F9B9E70A49BA
:104D700002220348F8E709490222FAE70220CFE7B6
:104D8000482B0020486B0020AC8B0020487B002083
:104D900000000034487800209078002074780020CB
:104DA00070B5434B03F66452D3F8A03F93428EB0E4
:104DB0000C467BD1CD78272D28BF2725272200211F
:104DC00004A8BBF00FFD2A4604F10C0104A8BBF0B7
:104DD000BFFC059B9DF836400093069B0193E4437E
:104DE000079B0293E4B2089B03938DF8364090F042
:104DF000ABFC14F0810F04F08705064601D1802D2D
:104E000013D1684631F0AAFBDFED2A7A2A4B20EE57
:104E1000270ADFED2A7AC3F8B46520EE270ABDEE33
:104E2000C00A10EE102AC3F8A82514F0820F01D191
:104E3000802D13D1684631F0ABFBDFED1E7A1E4B9F
:104E400020EE270ADFED1D7AC3F8B86520EE270AA9
:104E5000BDEEC00A10EE102AC3F8AC2514F0840F82
:104E600001D1802D13D1684631F0A2FBDFED117A1C
:104E7000114B20EE270ADFED117AC3F8BC6520EE56
:104E8000270ABDEEC00A10EE102AC3F8B02563064B
:104E90000CD5DDED0C7A9FED097A074B67EE877A2A
:104EA00003F5B862C2ED007AC3F8C4650EB070BDF8
:104EB000486B0020E02E6542487B00200000C8427D
:104EC00030B51E4C91B0084602A9FFF71BF8D4F884
:104ED000A02F04F664539A422DD19DF83C30072B45
:104EE00029D104F50054D4ED1E7ADDED056A9FED5D
:104EF000147AF8EEE77AE6EEC77AFDEEE77AC4EDCB
:104F00001E7A62F057FA226DA36F52689FED0D7AF8
:104F10009B1A07EE903AF8EEE77A054667EE877A35
:104F200017EE900AFBF7F0FA074ACDE900010621D7
:104F300028465BF0B7FB11B030BD00BF486B0020C6
:104F40000000C8420AD7233CFC550D0810B51D4B84
:104F500003F66452D3F8A03F9342044696B0084645
:104F60000FD108A9FEF7CEFF9DF8541003AA2046E2
:104F700061F0D2FB38B962F01DFA134A04215BF0EC
:104F800091FB16B010BDBDF8503023F004039BB266
:104F9000002BF6D0DDED0B7A9FED0C7A039B00938E
:104FA00067EE877A0022FDEEE77A114617EE903A17
:104FB00004A81DF0E7FB236804A9D3F8C4302046F9
:104FC0009847DEE7486B002010560D080000C842E5
:104FD00030B48D7A4B7A43EA0523CD7A43EA054310
:104FE000562B04460A461BD008D8522B12D0542BFD
:104FF00013D02046114630BC61F096BC03F180739B
:10500000863B23F07F43012BF3D8017C064830BC5C
:1050100054F0FABD30BCFFF7C3BE30BCFFF750BF41
:1050200030BCFFF793BF00BF4082002000207047D4
:10503000C82070470120704700207047002070474B
:1050400090F890308B4286BF00EB8100D0F894003E
:105050000020704790F890308B4286BF00EB8100B3
:10506000D0F894000020704703207047014B93F85C
:105070005A027047484B002070B504464C4810F067
:1050800021FC18B1236A43F400032362484810F05E
:1050900019FC88B1462064F0F5FEDFED467AB4EEE7
:1050A000E70AF1EE10FA07D8636A43F4000363627B
:1050B000A36A43F40003A362236A43F4F843236220
:1050C0003D4BD3F8A00F03685B6898470138182858
:1050D00015D8DFE800F03B430D4543434343143B01
:1050E0003B3B3B3B3B14434343433B14453B3B006F
:1050F000324A92F860348BB392F861248AB3304B11
:1051000093F8903F012B3DD0022B44D02D4B1D68CE
:10511000DDB12D4E284696F89A1C4EF075FCA0B1D4
:10512000236A43F48073236296F900331BB1636AE8
:1051300043F48073636296F89A1C28464EF09CFCF8
:1051400018B1A36A43F48073A36270BDD4E9092344
:1051500042F4E04243F4E0436262A362012300E0D0
:105160000023616A41F480626262A26A42F4806054
:10517000A062002BC3D041F4406142F440626162FE
:10518000A262BCE7236A43F480032362636A43F4A8
:1051900080036362BAE7236A43F480032362636A8D
:1051A00043F480036362A36A43F48003A362ADE720
:1051B000482B0020000000B4486B0020485B002012
:1051C000487B00203C910020484B002013B54FF451
:1051D0004470CDE900211DF0E7FE044628B1DDE969
:1051E000002162F005F9024B2360204602B010BD99
:1051F0000C580D08002070470020704700207047B1
:105200000020704700F50A503C3070470048704756
:10521000487E0D0800F58040D0F8A00F03685B6859
:105220001847000000F5804300F59A40D3F8A03FEE
:105230001B1A584258417047A22070472DE9F0418F
:1052400000F5A04303F2F45353F8042CDFED676A32
:1052500007EE902AB8EEE77AD3ED007AF8EEE77A17
:1052600000F5C24890B027EE267A67EEA67A08F1DC
:1052700038080446002340468DED017ACDED027AD0
:1052800003930BF035FE04F5C046002800F0A6801D
:10529000D6F86C3184330FCB0CAF87E80F0008AD24
:1052A00004AF87E80F0085E80F0001A9384603AB7B
:1052B00002AA31F097F99FED4E0AD6F8EC7301A8D7
:1052C00031F0E2FD294638468DED080ACDED090A98
:1052D0008DED0A1A16F004FC90F036FAD6F870320A
:1052E000C01A632804F587552DD8D6F86C010368D9
:1052F0009B689847042100F19402284656F046FF27
:10530000D6F86C010368DB689847052100F1940228
:10531000284656F03BFFD6F86C0103681B69984796
:10532000062100F19402284656F030FFD6F870218D
:10533000284602F52A72072156F028FF04F5C640D8
:10534000703013F01DFB40460CF0EAFF90B1D6F828
:10535000700187F089FF68B1D6F870216E21903214
:10536000284656F013FFD6F870216F21BC3228462C
:1053700056F00CFF04F5445204326921284656F0D9
:1053800005FF04F5495220326A21284656F0FEFEF8
:1053900004F5405393F9A22232B9D3EDA67AF5EE83
:1053A000C07AF1EE10FA06DD04F54F5214326B218B
:1053B000284656F0EBFE04F55054204680F0A6FA3D
:1053C00028B104F130026D21284656F0DFFE18F0B6
:1053D00097FA17F0A9FF10B0BDE8F08104F59950D5
:1053E00001A9083016F044FA76E700BF0AD7233C3B
:1053F000E02E654210B54FF48011044612F058F8C3
:1054000010B12046FFF71AFF4FF48001204612F03A
:105410004FF828B12DF0B2FEBDE810402BF040BD92
:1054200010BD000030B500F5995591B00023083546
:10543000029302A9002304460DF1070228468DF8C5
:10544000073018F033F803A9284617F027F808B9F1
:105450002D4B03933022002104A8BBF0C3F9A323F2
:105460008DF8103095238DF8113090F075F904F512
:10547000A042CDF81300D2F8F035ADF81B3004F59A
:105480008053D2F8F425CDF817104620D3F8201514
:10549000D3F82435ADF81D10ADF81F20ADF821303C
:1054A00064F0F0FC10EE103A1520CDF8233064F0D3
:1054B000E9FC10EE103ACDF8273004F535539FED96
:1054C000137AD3ED2F7A67EE877A284617EE903A53
:1054D000CDF82B30029BCDF82F309DF807308DF89A
:1054E0003330039B0D9318F0E7F904F58043302225
:1054F000D3F8E43F8DED0E0A04A904F587500F930D
:1055000056F080FF11B030BD2292CA7F0000C84221
:1055100030B58FB03522044600216846BBF062F9F1
:10552000A3238DF8003095238DF8013001238DF8E9
:10553000023090F011F904F5AA4304F54055783390
:10554000CDF803001B68D5F88406CDF80710CDF818
:105550000B3003681B699847ADF80F00D5F8840637
:1055600003689B689847ADF811001D4801F098FF4B
:10557000ADF81300D5F8840603685B69984710EE10
:10558000103AD5F88406CDF8153003689B69984722
:1055900010EE103A04F58041CDF8193001F6DC73B5
:1055A00035221B68CDF81D3004F5C043D86FCDF807
:1055B0002100D3F88000CDF82500986FD3F89C34F3
:1055C000CDF82900CDF82D3004F58750D1F8D43F1F
:1055D000CDF83130694656F015FF0FB030BD00BF31
:1055E000482B002030B587B01622044600216846BB
:1055F000BBF0F8F8A3238DF8003095238DF8013027
:1056000002238DF8023090F0A7F804F5A045CDF8FC
:1056100003002046CDF8071005F0CCF905F5BC6372
:105620008DF80B001B680393124B1B68D86A90F827
:105630009C308DF810300368DB69984795F8C935C0
:105640008DF812308DF811002DF098FD2CF08CFDA6
:10565000D5F8DC358DF813008DF81430162295F846
:10566000CA358DF81530694604F5875056F0CAFEE4
:1056700007B030BD442B002010B58AB02722044665
:1056800000216846BBF0AEF8A3238DF800309523C7
:105690008DF8013009238DF8023090F05DF8CDF8D7
:1056A00003000420CDF8071064F0ECFB10EE103A74
:1056B0001320CDF80B3064F0E5FB10EE103A4620D5
:1056C000CDF80F3064F0DEFB10EE103A1520CDF867
:1056D000133064F0D7FB10EE103A0320CDF81730EA
:1056E00064F0E0FB10EE103A1A20CDF81B3064F0A5
:1056F000C9FB10EE103ACDF81F3004F59F4370330C
:1057000027221B68CDF82330694604F5875056F0F0
:1057100079FE0AB010BD000013B5044600F58750AD
:10572000019056F0A1F9019856F038FA04F580532B
:10573000019893F9F4310BB156F0D8FA204602B033
:10574000BDE81040FFF798BF7047000030B500F586
:10575000C04389B093F84C22044600F5875552B1F6
:10576000D3F864011E22694689F0AEFE0F496A46ED
:10577000284656F0E3FF04F58043D3F8A00F0368F2
:105780005B68984704F50053014693F8DC212846EE
:1057900056F0F8FF04F59950083018F02BFB04F58B
:1057A000907009B0BDE8304025F0B0BD18590D0823
:1057B0009FED020A00224CF009BC00BF0AD7233C2F
:1057C00070B50446104E62F021FF104B2360502547
:1057D000601963F0D1F866513035B5F5547FF7D1D3
:1057E00004F5547064F044FF094A04F5EC6002F6D5
:1057F0003C318CF0D1FE01232046064984F89139D2
:105800004CF0F4FD204670BD50A90D0864A90D08A8
:10581000644D002048990D082DE9F04100F509512B
:105820009AB00D221831044655F022FA0022C048E1
:1058300027214CF043FB0421002064F0A3FE132138
:10584000012064F09FFE4621022064F09BFE15219A
:10585000032064F097FE64F065FC04F5C04393F9FF
:10586000043223B19FEDB30AB3484DF05FF94CF019
:10587000C3FFB24AB24E138843F0040313804FF0C3
:1058800000080AAF002110223846BAF0ABFF01230E
:105890008DF830303388ADF8283005A973680B9344
:1058A00038464CF013FAC8B19DF91430002B15DDC1
:1058B00063F02CF89DF81410036801391B68C9B215
:1058C000984758B1051D28464CF04AF930B9B368DD
:1058D000ADF8183006A928464DF042FC08F106083C
:1058E000B8F1240F06F10C06CCD1964800220DF138
:1058F0000B014BF01DFF06AD064620B34CF030F90E
:1059000008BB914B0FCB85E80F0004A928464CF04B
:10591000DDF9002840F03B814FF004088B4B0FCBA2
:1059200087E80F0005A938464CF0D0F928B105A842
:105930004CF016F908B148F0010803A930468DF87B
:105940000C804DF0BBFB824B0FCB85E80F0003A909
:1059500028464CF0BBF9002846D00998002204A93B
:105960004BF0E6FE064600283ED04CF0F9F805461E
:10597000002839D19DF80C30013BDBB2032B96BFD8
:10598000744A0346D35C8DF82830304639464DF0D2
:1059900095FB7148002205A94BF0CAFE06466CF043
:1059A00053FF78B16CF04EFF90F8302090F828103B
:1059B00090F84830114490F840200A44D34214BF74
:1059C0000125002586B130469DF90C804CF0C8F8C1
:1059D00050B91DB1B8F1000518BF01253946304650
:1059E0008DF828504DF06AFB04F50B500022B7EEFD
:1059F000000A012134304CF0E9FA04F50A50002283
:105A0000B7EE000A022110304CF0E0FA012304F551
:105A1000FB510093514A002308318E204CF052FA7A
:105A200094F9ACC9BCF1000F1AD14D4E0FCE3D46D2
:105A30000FC50FCE0FC50FCE0FC596E80F0085E836
:105A40000F006246042138464CF038FA9FED450AB3
:105A500045484DF06BF84548B7EE000A4DF066F842
:105A6000012504F50451424A00950023203140F2FB
:105A700005104CF027FA04F50B5002210430FFF713
:105A800097FE04F5085003212C30FFF791FE04F532
:105A9000085003213430FFF78BFE032104F50B502F
:105AA000FFF786FE04F50B5002210830FFF780FE59
:105AB000022104F50950FFF77BFE04F5095002218D
:105AC0000430FFF775FE04F5085002213C30FFF763
:105AD0006FFE04F5BF4014308CF066F8254A136859
:105AE000D90705D42449156004F5035308330B6026
:105AF00004F50C5020490122083001254CF034FAFD
:105B00001E4A0095002304F58751FD204CF0DAF978
:105B10001B4B1A68D20705D41A4A1D6004F592542B
:105B20000C341460174801214CF03AFA2CE000BF05
:105B300090960D08000096431C820E0820910020CC
:105B400000990D0854960D08104A0D08204A0D08BA
:105B5000304A0D088C960D085F960D0874DA0D0812
:105B6000404A0D08000000006C960D087B960D0859
:105B700010DF0E083C2B00200022002050680E0889
:105B8000402B00200C2200201AB0BDE8F08104A8B0
:105B90004BF0E6FF00283FF4BFAE4FF00C08BDE627
:105BA00070470000002070470020704700207047B9
:105BB00000207047002070477047000000207047A9
:105BC0000020704784B001A880E80E0004B00020D7
:105BD00070470000002070470020704770470000A9
:105BE00010207047004870474CA50D0800487047CA
:105BF0005CA50D0800207047704700000120704729
:105C00000120704700207047002343608360C36019
:105C100003614361002303767047000010B504461A
:105C2000FFF7F2FF0023637610BD0000027E531CD5
:105C3000DBB2042B037600EB820288BF002382EDE7
:105C4000010A88BF0376704710B50446FFF7EEFFE0
:105C5000D4ED017A9FED107A94ED020A637E77EE1F
:105C6000877A042B77EE807A94ED030A94BF013390
:105C7000052377EE807A94ED040A637677EE807AD6
:105C8000637E94ED050A77EE807A00EE103AB8EE66
:105C9000C00A87EE800A10BD0000000010B504465F
:105CA0001DF08AF9204610BD04F0A2BB03F0CEB966
:105CB00003F082BF03F0D6B901F0FCBE01F054BA84
:105CC00001F0D8BB01F018BCFCF7E0BFFCF78ABBC1
:105CD00038B51E4B036000F540530446D3F8180650
:105CE0001B4AC3F8682408B11DF06AF9194B2360F8
:105CF00004F5805393F8042F42B9D3F8005F2DB117
:105D000028462AF045F928461DF056F904F5915029
:105D100010307CF09DFF04F58F50143065F0A8FD25
:105D20000D4BC4F8983804F6F81059F0F9FC04F655
:105D3000CC1059F0F5FC04F62C1059F0F1FC04F5E8
:105D4000106059F0EDFC204638BD00BFE08C0D0816
:105D500030830E0834610E08E0270E0838B5434B37
:105D6000044640F8043B65F0A7FE04F110001BF068
:105D7000D1F904F1680052F0DDFE04F5907024F0D2
:105D8000A7FE04F5866019F0E1FF04F254501DF0FF
:105D900019F904F698002BF0B3F904F563604DF09F
:105DA00059FD04F5875056F061FA04F58F50143010
:105DB00065F046FD04F5915010307CF035FF04F598
:105DC00092500C3053F078FA04F5955067F052F881
:105DD00004F580530025264A83F8C45204F59650F2
:105DE00004F5965304331430136049F051FB04F565
:105DF00099502946083016F029F804F5CC50103097
:105E000075F00EFE04F5EC50143079F053FF04F5F4
:105E1000F5500C307CF062F804F5F85010307CF04E
:105E200097FC04F5FB50083014F032FF04F50350E2
:105E3000083076F053FA04F5045020306BF0DAFFA6
:105E400004F5005304F5075083F8DC51094D343054
:105E50007DF0BEFA2B6813B107488FF043FC204653
:105E600006494CF0C3FA2C60204638BD34610E0858
:105E7000FC9900207491002064A50D086C600E0848
:105E80002DE9F04F2DED028B04469FB0FFF766FF22
:105E9000E24B236004F50C500830FFF791FC04F549
:105EA0003250203004F500577EF0BCFD04F50A5353
:105EB0002233C7F8C83C04F53350062387F8CC3C9E
:105EC000343065F0CFF804F5355318330E9304F5EC
:105ED000BF431433C7F8703D0F934FF40063C7F806
:105EE000743D5A2387F8F43D04F5085907F65853D2
:105EF00004F5995809F11C09C94ADFEDCA8AC7F8A7
:105F00006C9D08F10808C7F8688DB7EE008AC3F8E1
:105F1000602104F53C50C44AC3F86821C3F8CC2181
:105F200083ED578AC3ED598A343059F019FF04F5CF
:105F30003D5059F015FFBD4BC7F8503F0E9B002652
:105F400087F8686F03F5FC70FFF75EFEB84BB94940
:105F5000C7F8503F87F8696F0E984CF047FAB64B78
:105F6000C7F8703F0E9BC7F8783F07F577630022AC
:105F7000C7F8748F04F53D555A63DA6304F53F5052
:105F8000012387F8B43F303508301CF0DBFB87F87D
:105F9000D86FAA4928464CF029FA04F53F504946E3
:105FA0001C307FF0F5F804F54450494634307EF05B
:105FB00053FD04F54A50494604F540570C307FF034
:105FC000B1FC2C22314607F58660BAF00BFC04F5D3
:105FD00051569B4904F550504CF008FA2836994B1D
:105FE000C7F8683406F108008EF0D4FA04F5525A66
:105FF00004F5535B0AF1140A0BF1380B50460AF111
:10600000140A5EF0B9FCD345F8D10723C7F81C3653
:106010000023A7F820364FF4CB701CF0CBFFC7F855
:10602000180604F5585024308EF0B4FA04F559508F
:1060300028308EF0AFFA844B1A6802B91E60834B89
:10604000C7F8683404F55A504FF48051C7F88456A5
:1060500008301BF061F904F55C5008304DF036F95A
:1060600004F55C501C306DF06BFF04F5974004F5AF
:106070008045743005F0ECF8754BC5F8F43B04F539
:106080009840103005F0E4F8724BC5F8103C04F568
:1060900098402C3005F0DCF86F4BC5F82C3C04F52B
:1060A0009840483005F0D4F86C4BC5F8483C05F5ED
:1060B0004763002204F59940DA609A605A6083EDE4
:1060C000008A043005F0C4F8654BC5F8843C04F53B
:1060D0009940203005F0BCF8624BC5F8A03C04F5AF
:1060E00099403C3005F0B4F85F4BC5F8BC3C04F572
:1060F0009940643005F0ACF85C4BC5F8E43C04F51D
:106100009A4005F0A5F85A4BC5F8003D04F59A40B1
:106110002C3005F09DF8574BC5F82C3D04F59A40FE
:10612000483005F095F8544BC5F8483D04F59A40C1
:10613000643004F59B4605F08BF804364F4BC5F8E8
:10614000643D304605F084F84D4BC5F8843D04F5B8
:106150009B40203005F07CF84A4BC5F8A03D04F583
:106160009B403C3005F074F8474BC5F8BC3D04F546
:106170009B40583005F06CF8444BC5F8D83D04F509
:106180009B40743005F064F8414BC5F8F43D04F5CC
:106190009C40143005F05CF83E4BC5F8143E04F505
:1061A0009C40303005F054F83B4BC5F8303E04F5C8
:1061B0009C40503005F04CF8384BC5F8503E04F583
:1061C0009C406C3005F044F8354BC5F86C3E04F546
:1061D0009D40083008F0C2F804F59D40443005F0B9
:1061E00037F8304BC5F8C43E2F4BC5F8E03E04F5F8
:1061F0009D404FF4C053A5F8343F2C4960304CF01B
:10620000F5F8FE2385F8AC3F052385F8D03F4FF025
:10621000FF3B274BC5F8A06F4CE000BFE08C0D089A
:10622000000080BF0000B4420000B4C29CA50D086D
:10623000ACA50D0854190F08B4160F085C160F080A
:10624000B4140F0830830E087C940020E0580D0829
:1062500004B10D0800B80D0820BB0D0800AF0D08F3
:1062600014B20D089CB20D087CB10D0884B00D0865
:1062700000B00D0890B70D088CB30D081CB30D08C5
:10628000E4A50D080CB40D0818B70D080CB50D08E1
:10629000FCB50D087CB50D0894B60D088CB40D083E
:1062A00090AE0D089CBA0D08D4A50D08143A0F083D
:1062B000A95C0108C5F8A46FC5F8D8BF119305F50E
:1062C0007F65864B85ED008A04F59F4004F5A04567
:1062D00022464FF4007100937430814B10941AF0F1
:1062E00071FA05F5AC63C5F850B5C3ED038A032315
:1062F0000026C5F8DC3505F5BF63C5F8A865C5F807
:10630000AC65C5F8B065C5F8B465C5F8B865C5F83D
:10631000BC6583ED008A734BC5F8203604F5AC4AA2
:10632000714BC5F828365046704BC5F83036C5F865
:106330001C46C5F82446C5F82C4644301CF002FA29
:10634000504660301CF0FEF950467C301CF0FAF9E3
:10635000674BC5F89036A5F894B60AF198001CF082
:10636000F1F9644B6449C5F8F4B65046C3F800A08F
:106370004CF03CF84FF6FF7304F5AD40A5F83C3601
:10638000A5F858B6783054F067F85C4BD7F88426F7
:106390001294CDE913345A4BCDE91534594BCDE95C
:1063A0001734594BCDE91934584BCDE91B34584BB0
:1063B0001D931EA911E903000CAB83E80300DDE97E
:1063C0001A010AAB83E80300DDE9180108AB83E892
:1063D0000300DDE9160106AB83E80300DDE91401E3
:1063E00004AB83E80300DDE9120102AB83E803009C
:1063F00004F5C0475146CDE900290E9B0F9842464F
:106400008BF0DCF908F51B7338463B6554301CF003
:1064100099F9384664301CF095F93846743004F523
:10642000C1491CF08FF909F170091C22314607F1AE
:106430008400BAF0D7F948467DF084F8354B3649E8
:10644000C7F8F03048464BF0D1FF344A3449116068
:1064500004F5C24328334FF0140CB0B20CFB001209
:106460000136127C002AF8D12E4A10802E4A166876
:1064700016B12E488FF036F904F5C2402C30136067
:106480007DF04AF82A4BC7F82C3104F5C24041464A
:10649000383009F01DFA274BC7F83034642387F8E9
:1064A0003434254BC7F8683404F5C840234BC7F88B
:1064B0006C34234930304BF099FF224BC7F830340D
:1064C00020460123C7F8906487F8986485F89035D2
:1064D0001FB0BDEC028BBDE8F08F00BFF4550D0876
:1064E000A95C0108AD5C0108B15C0108B55C01085C
:1064F0000000FFFF6490002018360E08B95C010808
:10650000BD5C0108C15C0108C55C0108C95C0108EB
:10651000CD5C0108D84F0D08B04F0D083091002018
:10652000E89A0D082C910020EC90002078A50D0829
:1065300018500D08BCA50D08C8D60D0820D70D08A9
:10654000288A0E08A0D80D0810B58EF003FC064C62
:10655000064B18602046FFF793FC2046044A054985
:10656000BDE81040B7F0FCBB482B0020442B0020B6
:1065700060F20020D15C01080069C0F34010704750
:106580000F299DBF302303FB0100503000207047CE
:10659000014B93F9A1027047484B0020014BD3F8FF
:1065A000B40C7047484B002008B503689B689847B7
:1065B00030B9044B93F8BA0FB0FA80F0400908BD27
:1065C0000020FCE7486B002008B504480EF0E8FE08
:1065D00010B9034B93F8B40F08BD00BF482B00203F
:1065E000486B0020022A10B50C4605D1BDE81040CA
:1065F0000948352210F044BE084BD3F8A00F0368B9
:106600005B689847A04205D162F080F9BDE8104070
:1066100062F006B910BD00BF482B0020486B002077
:10662000012910B50C4610D0022904D061B960F0E0
:10663000C1FE084A02E060F0BDFE074A06215AF09A
:1066400031F8064BC3F8D04110BD60F0B3FE044AE8
:10665000F4E700BFFCA60D08D4A60D08488B002067
:10666000EBA60D08012910B50C4614D0022907D05D
:10667000D1B90E4BC3F8901460F09CFE0C4A05E0B3
:106680000A4BC3F8901460F095FE0A4ABDE810402A
:1066900006215AF007B860F08DFE074A06215AF02D
:1066A00001F8024BC3F8904410BD00BF488B002096
:1066B0003BA70D0810A70D0824A70D08012903D03A
:1066C000022914BF00210221014BC3F8541C70475A
:1066D000484B0020012902D0022900D011B9024BF9
:1066E000C3F89414704700BF488B00206C2942DC2B
:1066F0003F2914DC382952DC26292DDC042964D0FA
:1067000010294CD17047A1F1AA030B2B47D8DFE821
:1067100003F05C46465C46465C464646465CA1F154
:1067200040032C2B3BD8DFE803F0443A3A3A3A3A9C
:106730003A3A503A3A3A3A503A3A3A3A413A413A7F
:10674000414141503A41503A3A50503A503A3A3A1F
:106750003A3A3A3A3A505000A1F12703112B1ED889
:10676000DFE803F0331D1D1D331D1D1D1D1D1D1DE7
:1067700033331D1D3333A0290DDC95290FDDA1F125
:1067800096030A2B0BD8DFE803F0200A0A0A202020
:106790000A200A0A1100B52903DCA929B3DC62F03A
:1067A00075BEA1F1D003022BF9D87047002362F027
:1067B0003FBE064B012283F88C24A3F58043D3F817
:1067C000B00C10B1642162F0E7B87047488B00202C
:1067D0006C2938B50346154600F3A0803F290FDC2D
:1067E000382907DC26296DDC042900F01A811029DC
:1067F00000F000812A461846BDE8384062F034BCFB
:10680000A1F140022C2AF5D801A050F822F000BFD7
:10681000CD690108F5670108F5670108F56701080A
:10682000F5670108F5670108F5670108F5670108D4
:10683000FD690108F5670108F5670108F5670108BA
:10684000F5670108276A0108F5670108F56701087F
:10685000F5670108F56701086F6A0108F567010827
:10686000C36A0108F5670108796A0108B96A010875
:10687000656A0108FB6A0108F5670108E36A010817
:106880002D6A0108F5670108F5670108BB69010871
:10689000056B0108F56701080B6A0108F567010837
:1068A000F5670108F5670108F5670108F567010854
:1068B000F5670108F5670108F56701088D6B0108A8
:1068C000336A0108A1F12702112A93D801A050F8D8
:1068D00022F000BFBB690108F5670108F5670108F0
:1068E000F5670108BF690108F5670108F567010848
:1068F000F5670108F5670108F5670108F567010804
:10690000F56701081D6A0108056A0108F5670108B5
:10691000F5670108176A0108116A0108A02921DC3E
:1069200095297FF767AFA1F196020A2A3FF662AF79
:1069300001A050F822F000BF0F6B0108F5670108B5
:10694000F5670108F5670108156B0108676B010819
:10695000F5670108756B0108F5670108F56701081F
:10696000356B0108B52923DCA9297FF743AFA1F1D5
:10697000AA020B2A3FF63EAF01A050F822F000BF5A
:10698000396A0108F5670108F5670108556B0108C8
:10699000F5670108F56701083F6A0108F567010816
:1069A000F5670108F5670108F5670108AD6B010897
:1069B000A1F1D002022A3FF61DAF01248FE0A91EEB
:1069C000834B4D424D4183F8AD5FF6E7AA1E554219
:1069D000804C554184F88B5460F0ECFC7E4A94F86E
:1069E0008B147E4B002908BF13467D4A062159F0BF
:1069F00059FEE2E70A21FFF7F5FDDEE72A4601210D
:106A00001846F8E72A460421FAE72A460321F7E761
:106A10002A460C21F4E72A460F21F1E72A460021F5
:106A2000EEE70B21E7E72A460D21E9E72A46052193
:106A3000E6E72A461521E3E72A461121E0E7AB1EE7
:106A40005A425A41634B93F830129142B5D083F8C1
:106A5000302260F0AFFC634A634B022D08BF13463F
:106A6000624AC3E729461846FFF728FEA5E72946EC
:106A70001846FFF7D5FDA0E7564CD5B1022D0DD134
:106A8000012384F88834A4F50053D3F8A00F0368D9
:106A90005B6A984710B1564800F09CFF60F08AFC92
:106AA000504A94F88814504B002908BF1346514AA5
:106AB0009CE784F88854E6E729461846FFF7D2FD9C
:106AC0007BE7012445B1022D09D1424BC3F888412F
:106AD000002283F8782202E03E4BC3F8885120461A
:106AE00038BD01242DB1022DF9D1434B83F8B440B8
:106AF000F5E7414B83F8B450F1E729461846FFF714
:106B0000E9FD5AE761F002FF61F08AFE55E72A4687
:106B1000072175E71846294662F000FA37487CF0ED
:106B200051FD044600283FF448AF2A4B0122C3F828
:106B30008821CDE7274BD3F84832002B3FF43DAFF7
:106B4000012425B1022DCAD183F82C40C7E783F870
:106B50002C50C4E7022D7FF430AF9FED290A244862
:106B6000FBF7B0FC29E7022D7FF427AF20480EF099
:106B700025FB22E701242DB1022DB0D1154B83F85E
:106B80008A44ACE7134B83F88A54A8E7022D19D145
:106B90000F4DD5F8A00F0368DB6B9847044650B142
:106BA0000121A5F5804003F041F998E715482946F1
:106BB0008CF082FE01E760F0FDFB134A042159F0DE
:106BC00071FDFAE60A48002103F030F9F5E600BF4E
:106BD000486B0020488B002050A70D08738F0D08CC
:106BE00058A70D0883790D086CB80D0868A70D0823
:106BF000482B002074A70D08484B0020388C00203B
:106C000000000000287A002087A70D0810B599B170
:106C100004681168416004B90160126801681B686A
:106C2000521A9A4202D80021084610BD017A012367
:106C300081F001010372F7E7037A3BB144682CB19C
:106C40001368029A12681B1B9342ECD90023C0E917
:106C50000033EFE70023C0E90533C0E9083383853B
:106C6000037780F828307047F0B52DED028B04468D
:106C700087B09F48B0EE408A0E467CF0ADFC40B134
:106C8000236933B1206B00F50E7010F0F5FD054659
:106C900038B12046FFF7DEFF002007B0BDEC028BC5
:106CA000F0BD236B93F93C22002A1EDD93F8A0323D
:106CB000DBB1904BD3F89424002AEAD12369D4EDB8
:106CC000007A991E4842F5EEC07A4841F1EE10FA7A
:106CD00084F82C0027D8C4E90822C4E9052284F8E6
:106CE0002D2084F828202277D7E7834FD7F8A00FEC
:106CF00003689B6B984728B107F5805797F8D835FC
:106D0000002BD6D07D4800210EF0E2FDDFED7C7A2D
:106D1000B4EEE70AF1EE10FACBDA784803F04AFE57
:106D20000028C6D1B5E76EB1F4EEC87AF1EE10FADC
:106D30003CDD236BD3F8C432DB0403D5714815F076
:106D40005DFB064684F82D608EF0FEFCD4ED027AE1
:106D50009FED6D7A039067EE877AFCEEE77A17EE87
:106D6000903A5B000593B4F90630CDED047A002B20
:106D70001EDC0023C4E9083384F8283094F9043079
:106D8000002B41DC0023C4E90533237794F82C0061
:106D9000002882D194F82D0000287FF47EAF94F86B
:106DA000280000287FF479AF207F76E71646C9E7F0
:106DB0000421524800F0B4FCB4F9063007EE903AD2
:106DC000F8EEE77A05ABF4EEC07AF1EE10FA009334
:106DD000CCBF0121002104AB03AA04F12000B0EED6
:106DE000408AFFF713FF0028C8D060F0E3FA064698
:106DF00018EE100AF9F788FB444ACDE90001042196
:106E0000304659F04FFCB9E7414E9FED427AD6F833
:106E10002025DFED416A06F58051D1ED8F7A82EAB7
:106E2000E270B0EE476AA0EBE270A7EEA66A07EE4A
:106E3000900AF8EEE77AF4EEC67AF1EE10FA53D83B
:106E4000D6F8240591ED906A07EE900AA6EE267A10
:106E5000F8EEE77AF4EEC77AF1EE10FA44D591ED48
:106E6000916A9FED2E7AA6EE267AF4EEC77AF1EEBD
:106E700010FACCBF01270027642113FB01F1284B36
:106E8000D3F8F005121A002AB8BF52428A422DDA0E
:106E9000D6F82425D3F8F435D31A002BB8BF5B42BB
:106EA0008B42ACBF0023012304F114000FB983F01F
:106EB000010505AB009303AA04AB2946FFF7A6FE24
:106EC00000283FF463AF60F075FAD6F82015D6F8C5
:106ED0002425642392FBF3F291FBF3F30092042147
:106EE000104A59F0DFFB51E70027C5E70023DBE735
:106EF000388C0020488B0020486B0020482B002055
:106F000000000034703E002000007A4480A90D0883
:106F1000483B00200000FA430000C8420000FAC3CA
:106F2000487B002091A90D0873B58289036BD207B5
:106F300004466CD493F93C22002A03DD93F8A02286
:106F4000002A64D1524DD5F8A01F05F56562914223
:106F50005DD0A5F54055B3F90860D5F8203507EEAA
:106F6000903AD5F82435B8EEE77A07EE903AF8EE85
:106F7000E77A6846CDED017A8DED007A2FF052FE6A
:106F8000730007EE903AF8EEE77AB0EEC00AF4EE3E
:106F9000C07AF1EE10FA42D4236B93F8F1223AB39F
:106FA00007EE906AF8EEE77AF4EEC07AF1EE10FAA6
:106FB0001EDB002183F8F112236B586B85F050F82B
:106FC000236B9FED347ADA6BD2ED067A05F22C72E0
:106FD00067EE877A92ED007AF4EEC77AF1EE10FA56
:106FE00006D5986B87F09CFA236B986B87F032F884
:106FF000A389226B13F0020302D192F8F11299B91E
:10700000002382F8F232236B93F8F10205E00020AE
:1070100083F8F102236B83F8F20202B070BD236B98
:10702000012283F8F122B7E705F24461D1ED007A3D
:107030009FED197AF0EEE76AF4EEC76AF1EE10FA06
:10704000DFDD05F23C61D1ED006A9FED146AB0EE20
:10705000E67AB4EEC67AF1EE10FAD2DD104991ED7F
:10706000007AB0EEC77AB4EEC67AF1EE10FAC8DD57
:1070700067EEA67AF5EEC07AF1EE10FAC1D5D5F832
:10708000243508498B42ACBF00230123B9E700BF78
:10709000486B00200AD7233CC2B8323E920A063F12
:1070A000884100206CEEFFFF08B5036B93F8F222D5
:1070B0003AB1DA6A92F8A020022A03D0002283F8BB
:1070C000F22208BD0B4B9FED0C0AD3ED007AF5EED2
:1070D000C07ADFED0A7AF1EE10FAD8BFB0EE670A97
:1070E000152062F0BBFEBDE808409FED050A1320A5
:1070F00062F0B4BE8C41002000A08CC500A08C457D
:107100000000000000F58040D0F8A00F03681B6C61
:107110001847000000F5005393EDB07A00F5C04029
:10712000B5EEC07AF1EE10FA5DBF036DDFED076AD0
:10713000D3ED017A806E5FBFF8EEE77AE7EE267A4C
:10714000FDEEE77A17EE900A704700BF0000C842D4
:1071500000F5005090F8000328B141F00101084209
:1071600014BF01200020704710B54B68516800F52E
:10717000C0448B42D8BF0A46D4F88400CCBF1A461C
:1071800019462CF01DFEC4F8840010BD10B504464D
:107190004D486AF08BFF10F0080217BF4B4BDFED34
:1071A0004C7A93ED4B7AD3ED4D7A1FBF77EE877A09
:1071B0009FED487A012267EE877A10F0010317BF2E
:1071C000424B9FED437AD3ED4D6A93ED4A7A1CBF53
:1071D00037EE667ADFED3F6A04F5005118BF27EEFF
:1071E000267AD1EDB26AF5EEC06A18BF0123F1EE3E
:1071F00010FA34DD354A9FED376AD2EDB26A66EE99
:10720000866A0122F4EE676AF1EE10FA58BFF0EEDA
:10721000667A04F5C04090F88C1029B373B1D0EDB4
:10722000246AF8EEE66AF4EEC76AF1EE10FA58BF87
:10723000F0EE476AFDEEE66AC0ED246A9AB190ED81
:10724000247AB8EEC77AB4EEE77AF1EE10FAD8BF36
:10725000B0EE677ABDEEC77A80ED247A03E0002AAB
:10726000D7D1002BD5D110BDABB1036DD3ED016AE1
:10727000F8EEE66A76EE876A90ED217AB8EEC77A84
:10728000F4EEC76AF1EE10FAD8BFB0EE667ABDEE42
:10729000C77A80ED217A002AE5D0036D93ED017A5B
:1072A000B8EEC77A77EE277A90ED217AB8EEC77AF2
:1072B000F4EEC77AF1EE10FA58BFB0EE677ABDEE81
:1072C000C77A80ED217ACEE7684C0020484B002039
:1072D000000000000000C84200F5C0400023C0F8D4
:1072E0008830704773B51646044600236A46304618
:1072F00000931BF015FB48B1DDED007A9FED277A76
:1073000067EE877AFDEEE77A17EE900A04F5C0453E
:10731000C5F8880033785B0718D595F88C30ABB189
:1073200004F5AD40012201A9783053F01BFA68B191
:10733000D5ED247ADDED016A9FED187AF8EEE77A53
:10734000E6EEC77AFDEEE77AC5ED227A04F5A043B2
:10735000D3F8DC35042B1FD004F50054B4F9FA221D
:10736000002A16DDD5F888309FED0D7A83EAE371A7
:10737000A1EBE37107EE901AF8EEE77A67EE877AF1
:1073800007EE102AB8EEC77AF4EEC77AF1EE10FADB
:1073900002D50023C5F8883002B070BD0000C84295
:1073A0000AD7233C37B50B785A0704460D461DD53E
:1073B00000F5AD40012201A9783053F0D3F9A8B10E
:1073C000D5ED017A2B78DFED1A6AF8EEE77ADB0764
:1073D00067EEA67A19D59DED017AB4EEE77AF1EE63
:1073E00010FACCBF0120002003B030BD2B78D5EDC2
:1073F000017A13F0010FF8EEE77A04F5C0440ED1DC
:1074000094ED1A7AB8EEC77AE7E704F5C044236D25
:1074100093ED017AB8EEC77AE7EE667ADBE7236D83
:1074200093ED017AB8EEC77A77EE877AE8E700BF86
:107430000AD7233C00F5005300F58042B3F9AA3285
:10744000D2F8A02F00EE103A00F59A439A42B8EE17
:10745000C00A0ED100F5A040D0F8DC35042B02D0D4
:1074600090F891352BB100F69470D0ED007A30EEA3
:10747000270A7047014608B501F5C041FFF7DAFF5A
:10748000D1ED1A7A9FED057AF8EEE77AE0EE477AC9
:10749000FDEEE77A17EE900A08BD00BF0000C84273
:1074A00037B500F5C045044695F88C30DBB100F5E2
:1074B000AD40012201A9783053F054F998B1D5EDCF
:1074C000247AD5ED256A9FED0B7AF8EEE77AE6EEA1
:1074D000877ADDED016AE6EEC77AFDEEE77A17EE10
:1074E000900A03B030BD2046FFF7C4FFD5F88430C2
:1074F000181AF6E70000C842014608B5FFF79AFFE0
:1075000001F5C041D1ED287A37EEC00ADFED047AEB
:1075100020EE270AFDEEC07A17EE900A08BD00BFE4
:107520000000C8422DE9F04100F5C04800F5C04513
:1075300008F1640874350446294640461BF064FC93
:1075400004F5A04704F5C04607F5AF6354362A4654
:10755000314683ED000A40461BF08CFB07F27C5756
:10756000DFED230A87ED000AB7EE001A76202CF033
:1075700087FB04F5355383ED770A2046FAF732FF8F
:1075800004F58043D3F8A00F03685B6898470B2885
:107590000DD008D80A2811D004F5C0440023C4F83F
:1075A0008830BDE8F0810E38C0B20128F4D82946F1
:1075B0002046FFF7F7FE0028EED011E029462046CE
:1075C000FFF7F0FE30B90B484FF48041FBF742FA69
:1075D0000028E1D12046FFF78FFFB0F5FA6FE6DD16
:1075E0002A4631462046BDE8F041FFF77BBE00BF8A
:1075F00000000000482B002010B52DED028B00F597
:10760000C043D3ED1E7A93F87430DFED1D8AB8EED7
:10761000E78ADA0728EE288A82B0044609D400F502
:10762000805202F5B362D2ED007AF8EEE77AA7EE67
:10763000E88A5B070FD504F5AD40012201A9783037
:1076400053F090F838B19DED010A30EE480A02B0CF
:10765000BDEC028B10BD204604F58054FFF70AFFF5
:1076600004F5B36393ED000A07EE900AB8EEC00A82
:10767000F8EEE77A28EEC00AA7EEA80AE5E700BF11
:107680000AD7233C73B504461646FFF761FD78B967
:1076900066BB04F5C245383528460AF075FCB8B318
:1076A00028460AF019F898BB2046FFF7A5FF09E025
:1076B00004F5005595F8D03CDB0705D505F6EC45FB
:1076C00095ED000A02B070BD04F5C24038300AF0F2
:1076D00081FC0028DCD095F89A1C04F563604CF01E
:1076E00089F90228D4D19FED0D0AEBE704F5A043F8
:1076F00093F8903F022BCCD104F5AD40012201A9B3
:10770000783053F02FF80028C3D09DED010AD9E757
:1077100004F5C04494ED280AD4E700BF000000003F
:1077200000F5C04393F88C20FFF7ACBF38B52DEDC2
:10773000028B00F5804200F59943D2F8A02F203348
:107740009A4204464DD100F58053D3F8285500F5F0
:107750000053B3F9F832002B66DD04F5B95292ED0F
:10776000037AF7EE007AB4EEE77AF1EE10FA5BD422
:1077700004F53652D2ED007AF6EE006A67EEA67A8C
:1077800087EE871AB5EEC01AF1EE10FA4CD907EE63
:10779000905A9FED288AB8EEE70A07EE903A04F572
:1077A000AD4004F5C044F8EEE70A20EE080A783050
:1077B00053F0E4F8D4F888309FED1F1ADFED1F0A6C
:1077C000002BBCBF07EE903AF8EEE77A4FF4297031
:1077D000B8BFA7EE880ABDEC028BBDE838402CF09C
:1077E0004FBA07F099FDF8B904F54053D3F8840671
:1077F00003681B69984704F50053DFED100AB3F9DD
:10780000F83201EE103A04F5AA4393ED1E0AB8EEE1
:10781000C11A054640F27F202CF032FABDEEC00AB4
:1078200010EE103A1BB296E7BDEC028B9FED030AF7
:1078300038BD00BF0AD7233C00007A440000000096
:1078400010B504468DF080FF04F50053D3F8E42C06
:10785000801A41F2883290420FD802212046FFF769
:1078600077FC50B104F5A044D4F8DC25042A04D1F7
:1078700003F6D84393ED000A10BD9FED010AFBE724
:107880000000000030B52DED028B00F5C045DFEDA6
:10789000268A95F88C3083B004465BB3D5ED247A04
:1078A0009FED220AF8EEE77A00F5AD4027EE800A58
:1078B000012201A9783052F08DFFD8B12046FFF7A0
:1078C00035FFDDED017A85ED250A37EE800A204689
:1078D0008DED010AFFF7B4FFDDED017A30EE270AE6
:1078E00020EE280ABDEEC00A10EE100A03B0BDEC6F
:1078F000028B30BD2A6DD5F8843052689B1A08EE91
:10790000103A2046FFF796FDB8EEC88A2046A0EE52
:10791000288AFFF795FFBDEEC88AB8EEC88AA0EEA8
:10792000288ABDEEC80ADFE70000C8420AD7233C18
:1079300010B500F580430446D3F8A00F03685B6AD6
:10794000984718B104F5C04494F8880410BD0000AD
:1079500038B500F5C0440D46D4F884300B44C4F863
:10796000843094F88C303BB1FFF7E2FF20B9D4F8B3
:1079700090102944C4F8901038BD000030B500F5CF
:107980000050D0F8F422D3070FD4094B0B201D78F8
:107990005C688D4204D1224214BF0120002030BD1A
:1079A000013803F10803F2D1F9E70120F7E700BF3E
:1079B000E8A90D0810B500F580430446D3F8A00FE0
:1079C00003685B68984701462046BDE81040FFF712
:1079D000D5BF000037B500F5C0440546A36EC4F816
:1079E00084300023C4F88830FFF7E4FFD0B105F5F8
:1079F000AD40012201A9783052F0B4FE90B1284682
:107A0000FFF796FF70B9DDED017A9FED087A67EE1A
:107A1000877A0123FDEEE77A84F88C30C4ED247A6E
:107A200003B030BD002384F88C30F9E70000C84271
:107A300038B504460D46FFF7BDFF30B10321284697
:107A40001AF04AFF80F00103D8B204F5C04484F86C
:107A50008D0038BD73B500F5C0444A68C4F8842071
:107A60000B780D46D90741BF236D5B689B18C4F89E
:107A7000843094F88D30064623B100F5C04174314E
:107A8000FFF7D6FF2B785B070FD506F5AD40012237
:107A900001A9783052F066FE38B1012384F88C30A9
:107AA0006B68C4F8903002B070BD002384F88C304D
:107AB000F9E70000F0B52DED028B044683B004F524
:107AC000C0450E468DED010AFFF7C4FFDFED330A16
:107AD0009DED010A40F24310B7EE001A2CF0D0F8E9
:107AE000D5F888305B4207EE903AF8EEE77A204608
:107AF00067EE807A04F50057FDEEE77AB0EE408A33
:107B000017EE901AFFF724FFD7EDBF7AF5EEC07A93
:107B1000F1EE10FA3EDDD5F88830002B3ADD204634
:107B2000FFF7BEFC07EE900ADFED1D6AB8EEE77ABC
:107B3000D7EDBF7A67EEA67AB4EEE77AF1EE10FAE7
:107B400028D531462046FFF785FF29463246643165
:107B50002046FFF7C7FBD5F888305B4207EE903A26
:107B6000F8EEE77A204667EE887AFDEEE77A17EEC0
:107B7000901AFFF7EDFEB5EEC08AF1EE10FA09DDBE
:107B8000D5ED227AB8EEE77AC7EE087AFDEEE77A0D
:107B9000C5ED227A03B0BDEC028BF0BD0000000001
:107BA0000000C8C2F0B500F5C04487B094F8743046
:107BB00003F00503052B07460BD053F009FE4FF4E5
:107BC000AE724FF4801153F0BBFD0025284607B07C
:107BD000F0BD1E486A4603211AF08EFE0028F4D03C
:107BE0001B4801AA03211AF087FE05460028ECD0A5
:107BF000184BDFED190A93ED000A40F26D10B7EE55
:107C0000001A2CF03DF804F174030FCBB0EE401ACB
:107C100002AEDFED111ADDED010A9DED000AB7EEAF
:107C2000002A86E80F002BF05DFFDFED0C7A20EED6
:107C3000270A3046FDEEC07A032217EE901A1AF09A
:107C400087FD31463846FFF705FFBFE79C8B0020D4
:107C5000BC8B0020C4800020000000000000C8424F
:107C6000F7B50E4602210446FFF772FA70B304F529
:107C7000A045D5F8DC35042B28D12046FFF79AFE25
:107C800020B304F5AD47783704F5C04101236A46B7
:107C90006431384652F050FCC0B104F5C0410123B4
:107CA00001AA7431384652F047FC78B19DED017A53
:107CB000DDED007A77EEC77A96ED007A37EE277A17
:107CC00005F29C5586ED007AC5ED007A03B0F0BD53
:107CD000F0B52DED048B00F5005489B000F5636616
:107CE00094F89A1C0391054630464BF083FE0399A5
:107CF000074630464BF090FE042F0399B0EE408AC1
:107D000021D1002305A88DED050A069307932FF0D6
:107D100009FA05F5B25005A908302DF0D1F8DFEDCC
:107D2000AC7A8DED050AB4EEE71AF1EE10FACDED5E
:107D3000060A8DED071A06DB05F5805393F8A47546
:107D400017F001070CD194F8D03C002262F3000335
:107D500084F8E82C84F8D03C09B0BDEC048BF0BD6D
:107D600094F8D03C9A075FBF43F0020384F8D03CFC
:107D700004F6D44383ED008A05F5335104F6EC4351
:107D800083ED001A2C312846FFF76AFF94F8E83C8F
:107D9000092B00F2898004F54F63D3ED000A9FEDB3
:107DA0008D9AB0EE480A2BF059FE00BB04F6D4437E
:107DB00094F89A1CD3ED008A30464BF04BFE07EE48
:107DC000900A9FED857AF8EEE77A78EEC88A67EE3A
:107DD000877AF0EEE88A67EE897AF4EEE78AF1EEC8
:107DE00010FAC2BF94F8E83C013384F8E83C04F58B
:107DF0004F6394F89A1CD3ED008A30464BF02AFE6C
:107E000007EE900AF8EEE77A9FED747A67EE897ACA
:107E100078EEC88A67EE877AF0EEE88AF4EEE78AB1
:107E2000F1EE10FA02DD002384F8E83C04F54F631C
:107E300083ED008A94F8D03CDA078DD52846FFF709
:107E4000DBFB04F6EC4393ED008A05F5C04330EE0E
:107E5000488A93F88C30002B70D005F5AD40012294
:107E600005A9783052F07EFC00286DD18DF06CFCB5
:107E7000D4F8E42C41F28831821A8A42034604F68F
:107E8000D84204F6DC4168D982ED008A284681EDAB
:107E9000008A0221FFF75CF918B105F5BF452A6A8F
:107EA000EA61C4F8E43C57E794F8D03C43F001039E
:107EB00084F8D03C05F5A04305F59C42D3F8DC6579
:107EC00005F58043301FD3F8A03F464202F114026B
:107ED0004641934211D005F59C42303293420CD07A
:107EE00005F59A42934209D13D4B05F5C240B3F8DE
:107EF0003E16383009F00CFC00B13E4694F8D03CF8
:107F0000590793D4002E91D002212846FFF720F97B
:107F100000288BD043F0040384F8D03C04F6EC43F3
:107F200005F551561868F8F7EFFA2836CDE9000143
:107F30002C4A0621304658F0B5FB77E72846FFF774
:107F400039FD002889D191E704F6EC4393ED000A4E
:107F50009DED058A38EE408A88E79FED200A92ED74
:107F6000007ADFED217A28EE008AA7EE278A82EDDB
:107F7000008AC4F8E40CD1ED007A38EE678AF3EE9B
:107F80000E7AB0EEC88AB4EEE78AF1EE10FA7FF707
:107F9000E3AE94F8D03C5B070ED504F6EC4405F54F
:107FA00051562068F8F7B0FA2836CDE900010F4A9B
:107FB0000621304658F076FB05F533502422002187
:107FC000103009B0BDEC048BBDE8F040B8F00ABC3D
:107FD000000000340AD7233CCDCC4C3DCDCC4C3EE8
:107FE000487B0020A8A90D08CDCC4C3FC5A90D08A1
:107FF00038B52DED028B0D460446FFF7FDFA002340
:1080000020462B70B0EE408AFFF71AFC0221204672
:1080100038EE400AFFF79CF828B104F5005494F8B4
:10802000D00C00F00100BDEC028B287038BD0000C0
:1080300070B50B7803F00503042B05460C46164675
:1080400014D105F5C04553F0C3FBB2B24FF4801113
:1080500053F076FB2A6D636852689B1A13F5FA7F1A
:10806000C8BF6360237843F00103237070BD000034
:10807000F8B500F5805300F5A047D3F89865D7F818
:10808000A055B542044619D00E4A1268D26A92F839
:108090009C209AB100F5C041751B25227431FFF771
:1080A000C7FF07EE905AB8EEE70ADFED077A04F54E
:1080B000355020EE270A183080F06AF9C7F8A0651D
:1080C000F8BD00BF442B00200AD7233CF8B500F5CB
:1080D000A04C00F5C0449CF893E505460F4604F11A
:1080E0005406BEF1000F4CD004F174030FCB86E8A8
:1080F0000F0001238CF8943597E80F0004F1740603
:1081000086E80F00E36F05F5C04674366BB9D4F806
:10811000803053B9E36EA26FE367236FC4F88030F9
:108120001AB9A16E30461AF013FB314628222846B0
:10813000FFF77EFF94F8741011F0040102D130466D
:108140001AF0CAFB05F5C04105F5C040324654316E
:1081500064301AF0C5FD30B104F15406643494E87B
:108160000F0086E80F00284606F0B0FC2846FFF70F
:10817000D9F9284607F096F82846BDE8F840FEF7FA
:10818000C1BF04F164030FCB86E80F0001238CF814
:1081900093358CF894E5AFE7F8B500F50053044645
:1081A000B3F95232002B0D4633DB0B7813F0020F7C
:1081B00014BF4FF0FF33012304F5C04606F1540706
:1081C00086F82C3006F164030FCB87E80F0095E8A2
:1081D0000F0006F1740787E80F0057223946204642
:1081E000FFF726FF2046FFF7F5FB2046FFF79AF939
:1081F000204607F057F804F5A043002583F894556E
:108200002046356383F8995506F060FC86F87A526B
:10821000F8BD4FF0FF33CFE72DE9F043364B1B6835
:1082200085B00546D86AF9F77FF9002861D105F5D0
:10823000005393F9683C5A1C54D0002B05F586670F
:1082400011DD95F84124242107EE903A01FB0272DA
:1082500092ED0B7AF8EEE77AB0EEC77AB4EEE77AF1
:10826000F1EE10FA3EDC05F5805305F5995693F8CA
:10827000A43513F0010406F1080629D0C3F3400821
:108280009B0732D495F8E41395F828444FF0B009D1
:1082900009FB015191F8C1314CBB022B18D968463A
:1082A0001AF050FA6946304615F054F8044678B191
:1082B00095F8E43309FB03534246D3F8D0116846DE
:1082C0001AF046FA15F01CFB694614F031FF04461B
:1082D000384617F00FFE304614F048FE2846FAF7ED
:1082E0008BFB204605B0BDE8F0830024F0E7444650
:1082F000EEE70020F6E700BF442B002038B50C4B1A
:108300001B680546D86A0C46F9F70EF910B100242F
:10831000204638BD15F0F4FA214614F009FF044652
:108320000028F4D005F5AC402FF016FDF0E700BFB3
:10833000442B0020F0B500F5A04300F5C046002214
:1083400083F8932583F8942506F16403044600EE30
:10835000101A0FCB87B006F1540585E80F0002AD67
:108360003246B8EEC00A2846164964324BF0B6F8D9
:1083700095E80F0006F1740787E80F0040F25712E6
:10838000394620460197FFF753FE01992046FFF733
:108390004FFB01992046FFF75DFB04F50053204693
:1083A000B3F95232002BB4BF4FF0FF33012386F8EC
:1083B0002C30FFF7B7F8204607B0BDE8F04006F0D4
:1083C00071BF00BF5062002010B5034904464BF056
:1083D00085F8204610BD00BF50620020F8B500F5BA
:1083E000C04505F1640304460E460FCB05F1540762
:1083F00087E80F0006F108012046FFF767FEB28804
:1084000002EB820202EB8202920012B204F5A04358
:10841000002AD8BF4FF4C872A3F88E252A6DA96F21
:108420005068091AC3F8601591680A31E967D26883
:108430000A32C5F880200022C3F8742583F89025FD
:1084400083F8A425C3F8642503F5AB62002111600D
:108450004FF0FF32C3F8502594F8411404F58662BA
:10846000242000FB012203F5B163D26A1A60F8BD33
:1084700070B50E4608310446FFF728FEB38804F5B0
:10848000A04543B3642213FB02F3C5F86035B5F988
:108490008E35002BD8BF4FF47A7304F53350D8BF14
:1084A000A5F88E35242200211030B8F09BF904F590
:1084B000C04304F5BF4093ED280A3146143089F0DB
:1084C00073FAD5F8DC35072B0CD120460421BDE822
:1084D0007040F9F755BFD5F86035002BD7DC40F672
:1084E000B833D2E770BD000030B5083104460FC97B
:1084F00085B06D4685E80F0004F5C041643128461B
:108500001AF08AFA20462946FFF7E0FD04F5804478
:108510000123C4F8C83F05B030BD00000B7A00F558
:10852000C04013F0020F14BF4FF0FF33012380F857
:108530002C3070477FB501F1080305460E460FCB7E
:108540006C4684E80F0005F5C041643120461AF0FE
:1085500063FA21462846FFF7B9FD31462846FFF762
:10856000DDFF04B070BD00007FB501F108030446D3
:108570000E460FCB6D4685E80F0004F5C04164310F
:1085800028461AF049FA29462046FFF79FFD204663
:108590003146FFF7C3FF337907EE903A337E9B07EE
:1085A00048BF9FED0A7AF8EE677A04F5C04448BFE9
:1085B00067EE877A9FED067A67EE877A0123FCEEF5
:1085C000E77A6364C4ED097A04B070BD0000803BB3
:1085D00000A00C477FB501F1080304460E460FCBFF
:1085E0006D4685E80F0004F5C041643128461AF055
:1085F00013FA29462046FFF769FD20463146FFF76A
:108600008DFFB38804F5C0444FF47A725343E3639B
:108610000123636404B070BD2DE9F34100F5C0454A
:108620000446743500F5C0400E46543029461AF011
:10863000B3F904F5A047C8B94FF0FF33C7F8503578
:1086400006F1080738461AF0ADF8032802463BD178
:10865000F16828461AF07CF8B28804F5C043204639
:108660005A6402B0BDE8F041FEF736BE23F0E4FDE7
:10867000F9F7DEFB012812D94FF0FF33C7F8503568
:1086800023F0DAFD90F8C432DFED140AB02202FBC9
:10869000030090ED300A28461AF05CFCD0E704F5A0
:1086A0008058D8F828052BF0BFFA08F5A563C7F85D
:1086B0005005D3ED007A9FED0A0ADFED080AF8EEC7
:1086C000E77A27EE800AE6E701AA002138461AF089
:1086D00075F80028C0D001990022BAE700007A445A
:1086E0000AD7233C7FB501F1080304460E460FCBA1
:1086F0006D4685E80F0004F5C041643128461AF044
:108700008BF929462046FFF7E1FC20463146FFF76A
:1087100005FF04F5C0440023636404B070BD00008D
:1087200037B504460D468DF00FF82062D5ED027A7C
:10873000F5EEC07AF1EE10FA15DD9FED127A67EED4
:10874000877AFCEEE77AC4ED077A5EF033FEE269E1
:108750004FF47A73B2FBF3F30B4A062103B0BDE882
:10876000304057F09FBF69F0EFFA0023009395F96E
:108770000D2095F90E3095F90C1069F081FAE06141
:10878000E3E700BF00007A4440AA0D082DE9F0435A
:108790002DED028B85B0044615F0B2F814F098F96F
:1087A00004F5805304F5A04693F820380BB900284F
:1087B00077D0D6F85035013373D1D6F87435002B05
:1087C0004BD08CF0C1FFD6F87435C01AB0F5FA6FF3
:1087D00067D394F8E423DFED5F7A9FED5F8A4FF073
:1087E000B00808FB024292ED780A20EE270A2BF02F
:1087F00033FA06F5AB69D9ED007A30EE670A2BF053
:108800002BFADFED567A20EE080A04F5515720EED8
:10881000270A2BF0C9F9FDEEC07A283717EE905AD7
:10882000C6F85055D9ED007A67EE887A17EE900AAF
:10883000F7F76AFECDE9020194F8E43308FB03433D
:10884000D3F8DC01F7F760FE454ACDE900012B467D
:108850000621384657F026FF23E004F59070F9F71B
:10886000E7FA02281DD994F8E433B02202FB03434F
:1088700093ED777AF1EE047AB4EEE77AF1EE10FA3E
:108880000FDD384B1B68D86A0368DB6998470128FD
:1088900003D08CF059FFC6F87405D6F87435002B58
:1088A0008FD104F54053D6F85015D3F884064A1CEE
:1088B000036846D01B6B98472B4810F0ADFC18B1ED
:1088C00004F5AC4031F0A8FC2046FEF715FED6F8C2
:1088D00060358342054637DA07EE905A9FED237ADA
:1088E000F8EEE77A04F5515767EE877A283717EEE6
:1088F000900AF7F709FE1E4ACDE900013846062125
:1089000057F0D0FE04F5C0444FF0FF330125C6F800
:10891000503586F8905504F164030FCB04F15407E9
:10892000743487E80F0084E80F00124869F088FB70
:10893000002386F89335284605B0BDEC028BBDE8D0
:10894000F0835B6B9847B7E7074810F045FC0028B9
:10895000C2D1F1E735FA8E3CE02E65420000C842F4
:1089600050AA0D08442B0020482B00200AD7233C96
:1089700074AA0D08684C0020F8B500F5C04600F553
:10898000C045543674350446294630461AF004F87A
:1089900004F5405730B304F5A043D3F850154B1CF1
:1089A00020D0D7F8840603681B6B984704F5C045B0
:1089B0006B6C012B44D06B6C022B05D12046FEF76B
:1089C00059FDAB6F984241DD2046FEF753FDAB6F7A
:1089D000C01A0028B8BF4042B0F5FA7FCCBF0020D3
:1089E000012034E004F5C040294664301AF00CFA46
:1089F000DFED177AB4EEE70AF1EE10FA16D530463D
:108A000029461AF0D1F89FED137ADFED130AF6EE3E
:108A1000007AE0EE077A28469FED100AFDEEE77A2D
:108A2000F8EEE77A27EE800A1AF094FAD7F884066F
:108A30009FED0B0A03682A469B6A31469847B5E7C3
:108A40002046FEF717FDAB6F9842B4DB0120F8BD5E
:108A500000004843A00CB345000096430AD7233CCE
:108A60000000000073B5384CD1ED026AD4ED1A7ADB
:108A70009FED367AF8EEE77A0546D7EE876A0E461E
:108A8000F5EEC06AF1EE10FA08DD5EF093FC304AB4
:108A9000062157F007FE012002B070BDD1ED037A28
:108AA000F5EEC07AA4F52964F1EE10FA94ED006AAF
:108AB00012DDF4EEC67AF1EE10FA0DD55EF07AFC16
:108AC00005462068F7F720FD224ACDE9000106217E
:108AD000284657F0E7FDDEE7DFED1F7A337CB4EE82
:108AE000E76AF1EE10FA54BFB0EE677AB0EE467A5C
:108AF0000BB90020D0E7B5EEC06AF1EE10FA0CDC3D
:108B000086EE876A03EB830307EE903AF8EEE77A86
:108B1000F4EEC67AF1EE10FAEBD595F82440002C6D
:108B2000E7D18CF011FEAB6AC01A337C4FF47A7235
:108B300053439842DDD9012385F824308CF004FE9C
:108B4000A8622046A8E700BF488B00200AD7233C34
:108B500090AA0D08A1AA0D080AD723BC38B505466E
:108B60007BF05AFF7AF038FD044640B98CF0ECFDFA
:108B70002B6AC01AEB69984284BFEC61012420463D
:108B800038BD000038B504460D468CF0DDFD04F517
:108B9000C0439FED067A9864D5ED027A67EE877A36
:108BA000FDEEE77AC3ED117A38BD00BF00007A44CC
:108BB00010B504468CF0C8FD04F5C0439A6C801AC9
:108BC0005A6C90424FF0000084BF5864012010BDE1
:108BD00000F5C04300F5AA415A6C91ED1E7A22EAD5
:108BE000E27207EE902AF8EEE77A0020B4EEE77A18
:108BF000F1EE10FA44BF58640120704710B500F53B
:108C0000005300F5C040B3F95232002BB4BF4FF00F
:108C1000FF33012380F82C3000F1740464300FC856
:108C200084E80F0010BD000038B504462DED028B1E
:108C3000F0EE408AB0EE608A09B301295ED0B5EE4D
:108C4000C08AF1EE10FA69DDDFED357AB4EEE78A1D
:108C5000F1EE10FA62D8FCEEC87A04F5515017EE26
:108C6000903A304A0621283057F01CFDFDEEC87AB4
:108C700004F5005417EE903A84F81F323CE0F8EE09
:108C8000000A2AF0EBFE40B104F580444FF0FF33B8
:108C9000C4F8D83FBDEC028B38BD04F50053B3F9DE
:108CA000282207EE902AF8EEE77AF4EEE87AF1EE61
:108CB00010FAC4D8B3F92A3207EE903AF8EEE77A00
:108CC000F4EEE87AF1EE10FAB9DBDFED157A68EE32
:108CD000A77A04F58043FDEEE77A04F5515017EECC
:108CE000902AFCEEE87AC3F8D82F062117EE903AC6
:108CF0000D4A283057F0D6FC0120CBE7FCEEC07AB5
:108D000000F5515017EE903A084A0621283004F534
:108D1000005457F0C7FCC4ED8D8AEDE70020B9E799
:108D20000000C842E7AA0D08C0AA0D08D4AA0D0881
:108D3000D1F80D3000EE903AD1F80930097A00EE02
:108D4000103AFFF771BF000070B58B88012B044605
:108D50000D4611D100F590763046F9F769F80228F2
:108D60000AD994F8E413B02303FB01612046AC3127
:108D7000BDE87040FFF7C2BA14F0C2FD05F108016A
:108D8000BDE8704014F0D4B9F0B500F5A047002458
:108D9000AB4B87F8994589B0054608460E4683F8DF
:108DA0008D402EF0EBFDA0B3012387F8903505F53B
:108DB0004053D3F884060368DB6B984705F5C0433E
:108DC00087F8974503A81C6319F0BCFCB7F83C165C
:108DD0004FF6FF73994208BF2146013101AA89B2BB
:108DE00005F5AC4030F09AFDF0B1BDF80630A3F1C6
:108DF00015025342534187F8913550B105F5C240F1
:108E0000BDF80610383008F083FC10B1002387F855
:108E1000913573885E2B4DD8522B07D8103B9AB2F0
:108E20000F2A21D90024D4E00346E4E7533B0B2B5F
:108E3000F8D801A252F823F0CD8F0108D98F01088C
:108E4000E98F0108258E0108258E0108258E01086D
:108E5000258E0108258E0108258E0108258E010822
:108E600035900108E98F01080F2BDBD801A252F8D9
:108E700023F000BF518F01088B8F0108958F0108E7
:108E80009F8F0108B38F01085D8F0108238F0108B0
:108E9000258E0108258E0108258E0108258E0108E2
:108EA000258E0108258E0108258E0108C38F010833
:108EB000A98F0108BD2B1AD8BB2B47D8B22B00F0C5
:108EC000A7800DD8702B00F09E80722BAAD1D6ED12
:108ED000027AFDEEE77A05F5C045C5ED117A35E079
:108EE000B32B9FD131462846FFF72EFF2EE0D42B1F
:108EF00000F0938040F6B832934200F09680D22B77
:108F000090D1B388012B21D803F0010387F8923563
:108F100005F55150B3884B4A0621283057F0C2FB63
:108F200014E0002305F5C24487F8C9353834718848
:108F3000204607F095FE314628B1204609B0BDE82D
:108F4000F04008F08FB82846FFF748FA012440E0C7
:108F500006F108012846FFF7B9F8F7E705F5C2441E
:108F600038341521204608F0D3FB48B1002387F898
:108F7000C9353146204609B0BDE8F04007F076BF5C
:108F800031462846FFF774FAE0E731462846FFF7F6
:108F9000D1FADBE731462846FFF7E6FAD6E7314655
:108FA0002846FFF717FBD1E731462846FFF79AFB23
:108FB000CCE705F59A4129222C3128460EF088F895
:108FC000C4E731462846FFF727FBBFE7012487F8AF
:108FD0009745204609B0F0BD002305F5C24087F84B
:108FE000C93531463830A9E705F5C2473837384624
:108FF00008F072FB3146044618B12846FFF774FAB0
:10900000E7E73846B7E731462846FFF7BBFD9DE75F
:1090100031462846FFF78CFE98E7B188003918BF23
:109020000121284600F002FF90E7317A064807F058
:1090300015FA8BE7314605F59A40FFF771FB85E796
:10904000488B0020F8AA0D08808C002000F5804293
:1090500000F59A43D2F8A02F9A4201D1FFF794BEAF
:109060000120704710B500F5804200F59A43D2F810
:10907000A02F9A4204460DD1194608222C310EF039
:1090800027F804F55150044ABDE810400621283065
:1090900057F008BB10BD00BF08AB0D082DE9F04F1D
:1090A0002DED048B00F5C04898ED6E8ADFEDD67A81
:1090B000B0EEC87AB4EEE77AF1EE10FA48BF00F5E8
:1090C0000053DFEDD27A42BFB3F9523208EE103AC4
:1090D000B8EEC88A00F58045B4EEE78AF1EE10FAE2
:1090E00094BF4FF0FF37012788F82C70D5F8C83FA0
:1090F0009BB004460E46F0EEC88A052B16D8DFE872
:1091000013F006002B0068008700C4005F0100F523
:1091100040543A46D4F884060368B0EE680ADB6A25
:1091200008319847BA4806F0F7F808B9002048E136
:10913000B84C236DB4F9F8115B68642201FB02316D
:10914000A4F5C040FFF7F6F8A4F5C04005F0BEFC5A
:109150000123C5F8C83FE9E700F540533A46D3F884
:1091600084060368B0EE680ADB6A08319847D8F8CD
:109170002830002BB8BF5B42012BD7DD98F82D308B
:109180001BB998F82E30002BD0D004F5B453D3ED92
:10919000040A93ED050AF1EE600AB1EE400AB5F05B
:1091A00027F9DFED9D7A20EE270A05F6CC7383EDD3
:1091B000000A10EE100AF7F7A7F904F55154283405
:1091C000CDE90001954A0621204657F06BFA0223AB
:1091D000BFE700F5C04901F1080A09F164094946F1
:1091E000504619F011FE30EE680AF1EE047AB0EE46
:1091F000C00AB4EEE70AF1EE10FA00F3E780D8F8FF
:1092000028300133022B40F2EB800323C5F8C83F1E
:1092100004F5405306F10808D3F8840603683A467B
:10922000DB6AB0EE480A41469847DFED7D6A9FED64
:109230007D7A05F6CC73D3ED007A012F18BFB0EE1E
:10924000667A04F5A95377EE877A93ED050A9FEDC8
:10925000767AA7EEC70A2AF0FFFCDFED747AB0EE4B
:10926000C00AB4EEE70AF1EE10FA7FF55FAF04F53D
:109270005150062128306E4A57F014FA0423C5F8DD
:10928000C83F41462046FEF721FF06F1080595E854
:109290000F000AAF0DF1380887E80F0088E80F00CB
:1092A00004F5804303F6CC7A9FED629A9AED000AAA
:1092B000DFED610A0393384630EE090A19F04AFEE1
:1092C000DFED5D0A9AED000A9FED5C8A404619F0D9
:1092D00041FE04F540534246D3F8840603683946FC
:1092E0009B6AB0EE480A984795E80F0004F5C2491A
:1092F0000DF1480B09F138098BE80F00DAED009AFF
:10930000484607F0D3FC79EE899A04F5C048F0EEA0
:10931000400A5846B0EE690A08F1640819F01AFECE
:109320005A463946404619F0DBFC834695E80F0063
:109330009AED000A16AF87E80F00F0EE680A30EEEB
:10934000090A384619F006FE394640462A4619F001
:1093500091FC04F5995007A90830F0EE408A8DED94
:10936000078A8DED088A8DED098A14F0C7F8002868
:1093700066D02946404619F053FC05A907A8CDED53
:10938000060A8DED050A2DF061FCDFED237A20EE53
:10939000270A2AF0F5FBB0EEC00ABBF1000F3FF43C
:1093A000C5AEF3EE0E7AB4EEE70AF1EE10FA23D56D
:1093B000039A0523C2F8C83F3146484607F056FDD8
:1093C00001201BB0BDEC048BBDE8F08F4946504630
:1093D00019F01AFDB4EEE80AF1EE10FA7FF50FAFBE
:1093E00004F540543A46D4F884060368B0EE680A9F
:1093F000DB6A5146984799E6F6EE007AF4EEE78A82
:10940000F1EE10FAD4DC91E600000034000000B464
:10941000482B0020488B0020E02E654230AB0D0821
:109420000000B4420000874335FA8E3CC2B8B23D1A
:1094300052AB0D080000344300007A4400000000E5
:10944000BBF1000F3FF472AEB2E700BFF0B50446C7
:1094500000F5C2408FB038300F4608F07DF9054660
:1094600038BB09AE304619F06DF904F5A0434FF64C
:10947000FF72B3F83C36934208BF0023013307AABA
:1094800099B204F5AC4030F049FAA8B104F5C044F3
:1094900007B1A56296E80F0001AD85E80F00D4F88A
:1094A00080300093743494E80E00044803F0B4F95B
:1094B000054628460FB0F0BD0125FAE79078002058
:1094C00070B5054605F5C046002106F015F8346B69
:1094D0006CB9284605F020FF10B90024204670BD65
:1094E000B36A012BF9DD8CF02FF93063F6E7716C6C
:1094F00049B18CF029F9336BC01AF36B9842ECD95F
:109500000023736401212846FFF7A0FF04460028CA
:10951000E3D005F55150054A0621283005F5A04550
:1095200057F0C0F8002385F89935D7E774AB0D08DC
:1095300038B50A468B88190A137EDB0748BF01EB52
:109540008101044648BF490005F0D6FF04F5A04359
:10955000002583F89955204605F0DEFE10B9002558
:10956000284638BD04F5C043596C39B1D3E9091216
:109570008A42F4DD012AF2DD5D6401212046FFF715
:1095800065FF05460028EAD004F55150024A06213D
:10959000283057F087F8E3E78CAB0D0838B505465F
:1095A00005F5C044898805F0A7FF636C6BBBA36A0F
:1095B000002BB8BF5B42012B02DC0024204638BDE3
:1095C00094F82D2094F82E306AB9002BF5D005F5CB
:1095D0005150A26E6423062192FBF3F328300C4A0B
:1095E00057F060F801E0002BF1D1012161642846B9
:1095F000FFF72CFF04460028DFD005F55150054A3F
:109600000621283057F04EF8D8E70021EFE700BFD9
:10961000A4AB0D08C2AB0D0810B504460B4808F00A
:109620007FFE48B10A4BDFED0B7AD3F8743193ED2E
:10963000090A20EE270A10BD04F50054B4F980325F
:1096400000EE103AB8EEC00AF5E700BF808C0020AB
:10965000488B00200AD7233C10B52DED028B00F576
:1096600000530446B3F984120029ACBF01224FF025
:10967000FF3200F5C0430029B8BF494283F82C20CF
:1096800089B205F039FF04F5AA43204693ED1E8AFE
:10969000FFF7C2FFB5EEC00AF1EE10FAD8BF9FED9A
:1096A0000E0ABCEEC00AB8EE400AB4EEC08AF1EE73
:1096B00010FA0AD804F551502830084A062156F00D
:1096C000F1FF0120BDEC028B10BD204605F024FE09
:1096D0000028EFD1F6E700BF00000000DCAB0D086A
:1096E0002DE9F04F00F5A0492DED028B4FF0FF332F
:1096F00000F5C04AC9F850350AF174030F46054613
:109700000FCBBC8897F8048089B004AE240A86E8A1
:109710000F001ED0574654373146384619F074FBB7
:1097200031463846B0EE408A19F03EFADFED567AFF
:10973000B4EEE78AF1EE10FA0BDBE3B200EE903AFA
:10974000DFED527AF8EE600A20EE270A304619F073
:1097500001FC05F5405B99F89425DBF884069FED44
:109760004C0A036805F5C0479B6A643732B305F5B8
:10977000C04132465431984705F50053B3F982325F
:10978000002B1EDD07EE903A09F5AF62F8EEE77A9E
:1097900092ED007AB4EEE77AF1EE10FA11DD05F5FC
:1097A000C04132465431384619F09AFAF8B90024CB
:1097B000204609B0BDEC028BBDE8F08F3246394639
:1097C000D9E7B8F1000F1CD1002C3CD1DBF884465E
:1097D00023682846D3F82080FFF71EFF09F26C5358
:1097E000D3ED000A2046C047B0EE408A0DE0002CC1
:1097F000DDD10AF164030FCB0AF1540585E80F00AF
:10980000D6E707EE908AB8EE678A3146384619F0F7
:10981000FBFAB4EEC08AF1EE10FA17DBB9F83C3669
:1098200003933146384619F0EFFABCEEC00A05F54D
:109830005150039B174A8DED000A0621283056F03F
:1098400031FF0124B4E79FED128ADEE705F5C04140
:1098500032465431384619F043FA04460028A6D05F
:10986000B9F83C3603933146384619F0CDFABCEED0
:10987000C00A05F55150039B074A8DED000A0621E9
:10988000283056F00FFF93E700000034E02E6542C9
:1098900000000000F4AB0D0812AC0D082DE9F047F4
:1098A0004B881F2B8AB004460D466BD80F2B41D82E
:1098B00004F55150BE4A0421283056F0F3FE9BE0D7
:1098C000A3F1BC02182AF3D801A151F822F000BF7D
:1098D000F9990108F9990108B1980108B1980108AE
:1098E000B1980108B1980108B1980108F9990108E7
:1098F000B1980108F9990108B1980108B1980108D7
:10990000B1980108F9990108B1980108B1980108C6
:10991000B1980108F9990108F9990108F999010824
:10992000B1980108B1980108F9990108B1980108A6
:10993000F9990108A3F110020F2AB9D801A151F831
:1099400022F000BF359A01081B9B0108259B0108E6
:10995000319B0108479B0108419A01080B9A0108B5
:10996000B1980108B1980108B1980108B1980108AF
:10997000B1980108B1980108B1980108519B0108FC
:109980003B9B01085E2B21D8522B91D9A3F15302A6
:109990000B2A8DD801A151F822F000BF5B9B010872
:1099A0006B9B0108759B0108B1980108B1980108EB
:1099B000B1980108B1980108B1980108B19801085F
:1099C000B19801089F9B0108759B0108722B00F05C
:1099D000E18007D8702B7FF46BAF0AB0BDE8F04789
:1099E000FFF7E6B8D42B09D8BB2B3FF669AFA3F13C
:1099F000B202012A3FF65CAF012052E0DF2BFBD020
:109A000040F6B8329342F7D052E700F5C2463836F6
:109A10001621304607F024F930B1294630460AB005
:109A2000BDE8F04707F00ABC20460AB0BDE8F047A1
:109A3000FEF7ACBE29460AB0BDE8F047FFF750BEBE
:109A400000F5C24538351521284607F061FE28B1DA
:109A500028460AB0BDE8F0470BF052B904F5A0451E
:109A600004F5BF46D5F8DC3504F5C04704F5C04819
:109A700004F5C049072B06F1140607F1540708F155
:109A8000740809F164090FD104F5AB44583401940A
:109A9000D5F86035009342464B463946304688F04B
:109AA00047F80AB0BDE8F0870DF127018DF82700CF
:109AB0004048FEF79DFA05F29C53D3ED007AD5F8A5
:109AC00080A505F5AE63D3ED000A05F27C5330EEB8
:109AD000670A93ED001A8DED070A04F5C140703056
:109AE000CDED060A8DED051A79F06CFD0546204690
:109AF00000F060FF9DF827309DED051ADDED060AA8
:109B00009DED070ACDE90203CDE900A54B4642468B
:109B10003946304687F062FFC3E7A98805F0ECFCC0
:109B20000020BEE729460AB0BDE8F047FFF700BDB8
:109B30000AB0BDE8F047FFF7C3BC29460AB0BDE84C
:109B4000F047FFF72BBD0AB0BDE8F047FFF784BD33
:109B50000AB0BDE8F047FEF70FBF294604F59A406A
:109B60000AB0BDE8F047FEF77DBF04F5C2402946C4
:109B7000383054E704F5C2463836304607F0ACFDBD
:109B800008B9304665E729462046FFF787FA0028DE
:109B9000F7D186E70AB0BDE8F047FFF719B82946C4
:109BA00004F59A400AB0BDE8F047FEF7D7BF00BF02
:109BB00030AC0D08482B002070B500F5804200F550
:109BC0009A43D2F8A02F9A4205460E4602D00024AE
:109BD000204670BDFFF762FE04460028F7D005F569
:109BE0005150318828305AF0A9FEF1E721F04003A6
:109BF000152B04D0A1F15E03584258417047012053
:109C00007047000000F5804200F59A43D2F8A02F7B
:109C10009A4207D100F5A040B0F83E365B1A584290
:109C20005841704700207047192962D8DFE801F0D9
:109C30000D1115191D2125282C6130333655393960
:109C40003C3F4246494D6151595D00F59B402030F3
:109C5000704700F597407430704700F59840103019
:109C6000704700F598402C30704700F59840483018
:109C7000704700F599400430704700F59940E6E7D9
:109C800000F599403C30704700F5994064307047CA
:109C900000F59A40704700F59A40E4E700F59A40D5
:109CA000E5E700F59A40F1E700F59B40E3E700F5B2
:109CB0009B40E7E700F59B405830704700F59B401C
:109CC000C9E700F59C401430704700F59C403030E7
:109CD000704700F59C405030704700F59D400830BB
:109CE000704700F59D404430704700F59C406C3053
:109CF000704700207047000000290DDB074890F8EE
:109D0000CC2CCBB29A4207D3D0F8C83C0122595C84
:109D1000A0F500500DF0B4BA704700BF484B0020CA
:109D20002DE9F34100F5005300F5515593F8983CA7
:109D300003F0010603F0020803F004075B07044682
:109D400005F1280535D01F4A0621284656F0AAFC01
:109D500026B104F53F501C307BF06CFCB8F1000FCD
:109D600004D004F5445034307BF0E0F927B104F519
:109D70004A500C307CF088F804F5C044012384F884
:109D80008934114A114B1249B8F1000F08BF1A4625
:109D9000002F08BF1946CDE900210E4A0621002EEA
:109DA00018BF134628460C4A56F07CFC02B0BDE8AA
:109DB000F0810A4A0621284602B0BDE8F04156F07B
:109DC00071BC00BF5DAC0D0852AC0D08D0950E08FB
:109DD00059AC0D084CAC0D086EAC0D0880AC0D08EC
:109DE00010B5044600F53F501C307BF04FFC04F5E5
:109DF000445034307BF0C6F904F54A500C307CF006
:109E00007DF804F5C04393F889245AB1002283F801
:109E1000892404F55150044ABDE810400621283039
:109E200056F040BC10BD00BFA0AC0D0809B1FFF753
:109E300077BFFFF7D5BF000000F580430949D3F88D
:109E4000A02F8A420CD093F8AD3F3BB900F59A4160
:109E50008A4203D100F5A04090F892351846704729
:109E60000023FBE7E878002010B504468BF06CFC7B
:109E7000054BD3F8C03FC01A642804D82046BDE87B
:109E800010405EF0BDBC10BD486B002010B500F561
:109E90003254D4ED027AF5EEC07AF1EE10FA8AB0BF
:109EA0004FF0000304F1080445D907930893099380
:109EB00006AB019300F5995007AB009303AA05ABDD
:109EC00004A9083013F0BAF930B3DDED080A9DEDAE
:109ED000070AB4F0F1F8DDED090AB4F0EDF8D4EDBD
:109EE000007A9DED047A77EEA76AB4EEE70AF1EE08
:109EF00010FAF4EEC76AACBF01200020F1EE10FAB0
:109F00000CD802309DED037AF4EEC77AF1EE10FA28
:109F10000CD8003818BF01200AB010BDF4EEC77A83
:109F2000F1EE10FA9CBF0130C0B2EBE7012894BFFC
:109F300000200120F0E70020EEE7000038B5124BCA
:109F40001A7A0446FAB901251D7253F053FA2A46CB
:109F500004F5C2451121383553F004F8284607F0BE
:109F60003FFC80B1284607F0F7FB062238B104F524
:109F70009C411431BDE8384004480DF0A9B804F5FF
:109F80009B415831F6E738BDE88F0020482B002070
:109F900010B5074B1A7A4AB100241C7253F02AFA02
:109FA00022461121BDE8104052F0DCBF10BD00BFB9
:109FB000E88F00202DE9FF41054605F599586846D0
:109FC00008F1080818F0BEFB6946404613F08AFA0B
:109FD0000646E8B1374879F0F5FA50B105F5325345
:109FE000D3ED027AF5EEC07AF1EE10FA94BF0126B5
:109FF000002605F5C240383007F0F2FB2E4C2F4FFB
:10A0000000B146B1002328462380FB73FFF7C0FF51
:10A0100004B0BDE8F0812846FFF738FFA0B36378AD
:10A020007BBB23780133DBB2082B237002D140467F
:10A0300013F070F92378092B02D1404613F062F92E
:10A040002378092B1DD94FF48573238053F0D2F95F
:10A050000222102152F086FF8BF076FB6368C01A53
:10A0600047F23053984209D905F55150144A02215C
:10A07000283056F017FB8BF067FB60602846FFF72F
:10A080005DFF6378FB73C3E72378002BF9D0013BB6
:10A090006278DBB22370002AF3D0002BF1D1667016
:10A0A00053F0A8F93246102152F05CFF2846FFF722
:10A0B0006FFFE6E7388C0020E88F002095900020A5
:10A0C000B4AC0D0810B500F5A044D4F8DC35042B71
:10A0D00001D1012010BD00F5C240383008F006F96A
:10A0E0000028F6D194F80806F4E7000073B500F5EF
:10A0F00080450192A5F8B81F04468BF025FBC5F8F2
:10A10000BC0FD5F8A00F03685B68984785F8B60FB9
:10A11000D5F8A00F03685B689847019A182818D8EB
:10A12000DFE800F00D170D0D0D0D0D0D0D17521779
:10A130005917595917414141171717415900334BC6
:10A1400093F88A3403B304F59941043120460CF0A6
:10A15000BFFFD5F8A00F95F8B66F03685B68984706
:10A1600004F55154864204F1280447D0D5F8A00FD5
:10A1700003689B689847264A03460421204602B09C
:10A18000BDE8704056F08EBA04F5005393F994324E
:10A19000022BD8D0042B0BBF04F5994104F597414D
:10A1A00020317431D2E704F5C043D3F8FC33D9022F
:10A1B00003D504F59A412C31C8E704F59C419B0670
:10A1C0004CBF30311431C1E720460192FFF77AFFCE
:10A1D000019A0028BDD104F50056019296F99432F7
:10A1E000002BB6D0D5F8A00F03685B68984785F8B8
:10A1F000B60F96F99432019A022BCAE7054A042158
:10A20000204602B0BDE8704056F04CBA488B0020A2
:10A21000C4AC0D08E6AC0D08F0B5044604F5804664
:10A2200085B00F4615465EF071FAD6F8A00FA6F875
:10A23000B87F03685B68984718281ED8DFE800F0ED
:10A240000D0D0D0D0D0D0D0D0D1D607D0D0D6C6CAD
:10A250001D4E4E4E1D1D1D4E0D003B4BD3F8DC25F3
:10A26000012A21D104F5005393F89532023B012BCA
:10A270001AD904F5405383F86424D6F8A00F334A62
:10A28000334B052D18BF134602680393926890471D
:10A2900004F5515428340090039B2E4A0421204693
:10A2A00056F000FA05B0F0BD2B4B93F88A343BB161
:10A2B00004F599412A46043120460CF009FFDCE7F9
:10A2C00004F5005393F99532032BD6D0022BEFD02F
:10A2D000042B2DD12A4604F59A41EDE704F5C0433D
:10A2E000D3F8FC33DA0223D49B0604D504F59C4151
:10A2F0002A463031E0E704F59C412A461431DBE779
:10A300002046FFF7DFFE0028B7D104F5C240383001
:10A3100007F090FA0028EED104F5005393F9953236
:10A32000032BAAD0022BC3D0042BD3D0012BA4D152
:10A3300004F59A412A462C31BEE704F5005393F9FF
:10A340009532042B99D1C5E7487B0020FCAC0D0861
:10A35000F3900D0804AD0D08488B002070B500F592
:10A36000515504462835124A0421284604F58046F2
:10A3700056F098F90023A6F8B83F04F5005393F877
:10A38000DC31032B12D196F8B61F302220460CF098
:10A3900077FFD6F8A00F03689B689847054A0346E5
:10A3A00006212846BDE8704056F07CB970BD00BF5C
:10A3B00018AD0D082FAD0D0800F5405310B5002263
:10A3C0000529044600F5515083F8642400F1280063
:10A3D0000CBF054A054A042104F5804456F062F991
:10A3E0000023A4F8B83F10BD48AD0D0859AD0D08C5
:10A3F000013A38B50446052A3ED8DFE802F04A1B88
:10A4000086113D0300F5C04393F84C3243B100F58B
:10A410009C4104226C314148BDE838400CF058BEE4
:10A4200004F5C04393F84C3223B104F59C41042257
:10A430001431F0E704F58043D3F8A02F04F59C43D2
:10A4400014339A4225D004F59C436C339A4220D0B1
:10A4500004F5A043D3F8DC35042B1AD0304D95F821
:10A46000D13FB3B12F4905F5B0502FF029FE20B1EF
:10A470002D4B012283F8082638BD2A4905F5B05036
:10A4800030F01EF928B1042204F59A41A5F5804068
:10A49000C2E704F58043D3F8A02F04F59C4314339E
:10A4A0009A42E9D004F59C436C339A42E4D004F517
:10A4B000A04304F5C2403830D3F8DC5507F016FF4E
:10A4C0000028D9D1042DD7D004F5005393F95F3279
:10A4D000022B0DD004F59A41204604222C310CF0B9
:10A4E000F7FD04F508501F30BDE8384048F054B877
:10A4F0000B4890F8D13F002BECD00A4900F5B05042
:10A500002FF0DEFD0028B3D1E4E700F5C140BDE83F
:10A510003840012214217030F7F73ABB482B002055
:10A52000486B0020AC8B0020487B002070B52DEDDF
:10A53000068B04468BF0FCF8414BB4F8BE101A8829
:10A54000404E8A420546404A06D0198000233060BA
:10A550001370BDEC068B70BD33683C49C31A8B4247
:10A5600065D9012313705EF0D1F95EF089F835608A
:10A570005EF0CCF95EF084F85EF0AAF80428E8D921
:10A580005EF0C4F8204600210AF0CCFF20460021EE
:10A59000B0EE40AA0AF0D0FF20460121F0EE409A2A
:10A5A0000BF096F900212046B0EE408A0AF0CEFF6B
:10A5B00004F5C1407030F0EE408A79F00DF89FED5F
:10A5C000249A0028B0EE4A0A4FF0040008BFB0EE0B
:10A5D000498A5FF043FCB0EE690A13205FF03EFC4D
:10A5E000B0EE680A15205FF039FCB0EE680A1A2058
:10A5F0005FF034FCB0EE480A46205FF02FFC0121EA
:10A6000008465FF037FFB0EE490A02205FF026FCF3
:10A61000B0EE490A03205FF021FC20460BF08CFBD2
:10A62000BDEC068B2046BDE870400CF0DDBA127818
:10A63000002A8ED044F6206293428AD993E700BF65
:10A64000F48F0020F88F0020F68F0020400D0300CB
:10A650000000000000F5804200F59A43D2F8A02FD8
:10A660009A4204D100F5A04090F80806E8B10F4BDB
:10A6700093F8DC0103F58043A0F12702012A93F847
:10A6800098340FD92C2809D00A2809D0A0F131021A
:10A69000504250410A2B18BF002070470120F9E7B3
:10A6A000012070470A3B584258417047484B0020F0
:10A6B00008B500F5005393F8202142B193F85C31BE
:10A6C0002BB1FFF7C7FF80F00100C0B208BD012029
:10A6D000FCE700002DE9F04700F50055AF4F95F875
:10A6E0005C81044600F5C1408AB0703078F06AFFA2
:10A6F000D7F8DC35042B064642D1012104F5045776
:10A70000DFF8ACA22037384668F000F89AF89834A1
:10A710000A2B814604D1002E54D100238AF89834A4
:10A7200095F82031002B59D195F926319C4D012BFC
:10A7300003D0063BDBB2012B11D895F8DC310A2B94
:10A740000DD104F58046D6F8A00F03681B6A984720
:10A7500028B1D6F8A41F2B2220460CF0B9FC9AF899
:10A7600098340A2B04BF37238AF8983495F8DC31E3
:10A770000A2B02D1372385F8DC310AB0BDE8F08717
:10A780000028BAD004F58043B7F83E96D3F8A00F5E
:10A7900003685B6898471428AFD004F5C24038308E
:10A7A00007F0F2FB0028A8D14946A7F5A040FFF723
:10A7B0001DFA01460028A1D097F804164B1E5942F5
:10A7C00059419BE740EA0803DBB2002BA8D1AAF568
:10A7D000C04000F0EFF800289FD0A1E7002ECCD0B9
:10A7E00004F5BF40143087F06FF80028C5D120462B
:10A7F000FFF730FF0028C0D1B9F1000F00F0BD8095
:10A8000068494A46384667F059FB95F92681B8F100
:10A81000010F06D040F38580A8F10603DBB2012BBF
:10A820007FD85FFA88F8B8F1010F4DD104F5804266
:10A8300004F59A43D2F8A02F9A4209D104F5A04317
:10A8400093F8083623B195F85F32013B012B94D978
:10A8500004F59A410A222C31204606AE0CF038FC51
:10A86000304617F06FFF95F9392192BBB8F1010F0F
:10A870002FD004F5C048B5F93A31D8F85010DFEDC3
:10A880004A5AD1ED017A002BF8EEE77A52DD07EE55
:10A89000103AF8EEC76AE6EEA57A3046FDEEE77AA2
:10A8A00017EE901A17F054FF00233846CDE9043311
:10A8B00067F0C8FF04A968F009FD002857D0049B81
:10A8C0000893059B099317E004F59A410A22643125
:10A8D000C2E72046FCF71EFC07EE900A6F4604F51F
:10A8E000C042643221463846B8EEE70AFDF76CFDF7
:10A8F00097E80F0086E80F0095F92631012B10D05C
:10A9000031462046FDF794F831462046FDF744FCD9
:10A9100095F92631072B04D104F54054012384F81E
:10A92000623452F067FD4A4609210AB0BDE8F0479B
:10A9300052F018BBD5ED4A6A95ED4D5A95ED4B7A1C
:10A9400035EE076A36EEC57AB4EEC67AF1EE10FA45
:10A9500089BF37EE067A95EDB07A27EE257AF6EEC6
:10A96000006A94BFE7EE257AE7EE267A95E7D8F8F5
:10A9700050309A680892DB68A4E7B8F1000F3FF402
:10A98000FCAE95F85C31002B7FF4F7AE04F5515026
:10A99000064A0521283055F085FEC2E7487B002095
:10A9A000484B002074AD0D080000C8427DAD0D0875
:10A9B000488B002010B5044600F5C140703078F097
:10A9C0000BFE98B104F5C240383008F085F960B943
:10A9D00004F5AB4494ED187ADFED087AB4EEE77A2B
:10A9E000F1EE10FAACBF0120002010BD04F5AB441D
:10A9F00094ED187ADFED027AF0E700BFCDCCCC3DC4
:10AA00006666663F70B500F5804600F59D43D6F852
:10AA1000A02F08339A42044600F5A04502D195F8CC
:10AA2000D805D0B904F5C240B5F83E16383006F066
:10AA300017F998B9D6F8A03F04F59A44A3420CD16F
:10AA400095F8D8354BB1D5F8DC35032B05D1B5F8E1
:10AA50003E06A0F116035842584170BD0020FCE7A5
:10AA60002DE9F74F00F5804200F59A43D2F8A02F68
:10AA70009A42044600F5A04504D100F5005B9BF91D
:10AA800038323BB90023C5F8CC3585F8C93503B059
:10AA9000BDE8F08F8AF058FED5F88465804636B15F
:10AAA000861B40F6C3139E4294BF00260126204613
:10AAB000FFF780FF019028B1002785F8C8754FF097
:10AAC000000A46E004F5C140703078F07BFD814615
:10AAD0000028F1D004F5BF4A0AF1140A504686F066
:10AAE000F3FE0746002845D095F8C8A5BAF1000F37
:10AAF0003BD156B304F5805041F27071D0F8202557
:10AB0000002AB8BF52428A4206DCD0F82425002A27
:10AB1000B8BF52428A422BDD04F5AC4104F5C04077
:10AB20004431643018F070F9DFED487AC5F8CC850F
:10AB3000B4EEE70AF1EE10FA4FF000024CBF4FF00E
:10AB4000010A4FF0000AC5F8D025012285F8C82572
:10AB5000374604F59070F7F76BF9022832D9002FC9
:10AB600044D10023C5F8CC3591E7019EB246ECE70D
:10AB70005646EAE7504686F08FFE824648B1002EE0
:10AB80009DD04FF4FA73C5F8D0354FF0000A4F4608
:10AB9000DFE7D5F8DC25012A07D0032AD9D12046E2
:10ABA000FFF730FF00288AD1E9E7DBEDB67AF5EE52
:10ABB000C07AF1EE10FA82DD95F8D835002B7FF4DB
:10ABC0007EAFDEE704F5FB5604F50059083699F828
:10ABD000B610304610F03EFB0028C2D099F8B610EF
:10ABE000304610F02FFC0028B9D1BAE7D5F8CC05D3
:10ABF00010B9C5F8CC854AE7D5F8D025A8EB0008F0
:10AC00009045FFF444AF95F8C925002A7FF43FAF83
:10AC1000012285F8C9259BF83812CB0705D504F524
:10AC2000C1400C217030F6F7B3FF04F551502830C5
:10AC3000BAF1000F06D0064A022103B0BDE8F04F7A
:10AC400055F030BD034A5146F7E700BF0000964279
:10AC500094AD0D08AAAD0D082DE9F04F2DED028B36
:10AC6000044685B0002304F5005903938AF06CFD77
:10AC7000D9ED8D7AF5EEC07AF1EE10FAC4BF9FEDF2
:10AC8000C47A67EE877A04F5907BC8BFFCEEE77A5A
:10AC900080465846CCBF17EE907A9627F7F7C8F84B
:10ACA000022840F2028194F8E4339FEDBA7AB02290
:10ACB00002FB0343D3ED777A67EE877AFCEEE77AFF
:10ACC00017EE903A9F428CBF00270127B9F928322E
:10ACD000022BB8BF022307EE903A04F59950B8EE64
:10ACE000E78A03A9F6EE087A083028EE278A12F0E0
:10ACF000D7FB054640B1DDED037AF4EEC87AF1EEFC
:10AD000010FAACBF012500255846F7F791F8012845
:10AD100004F5A0461AD804F5C140703078F052FC12
:10AD2000A0B19DB906F5BC6393ED007ADFED9A7A88
:10AD3000B4EEE77AF1EE10FA08DDDDED037AF4EE19
:10AD4000C87AF1EE10FAACBF0125002504F5C24027
:10AD5000383005F0DDF98246002840F0F78004F530
:10AD6000C140703078F02EFC002800F0FD8094F88F
:10AD7000E43304EB0313D3F890317BB158460193CD
:10AD8000F7F756F8012800F29280019BA8EB030028
:10AD900041F2873398428CBF00230123D6F88025E7
:10ADA00002B11BB9002D40F084803D4604F580427D
:10ADB00004F59A43D2F8A02F9A4219D199F960323A
:10ADC000002B7ED1002386F8CA35D6F8DC35042B5B
:10ADD00000F0A880072B00F0BB80032B08D1204691
:10ADE000FFF710FE20B1002586F8C955C6F8845536
:10ADF00096F8CA3503B18DB907EE905A9FED677A80
:10AE0000F8EE677A06F5BC6367EE877AD3ED006AE1
:10AE10009FED637AE6EE877AC3ED007A2046FFF76E
:10AE2000C9FD0546A0B196F8E415C6F8808509B9B4
:10AE3000C6F8E88504F5804204F59A43D2F8A02FBD
:10AE40009A4205D1D6F8843503B109B9C6F884858C
:10AE500086F8E45571F046FB294671F01FFB514B13
:10AE600020465D71FFF7FCFD2046FAF7BBFB35B1CC
:10AE700099F8DE311BB98AF067FCC9F8E00189F85E
:10AE8000DE512046FFF796FD00287ED104F5C14033
:10AE9000703078F0A1FB80F00100C0B286F8EC05BC
:10AEA00005B0BDEC028BBDE8F08F00270EE75346DE
:10AEB00074E728F063F927F057F900287FF475AF9D
:10AEC00074E75B4207EE903A04F6E853F8EEE77A4F
:10AED00093ED007AF4EEC77AF1EE10FA13DD012358
:10AEE00086F8CA35C6F8D48506F5BC63DFED2E7A40
:10AEF00093ED007AB4EEE77AF1EE10FA7FF765AFE2
:10AF0000C3ED007A61E796F8CA35002B3FF45DAFD8
:10AF1000D6F8D43540F6B832A8EB030393423FF697
:10AF200051AF52E704F5BF40143086F0B5FC00285D
:10AF30003FF45EAF06F5AE6393ED007ADFED1A7A6B
:10AF4000B4EEE77AF1EE10FA7FF752AF01254FE742
:10AF500006F5AE6393ED007AFEEE007AB4EEE77A82
:10AF6000F1EE10FAF2D443E7D6F8DC35002D18BF25
:10AF70003D46012B01D100253AE704F5BF401430CE
:10AF800086F080FC0028F6D132E7002086E700BF7B
:10AF90000000B4420000C8429A99993E9A99193E1D
:10AFA0009A99593F95900020CDCC4C3E0020704797
:10AFB0000020704701207047034BD3F8DC05431E87
:10AFC00058425841704700BF487B002030B587B0D9
:10AFD00002A817F0B7FB3B4886F054FC20B13A4971
:10AFE0003A48FCF737FD1FE0364886F055FCE8B1DB
:10AFF000374C04F12405234604F11002A4F110019A
:10B00000A4F1D000009586F06DFCCDE90045A4F6D2
:10B01000EC2292ED000A2F4904F11003A4F1100272
:10B02000A4F1D00086F020FC07B030BD254802A96D
:10B0300086F070FC08B102A9D2E7274CD4F8503C46
:10B04000002B0CDD94F8F03B4BB1A4F500502049E7
:10B05000FCF700FDA4F50050FCF73EF9E4E71B48BF
:10B0600004F05AF90028BAD11C4C94F874305B07EC
:10B0700020D4D4F88830002BB1D0134AA2F120019B
:10B08000A2F1100017F02CFE0028A8D1144C0F4894
:10B09000D4ED007AB7EE000A04F6F82130EE670A24
:10B0A000FCF708FD094804F6D82204F6F821FCF75D
:10B0B0005BF8B9E7A4F5C040FCF774FD0028B3D1F4
:10B0C000D7E700BFDC8A0020BC8B0020482B002083
:10B0D000AC8B002018580020484B0020488B0020E3
:10B0E000C480002008B50A4890F8D132013B012BFA
:10B0F00003D8A0F50050F8F751F90648F8F714F80E
:10B100000448F8F70BF9BDE808400248F8F76CBCB2
:10B11000484B0020482B002010B5044607480CF08F
:10B12000CFFE50B1064B93F8790230B12368204628
:10B130009B6B984780F00100C0B210BDB88E002014
:10B14000488B0020124B984210B5044601D10020D4
:10B1500010BD03F11C029042F9D003F13802904275
:10B16000F5D003F174029042F1D0D4339842EED07E
:10B1700003681B6A984720B1064B93F86234002B92
:10B18000E5D1206907F0CCF880F00100C0B2DFE71C
:10B1900058770020485B0020174B984210B50446B2
:10B1A0000ED003F11C0290420AD003F13802904203
:10B1B00006D003F17402904202D0D433984206D1F3
:10B1C0000E4B93F98902B0FA80F0400910BD036874
:10B1D0001B6A984718B10A4B93F8623443B9206947
:10B1E00007F09EF830B12069BDE8104009F03EBC80
:10B1F0000020EBE70120E9E758770020484B0020CA
:10B20000485B002073B50F4E0D46114696F9042297
:10B210001AB90124204602B070BD036801915B6930
:10B22000984704460028F4D1D6F8FC33019913F46A
:10B23000802FEED00448054B00682A46C06A24F0EF
:10B2400041FEE7E7488B0020442B0020BCAD0D08F1
:10B25000094A0260094A4260111F816002F1080137
:10B26000C160A2F1380102F59C724261A2F59F42D1
:10B2700001618261704700BF08AE0D08B88C0020E4
:10B2800008B503681B6E98470648D0F8A02F00F653
:10B29000E4439A4205D0BDE80840A0F58040FEF79F
:10B2A0009FBD08BD486B00202DE9F7435C4C04F5B9
:10B2B000AB6300221A60A4F54073C11A4B42A4F597
:10B2C00000594B4189F8F83604F5AD63002584F840
:10B2D0003C55A4F8925584F8965584F8545584F852
:10B2E000C95584F8CA55C4F8BC55C4F8B855C4F853
:10B2F000B455C4F8C4551A60836904F58058D3F86E
:10B30000FC31A4F88C3508F1640306460FCB08F134
:10B31000540787E80F0084F8955584F8A455C8F8B9
:10B3200030508AF011FA44F8580C336830465B69A3
:10B3300098474FF0FF3384F8995589F8645444F8DE
:10B34000283C84F89805306906F07EF988F88D501D
:10B3500084F8975533683046DB6D9847A4F58057DD
:10B360000546002858D0336830469B6B984784F8D0
:10B37000D805D9F884060368DB6B9847A4F5E0503C
:10B380007AF0C0FAA4F5A0400AF01EF8A7F5F7502D
:10B3900067F022FA94F80836CBB1A4F5A040FFF785
:10B3A00009FBA0B908F1F00078F016F978B9D7F8E0
:10B3B000A00F03685B6B984748B95BF0FBFF194A25
:10B3C000062155F06FF904F5C0602EF025FF1648F0
:10B3D000F7F708F8336993F9CC206AB1586801A9E6
:10B3E00012F05EF834699DED010A014604F188000F
:10B3F000FBF73AFC84F84101336830465B699847B3
:10B4000050B1336993F93C22002A02DD93F8A0324F
:10B4100013B9002387F8AD3F284603B0BDE8F08399
:10B42000487B0020C8AD0D08482B002070B503688C
:10B430005B6E0E4615469847044650B995F90030A4
:10B440003BB90548054B00683246C06A294624F0DE
:10B4500039FD204670BD00BF442B0020ECAD0D0827
:10B4600010B50E4C20467AF049F804F5AC7079F02E
:10B47000C1FD04F52C707AF0EFFC094B03F5A042F6
:10B48000002182F8541502F5AB62002103F5005348
:10B490001160012283F8282F10BD00BF245B00201B
:10B4A000482B002008B52DED028B1520B0EE408A08
:10B4B0005EF0D4FCB0EE480ABDEC028B1A20BDE869
:10B4C00008405EF0CBBC000008B5084890F989320E
:10B4D0000121A0F5005033B10AF0FAF9BDE80840A7
:10B4E00046205EF0BBBC0AF01BFAF7E7484B002091
:10B4F00001207047012070470120704701207047EC
:10B5000001207047192070470048704770AE0D0841
:10B510000048704780AE0D0884B038B505AC84E8AB
:10B520000E00054614210C48FCF728FA2A6964230A
:10B53000B2F9C01068B103225943204617F008F948
:10B5400005482146FCF728FEBDE83840012004B03C
:10B5500070470122F0E700BF482B002013B50F49C8
:10B5600001AAA1F1100017F0DBF940B1DFED0C7A70
:10B570009DED017AB4EEE77AF1EE10FA0CD8094CA1
:10B58000D4F8840603689B6B984728B106492E229D
:10B59000A4F540500BF09CFD02B010BDBC8B002008
:10B5A000000000B4485B00205C79002030B51D4CE1
:10B5B0000546D4F8A40F036887B05B69984738B193
:10B5C00019491A482F220BF083FD012007B030BD26
:10B5D000174806F0A5FE0028F2D1A4F58054D4F84F
:10B5E000840603689B6B984728B1D4F884060368E7
:10B5F0001B6C984798B10F4B0FCB02AC84E80F003F
:10B60000284601F06DF82868059B009394E80E0029
:10B61000446C2846A0472846FFF7A0FFD5E7064B15
:10B62000EAE700BF486B00205C790020482B00202F
:10B63000808C0020AC8B0020BC8B002010B5044611
:10B64000FFF78CFF2046BDE8104001F085B80000F0
:10B65000042070470048704775B40D0800487047D3
:10B6600075B40D08037F73B1D0ED087AFDEEE77A6B
:10B6700017EE903A084AC2F8F035437F3BB1436A6F
:10B68000C2F8F43570478369D3F8F831F2E783697B
:10B69000D3F8FC31F4E700BF487B002008B5002355
:10B6A000838300F12801806911F010FF012008BD9B
:10B6B00070B56E4E2DED048B06F59F4304460121B7
:10B6C000304693ED1C9ADFED6A9A09F02BFF0121B9
:10B6D000B0EE408A304609F02FFFC8EE297A06F511
:10B6E0000055A069B5F9AC3204F1280108EE903A92
:10B6F000F8EEE88AB5F9AE3268EEA78AC0EE297A8C
:10B7000008EE103AB8EEC88A28EE278A11F0DEFE5D
:10B7100095F9B23263B39FED577AF0EEE87AF4EE22
:10B72000C77AF1EE10FA23D5227FA369002A55D1FA
:10B73000012222770022226294ED087ADFED4E7A10
:10B74000D3F8F8314D4A4E4867EEC77A9FED4D7AEF
:10B7500067EE877AB0EE490AFDEEE77A17EE901AA7
:10B760000B44C2F8F0350023012279F057FE08E0BF
:10B77000002343482377F0EE490AB0EE680A79F0D7
:10B7800049FE04205EF06AFB95F9B23243B19FEDA9
:10B79000397AF0EEC87AF4EEC77AF1EE10FA28D4CE
:10B7A000002339486377F0EE490AB0EE480A79F091
:10B7B0008BFA13205EF052FBB5F9B032002B03DD9B
:10B7C000324E96F9A23263BB28482021F7F742F99E
:10B7D000002843D1254809F0C7FC42E0D3EDC56AF3
:10B7E00096ED467AD4ED087AE6EE877AC4ED087ACB
:10B7F000A2E7637F2BB901236377A369D3F8FC31F8
:10B8000063621E4B616AC3F8F415A369D3F8FC01A7
:10B810000023091A1A461C48B0EE490A79F03AFB8F
:10B82000C7E70121A6F5405009F090FE80EE297A85
:10B83000B5F9B032002106F5237007EE903AF8EE24
:10B84000E77AF0EE490A27EE870A7AF005FABDECAE
:10B85000048B2046BDE87040FFF724BE0348F7F78D
:10B860002FFF07EE900AB8EEE70AF0E7482B00201A
:10B8700000A08C4500000034E02E6542487B00208B
:10B88000245B00200000C8427C5C0020485B002054
:10B890002DE9F04F2DED0C8BDFF8A8A39FEDDEDA3C
:10B8A0009FEDDE9A97B00AF59F4300F12805044604
:10B8B0000121504693ED1CBA09F034FE0121504697
:10B8C000F0EE408A09F038FE01215046B0EE408A81
:10B8D00009F03CFEDFEDD27A88EEA77A0AF5005631
:10B8E00001A8B6F9AC320AF5A04B0AEE903AF8EE90
:10B8F000EAAAB6F9AE32DFEDCB8A6AEE87AA88EE05
:10B90000277A0AEE103AB8EECAAAB6F9B0329FED1D
:10B91000C68A2AEE07AA80EE277A09EE903AF8EE58
:10B92000E99A6AEE8D7A69EE879AF0EEEACAF4EE49
:10B93000C8CACDED017AB0EECACA6AEE0D7AF1EE50
:10B9400010FAF0EEE9BAB4EEC8CACDED027A58BFEB
:10B950004FF0010969EE8D7A48BF4FF00009F1EE12
:10B9600010FAF4EEC8BA9AED460ACDED037A54BF48
:10B970004FF001084FF00008F1EE10FA54BF012714
:10B9800000272BF0D5FA01A928462AF07BFD28468E
:10B990002AF072FE28462AF0E1FD20EE090A284628
:10B9A00020EE280ABDEEC00A10EE103ACBF8F035B2
:10B9B0002AF0EEFD20EE090A20EE280ADFED9B8A30
:10B9C000BDEEC00ACDED0D8A10EE103ACBF8F4357D
:10B9D0000DF1280B4FF07E535946A0690A93CDED27
:10B9E0000C8ACDED0B8A11F071FD0021504609F053
:10B9F0006FFFB0EEC00AB4EEC80AF1EE10FA16D529
:10BA00005046FEF7D7FF90B9F4EEC8CAF1EE10FA2F
:10BA10000DD5B4EEC8CAF1EE10FA08D5F4EEC8BAE6
:10BA2000F1EE10FA44BF9BE80F0085E80F000AA86A
:10BA30002AF086FE294612A88DED141A8DED120A01
:10BA4000CDED130ACDED151A2AF08CFE0DF1100A7A
:10BA500051460EA88DED101ACDED048ACDED058A64
:10BA6000CDED068A8DED0E0ACDED0F0ACDED111A42
:10BA70002AF042FCB6F9AC32DFED6D7A01EE103AF5
:10BA8000B6F9AE3209EE103AB6F9B03208EE903A95
:10BA9000B8EEC11AB8EEC99AF8EEE88A21EE271A74
:10BAA00029EE279A68EEA78AF4EEC8CAF1EE10FADA
:10BAB00021EE0D1A29EE0D9A68EE8D8A07D594F8BD
:10BAC0003830DFED5A7A002B18BFB0EE671AB4EEAB
:10BAD000C8CAF1EE10FA07D594F83930DFED537A81
:10BAE000002B18BFB0EE679AF4EEC8BAF1EE10FA68
:10BAF00007D594F83A30DFED4D7A002B18BFF0EE01
:10BB0000678A9AE807000DF11C0B8BE80700F1EE3D
:10BB1000410AC2209DED070A28F0B2F8C3208DED3E
:10BB2000070AB0EE491AF1EE490A9DED080A28F01D
:10BB3000A7F8B0EE681AF1EE680A8DED080AC42085
:10BB40009DED090A28F09CF8514658468DED090AEA
:10BB50002BF084F912A928468DED120ACDED130AB7
:10BB60008DED141A06F57E662AF08CFC28462AF024
:10BB700083FDDDED076A96ED007A2E4B9FED270AD7
:10BB8000C6EE877A5846DDED086ACDED077AD3ED2B
:10BB90004E7A86EEA77ADDED096A8DED087A86EE9B
:10BBA000A77A8DED097A2BF0C3F9B9F1000F01D016
:10BBB000CDED07AAB8F1000F01D08DED08AA0FB1A5
:10BBC000CDED099AF0EE4B0A9DED070A1A4879F07F
:10BBD00021FC04205EF042F9F0EE4B0A9DED080ACC
:10BBE000164879F071F813205EF038F90021F0EE74
:10BBF0004B0A9DED090A12487AF02EF82046FFF70D
:10BC000051FC84F8389084F8398084F83A7017B081
:10BC1000BDEC0C8BBDE8F08F35FA8E3CE02E654212
:10BC200000A08C450000C842000000340000000065
:10BC3000CDCC4C3E485B0020245B00207C5C002087
:10BC4000D45D0020482B002010B50446FFF73CFCD3
:10BC50000B4B93F9B222022A0DD1B3F9B022002A7C
:10BC600009DD03F5805393F9A23223B12046BDE8E4
:10BC70001040FFF70DBE2046BDE81040FFF718BD8D
:10BC8000484B00200A207047004870473ED40D08FA
:10BC9000004870473ED40D080120704701207047CE
:10BCA0000120704701207047034BD3F8DC05031FC8
:10BCB00058425841704700BF487B002070B5054688
:10BCC0002D48D0F8A42F00F664539A4215D12B6961
:10BCD00093F844318BB100F5B0502DF067FE044667
:10BCE00058B95BF067FB254A032154F0DBFC2B6954
:10BCF000012283F84321204670BD214C94F84C3238
:10BD000023B194F904329A1E534253411D4E86F8D2
:10BD1000983504F164030FCB04F15405743485E8BD
:10BD20000F0084E80F0006F5C0602EF0B5FC164B3E
:10BD30001C68E56A2B6828465B689847B0B195F89F
:10BD40004D309BB1E36A9B8F83B15BF033FBE36AB9
:10BD50000E4A9B8F062154F0A5FCE36A06F5C060ED
:10BD6000998F2EF085FAE36A00229A87084886F0B8
:10BD70000BFD0124BFE700BF486B002068AF0D0832
:10BD8000488B0020487B0020442B002082AF0D0808
:10BD9000B055002038B50D4C94F80436012B10D165
:10BDA00004F5C0602BF05EFDB4F83E560848294605
:10BDB00005F0AEFC28B9152D03D104F6947085F07A
:10BDC00041FE0023C4F8843538BD00BF487B002005
:10BDD000808C002008B511F093FD90F87C32DB07D1
:10BDE00004D5BDE8084002482EF0F2BA08BD00BFF5
:10BDF0004881002038B5344C94F80436012B0ED01D
:10BE0000A4F535710822A4F5A0400BF061F95BF0B0
:10BE1000D1FABDE838402D4A062154F043BC2C48E5
:10BE2000B4F83E5605F098FC20B1BDE838402848EB
:10BE300008F0C6BD162D05D0152D36D1D4F8DC3549
:10BE4000072B0AD123480CF05BFF22480DF0A4F821
:10BE5000BDE838401F480CF0B5BFA4F5A040F7F787
:10BE600053FFA4F5A040F7F72FFEA4F54053D4F8F4
:10BE7000F01593F9F02264235A4304F6947085F088
:10BE80003DFDC4F8F00504F6947085F079FE30B1FC
:10BE9000BDE838409FED100A46205DF0DFBFA4F5F5
:10BEA000A040BDE83840F7F7F3BB1E2D18BF4FF098
:10BEB000FF33084818BFC4F85035F7F725FF054889
:10BEC000F7F702FE0348ECE7487B00209CAF0D0823
:10BED000808C0020482B00200000000070B5144822
:10BEE00090F904320E46154613B90124204670BD60
:10BEF000D0F8FC335B0312D5A0F5805300F59C709D
:10BF0000B3F83E1604F0ACFE044640B9094B0A48AB
:10BF1000006832462946C06A23F0D4FFE6E70748A6
:10BF20002DF044FD04460028DFD1054BEFE700BFAC
:10BF3000488B0020C8AF0D08442B0020488100200A
:10BF4000DCAF0D0810B5144BB3F83E36532B044646
:10BF50001ED10AF0C7F89FED110A46205DF07EFF62
:10BF60009FED0E0A49205DF079FF9FED0C0A4A20F3
:10BF70005DF074FF46205EF051F849205EF04EF807
:10BF80004A205EF04BF82046BDE81040FFF768BA43
:10BF9000BDE81040FFF7A6B8487B00200000000075
:10BFA000082070470048704768B00D080048704787
:10BFB00074B00D080120704708B50248FDF7B0FEC7
:10BFC000012008BD482B0020014800F05FB900BFE8
:10BFD000CC77002010B50446FFF784F82046BDE872
:10BFE0001040FFF771BA0000012070470048704709
:10BFF000ECB00D0800487047F4B00D080120704700
:10C000000120704710B5044B03F1740464330FCB67
:10C0100084E80F00012010BD488B002008B50B48B4
:10C0200000F5A04200F500530321D3F8C03C93FB78
:10C03000F1F3C2F8F035F7F7ABFD0448F7F744FD2C
:10C04000BDE808400148F7F723BB00BF482B00209C
:10C050000720704700487047B0920D0800487047AD
:10C060006CB10D0801207047012070470120704716
:10C070007047000008B5002303774362034886F049
:10C0800083FB0348FBF7A6FC012008BDB055002048
:10C09000482B002010B5194CD4F8A83CB3F908304F
:10C0A00023B9D4F8B43CB3F90830F3B100230377D3
:10C0B0004362D4F8A80C5CF019FD04F54C63D3ED91
:10C0C000007A0F48F8EEE77A27EE800ABDEEC00A44
:10C0D00010EE103AC0F8F035A0F5A040F7F758FD83
:10C0E000BDE81040074803F015B8037F002BE0D0EF
:10C0F000A4F50050F7F708FEF2E700BF484B002018
:10C10000487B0020482B002070B54E4DDFED4E7A65
:10C1100095F8E4339FED4D7A2DED048BB02606FBA8
:10C12000035393ED788A9FED4A9A28EE278A05F506
:10C13000A953BDEEC88A93ED050AF8EEC87A044605
:10C1400067EE897A97EE870A27F086FD237FF0EE67
:10C15000408A002B62D105F50053D3F8A83CB3F90F
:10C160000830002B5AD1284608F0FEFF002855D190
:10C1700095F8E43395F8281406FB035393F8C1218E
:10C1800000294BD1012A49D993ED777AF0EE087A4C
:10C19000B4EEE77AF1EE10FA40DBDFED2E7AB0EE86
:10C1A000E80AB4EEE70AF1EE10FA37D5636A93B302
:10C1B00089F0CAFA636AC01AB0F5FA7F32D8237FD1
:10C1C000002B3CD0244DA5F1200696E80F0085E811
:10C1D0000F0094ED088AA5F110013046B8EEC88A28
:10C1E00016F012FE28EE098ADFED1C0A284670EED2
:10C1F000200AB0EE480A16F0ADFE194B9FED190A61
:10C20000D3F88406BDEC048B03682A4631469B6A4A
:10C21000BDE87040184789F097FA6062636A002BA6
:10C22000CDD0C5E7104D84ED088A01232377002384
:10C23000636205F110030FCB85E80F00BFE7BDEC8B
:10C24000048B70BD482B00200000C84235FA8E3C9C
:10C250000AD7233CDB0FC93FBC8B002000007A4487
:10C26000485B0020000000009C8B0020036A0B60EC
:10C27000007F70470520704700487047E4B10D0803
:10C2800000487047F4B10D080120704738B54B4D98
:10C290002DED028BD5F8A80C9FED498A5CF026FCA9
:10C2A000D5F8C03C07EE903AF8EEE77A05F5405431
:10C2B00027EE800AA5F50050BDEEC00A10EE103A38
:10C2C000C4F8F035F7F764FCD5F8AC0C5CF00EFC64
:10C2D000B5EEC00AF1EE10FADABF05F6C443D3EDAD
:10C2E000007AD5ED907A3748CBBF20EE270A20EEB2
:10C2F000270A20EE080A28EE400ABDEEC00A10EE1A
:10C30000103AC4F8F435F7F70FFC95ED907AD4F8AD
:10C31000F40505F6C44327EE087AD3ED007A27EE3C
:10C32000888AFDEEC77A17EE902AFDEEC87A17EEDE
:10C33000901A27F045FDC4F8F4052248FDF77CFD6E
:10C3400020B1D4F8F4355B42C4F8F4351E4B93F8B1
:10C35000B43F63B195F99432022B08D10023012137
:10C360004620C4F8F035C4F8F4355EF0DBF85CF034
:10C37000CDFA5F215DF024FAE8B15DF0F1F9022811
:10C3800019D194F89535B3B904F5AD6393ED007AFE
:10C39000D5EDB87AB4EEE77AF1EE10FA0BD50123B9
:10C3A00084F89535BDEC028B084A0948BDE8384051
:10C3B000042154F077B9BDEC028B38BD484B002006
:10C3C0000000C842482B0020486B0020FCB10D083B
:10C3D000B05F002010B50446FEF784FE2046BDE89D
:10C3E0001040FFF771B80000062070470048704702
:10C3F0007CB20D08004870478CB20D0801207047D0
:10C4000001207047012070470120704770470000ED
:10C4100008B5044886F0B8F90348FBF7DBFA0120B9
:10C4200008BD00BFB0550020482B002038B50F4C88
:10C4300004F50055D5F8A80C5CF058FB04F5335210
:10C44000D2ED007AF8EEE77A04F5A04327EE800AF1
:10C450002046BDEEC00A10EE102AC3F8F025F7F70B
:10C4600097FB2046BDE8384002F054BE482B002020
:10C470000F2070470048704704B30D08004870470C
:10C480000CB30D0801207047012070470120704750
:10C4900001207047012070470120704730B5184BCC
:10C4A0002DED028B002283F8622403F541532433DF
:10C4B00005460FCB85B06C4684E80F00114804F0A8
:10C4C0008DFB90B1A86900F57F702AF061FB0D48E3
:10C4D000B0EE408A04F0EAFBF0EE400A9FED0A0A53
:10C4E000204628EE000A16F035FD00230748EB61D0
:10C4F0002146FBF751FE012005B0BDEC028B30BD9B
:10C50000485B0020808C0020E02E6542482B0020F4
:10C5100038B5424C94F899354BB104F5805393F8F3
:10C520004C3223B1BDE838403D4808F01BBAD4F87E
:10C53000B435002B18DC3B48F7F7E6FBD4F8B835E8
:10C54000002B29DC3748F7F7BFFA374890F86234F8
:10C55000002B46D00121A0F5405009F0B9F9BDE803
:10C56000384046205DF07ABC89F0EEF8D4F8B43556
:10C57000C01A40F6B7339842DDD82C4DD4F8A80540
:10C58000D5F8C02C514227F01BFCC4F8F005A5F5E6
:10C590000050F7F7FDFAD1E789F0D6F8D4F8B835AE
:10C5A000C01A40F6B7339842CCD8204BDFED206A52
:10C5B00093ED907AD4F8AC0503F6C443D3ED007A3A
:10C5C00027EE267A67EEA67ABDEEC77AFDEEE77A09
:10C5D00017EE102A17EE901A27F0F2FBC4F8F405B4
:10C5E000B3E7A0F5805090F91F32012B04DCBDE8C1
:10C5F00038400C48F7F74CB8D4F8C435002BF6D0C7
:10C6000089F0A2F8D4F8C435C01A40F6B73398427E
:10C61000EDD804F5B86494ED000AA0E7487B00204B
:10C62000808C0020482B0020485B0020484B0020D5
:10C630000000C842D0ED077A0348FCEEE77A17EE17
:10C64000903A99B202F058BF482B002084B010B540
:10C6500003AC84E80E000B4821466F22FBF7E8FC90
:10C660009DF80C1011F0040102D1204616F034F9A7
:10C6700004482146FBF790FDBDE81040012004B0BE
:10C68000704700BF482B0020B0EEC00AFDEEC07A14
:10C6900038B54FF6FF7205460C4617EE900A00219A
:10C6A00027F08EFB07EE900A002CF8EEE77A054B98
:10C6B000C5ED077A14BF4FF0FF32012283F82C201A
:10C6C00038BD00BF488B0020FEF780BC0C207047AF
:10C6D00000487047E5B50D0800487047D2EC0E08D9
:10C6E00008B50C48FCF78AFA0A480B49FBF7A0F991
:10C6F0000848F6F739FC40B106484FF48051F6F788
:10C70000A9F910B10348FBF765F9024802F0DEF918
:10C71000012008BD482B0020BC8B002008B50D4827
:10C72000F7F7F2FA0B48F6F71FFC50B109484FF43F
:10C730008051F6F78FF920B1BDE80840054802F0B6
:10C74000E9BC0448F7F7C0F9BDE808400148F6F72E
:10C750009FBF00BF482B002008B509484FF4805107
:10C76000F6F778F930B107480022D0F88410743019
:10C7700015F0EEFFBDE808400148002102F0BCBE04
:10C78000482B0020488B0020881A10B527F040FA6B
:10C790000F4B9A6A0028B8BF4042002AB8BF5242E5
:10C7A00048F6A041B2FBF1F24FF47A7102FB01119D
:10C7B00088420BDC93F87420D20605D503F174048B
:10C7C00064330FCB84E80F00012000E0002010BD8F
:10C7D000488B002013B504468069019100F57F70F5
:10C7E0002AF0D6F9DFED0A7A20EE270A27F0B2F90F
:10C7F000DFED087A019920EE270A2046FDEEC07A87
:10C8000017EE902A02B0BDE81040FFF7BDBF00BF91
:10C81000E02E65420000C84284B070B52DED048B57
:10C8200086B00FAD85E80E004D4CDFED4E8A064612
:10C83000D4F8840604F5405494ED100A0368B0EE71
:10C84000C00A5B6A9847B4EEE80AF1EE10FAB0EE5F
:10C85000408A07DA012006B0BDEC048BBDE87040C9
:10C8600004B070474049284616F0DAF902A8CDED29
:10C87000030A8DED020A2AF05BFA04A88DED040A82
:10C88000B0EE480ACDED050A2AF00EF913A92846A4
:10C890008DED000ACDED010A16F0C2F902A88DED6A
:10C8A000020ACDED030A2AF0BDF9B4EEE80AF1EE72
:10C8B00010FACFDBB4EEC08AF1EE10FA9FED2B9A9E
:10C8C000DFED2B8ADFED2B9A2BD802A869462AF0E0
:10C8D000DBF804A88DED040ACDED050A2AF058F91D
:10C8E000684620EE098A2AF053F994F92C3007EEB5
:10C8F000903AF8EEE77A28EE288AA7EEA90A27F000
:10C90000ABF920EE090ABDEEC88A20EE280A18EE1F
:10C91000101AFDEEC07A304617EE902AFFF734FF6A
:10C9200099E738EE400A38EE088A80EE080AB1F03E
:10C930002BFD02A8B0EE408A2AF02AF994F92C3097
:10C94000F0EE007AB0EE697AA8EE677A07EE903AD8
:10C95000F8EEE77AA7EE270A27F07EF9C0E700BFD6
:10C96000485B002000000034AC8B0020E02E6542C4
:10C970000000C842DB0FC93F10B504460848F6F76F
:10C98000F3FA20B92046BDE81040FEF71FBB04486B
:10C990004FF48051F6F75EF80028F3D010BD00BFC9
:10C9A000482B00200020704700487047F4B30D0862
:10C9B00000487047FCB30D0800207047036993F8E6
:10C9C000140118B1D3F8C402C0F3801070470000FE
:10C9D00038B5154C05460021204608F0A3FD04207B
:10C9E0005DF03CFA0021204608F0A6FD13205DF022
:10C9F00035FA0021204608F0A9FD2846FEF752FD31
:10CA00002046012108F064FF46205DF027FAAB695B
:10CA100004F5A044D3F8F831C4F8F035AB69D3F885
:10CA2000FC31C4F8F43538BD482B0020FEF718BDA2
:10CA3000172070470048704774B40D0800487047CD
:10CA40007CB40D0801207047012070470120704719
:10CA500010B50369002283F8402103690446D3F826
:10CA60003C0103689B689847A36818687FF050FAF8
:10CA7000206904F02BFE0349A06910F027FD012076
:10CA800010BD00BFB87700201FB50D4C9FED0D0AFB
:10CA900004F5C04304F5A044D3F86C016C302AF0CF
:10CAA000F3F9FDEEE00ABDEEC00A10EE903AC4F8CC
:10CAB000F43510EE103AC4F8F03504B010BD00BFE4
:10CAC000482B00209F0CB34530B52DED028B83B071
:10CAD000044688F039FE0146206900F50E700BF01F
:10CAE00039F938B1204603B0BDEC028BBDE83040C7
:10CAF000FEF7F8BA206990F84031BBB1012104F08B
:10CB00006BFDA368DFED400A1868036801215B6EC6
:10CB1000B0EE600A9847206903F0BEF93B4803B0C5
:10CB2000BDEC028BBDE83040FFF78EB8384DDFED2D
:10CB3000398A022104F050FDD5F8AC0C5BF0D6FF29
:10CB40002369D3ED390A93F93C2220EE200A002A0A
:10CB500060EE280A3FDD93F8A032002B3BD0D5F8D9
:10CB6000B40CCDED000A5BF0C1FF2369D5F8A80C29
:10CB700093ED3A8A20EE080A20EE288A5BF0B6FF91
:10CB8000236993ED381A20EE410A20EE281ADDEDD4
:10CB9000000A2069CDED010A8DED001A03F0B8F905
:10CBA000A36895F9B22218689DED001ADDED010A1F
:10CBB0000368F0EE408A2AB31B6CB0EE480A98472F
:10CBC000A36818680368F2EE040A5B6E0021B0EEF9
:10CBD000680A9847A2E7D5F8A80CCDED000A5BF0EB
:10CBE00085FF2369D5F8B40C93ED388A20EE080A46
:10CBF00020EE288A5BF07AFF236993ED3A1A20EE43
:10CC0000010AC2E7DB6BD8E7000000009077002044
:10CC1000484B00200000C84212207047004870476F
:10CC2000F4B40D0800487047FCB40D0801207047AB
:10CC3000012070470120704738B52DED028B436805
:10CC40009FED1C8A1D680446006904F065F923699C
:10CC500093ED131AD3ED110A434200EE103A21EE80
:10CC6000081A60EE880AB8EEC00A284680F00AFB6F
:10CC7000636820691D6804F04FF9236993ED131A66
:10CC8000D3ED110A434200EE103A21EE081A60EE8D
:10CC9000880AB8EEC00A284680F06EFB9FED060AAF
:10CCA000206903F025F9206905F0CAFEBDEC028B6E
:10CCB000012038BD0000C84200000000014800F01B
:10CCC00071BE00BF0479002013B5044600698830A6
:10CCD000FAF72AF988F038FD0146206900F50E7050
:10CCE0000BF038F828B1204602B0BDE81040FEF73E
:10CCF000F9B9206990F840313BB3012104F06CFC94
:10CD0000A368DFED170A18680368B0EE600A5B6E6F
:10CD100001219847206903F0BFF863689FED100A6E
:10CD2000186881F0D9FC0F48F6F7FEF90D48F6F7C0
:10CD3000F5FA20469FED0A0AFEF7B4FB2069883019
:10CD400002B0BDE81040FAF7AFB9074804F0A8FDFB
:10CD50002069019004F046F9019806F07DFAE2E7B7
:10CD600000000000482B0020808C00201420704719
:10CD7000004870477AAE0D0800487047E5EC0E0891
:10CD8000012070470020704770B504460E4800F03F
:10CD90003BF82369002583F84051206904F05EFFC9
:10CDA0006069052103F01AFD084826690221FAF797
:10CDB000B7FC86EDB70A2369C3F848512369C3F865
:10CDC0004C51012070BD00BF3C790020482B002051
:10CDD000014800F0E7BD00BF04790020014800F0E1
:10CDE00069B800BF3C7900201320704700487047A5
:10CDF000E4B50D0800487047ECB50D0801207047F8
:10CE0000012070470120704738B52DED028BDFED12
:10CE1000240AC3689FED238A0446B0EE600A1868AE
:10CE20007CF0F8FBE36818687CF0D2FC636820694A
:10CE30001D6804F071F8236993ED131AD3ED110AFC
:10CE4000434200EE103A21EE081A60EE880AB8EE6E
:10CE5000C00A284680F016FA636820691D6804F04D
:10CE60005BF8236993ED131AD3ED110A434200EEE8
:10CE7000103A21EE081A60EE880AB8EEC00A284679
:10CE800080F07AFA206905F0DBFD256988F05CFC0A
:10CE9000C5F86C01BDEC028B00230120E36138BDB5
:10CEA000000000000000C842014800F07BBD00BF48
:10CEB0000479002030B52DED048B0446006985B05F
:10CEC0008830FAF731F838B1B64805B0BDEC048BBC
:10CED000BDE83040FFF7F8BE88F036FC0546206913
:10CEE000294600F50E700AF035FF38B1204605B02E
:10CEF000BDEC048BBDE83040FEF7F4B8206990F833
:10CF0000403163B3012104F067FBA368DFEDA60A9B
:10CF1000186803680121B0EE600A5B6E98472069CB
:10CF200002F0BAFF63689FEDA00A186881F0D4FB95
:10CF3000DFED9D0AE368B0EE600A18687CF06AFBDA
:10CF4000E36818687CF044FC9848F6F7EDF89748D9
:10CF500005B0BDEC048BBDE83040F6F7DFB9C36A1D
:10CF600093F8CB3013B99248FFF74EFF206903F0D6
:10CF7000F9F818B1E36818687CF048FB2369D3F826
:10CF80006C31EB1AB3F5FA7F0BD9E368DFED860A53
:10CF90001868B0EE600A7CF03DFBE36818687CF02E
:10CFA00017FC23699FED838AC3F86C510221206925
:10CFB00004F012FB636820691D6803F0ADFF23696C
:10CFC00093ED131AD3ED110A434200EE103A21EE0D
:10CFD000081A60EE880A2846B8EEC00A80F052F9B6
:10CFE000D4E9033518687CF07FFBA36818680368F0
:10CFF0009B6EF0EE408A984703AAF0EE400A02A921
:10D00000B0EE680A284602F0C7FFE368DDED030AC8
:10D0100018689DED020A7CF0FDFA6368186880F0DC
:10D0200023F918B96368186881F014F8E368624D51
:10D03000186801217CF038FDE36860481B689B6834
:10D04000D3EDCF7AFDEEE77A17EE903AC5F8F035DA
:10D05000E3681B689B68D3EDD07AFDEEE77A17EEA4
:10D06000903AC5F8F43504F01BFC2369D3F83C0171
:10D07000036805F2F4525B6B05F5BE61984748B151
:10D0800063681B68D3F88823C3F89423D3F88C23F0
:10D09000C3F898232069DFED4A9A04F011FBD5F814
:10D0A000F035206907EE903A012105F2F453F8EECD
:10D0B000E78A93ED009A06F069F8A368B8EEC99A7A
:10D0C000186820EE290A036868EEA98A29EE299AD1
:10D0D000DB6A20EE081A69EE080A28EE880A9847EB
:10D0E000384BD3F8A02F03F614618A4248D1636904
:10D0F00093F86430062B0AD8206903F081FC30B124
:10D100006069072103F06AFB206904F0A7FD274846
:10D110000221FAF705FB206903F050F8636993F8E0
:10D120006430072BB0EE408A08D12369D3F8C432AB
:10D130009B0403D4A069012110F08EFE6368B5EE54
:10D14000C08AF1EE10FA1868CCBF01210021B1EEBF
:10D15000480A80F01DF9206907F092FD206903F06C
:10D16000F9FE1248F5F7E0FF1048F6F7D7F89FED03
:10D170000E0A2046FEF796F905B0BDEC048B30BDD3
:10D1800003F664539A42206907D190F8423123B1E3
:10D190009FED050A02F0ACFEE0E7019003F022FFEC
:10D1A0000198F7E72079002000000000482B0020BC
:10D1B0003C7900200000C842487B0020808C002081
:10D1C0000AD7233C486B0020152070470048704761
:10D1D00064B60D080048704764B60D08012070471A
:10D1E0000120704700207047C369012B06D1044B12
:10D1F00093F80C03431E5842584170470020704773
:10D20000488B00200E4BB3F95222B3F9843207EE5B
:10D21000102A07EE903AB8EEC77AF8EEE77AB0EE49
:10D22000C77AF0EEE77AB4EE677AF1EE10FAC8BF8B
:10D23000F0EE477AB7EE080A27EE800A704700BF83
:10D24000484B00202DE9F043844D2DED048B95F8DB
:10D250007C928BB00446B9F1000F0BD0804931228B
:10D26000A5F5C04009F034FF01200BB0BDEC048BE4
:10D27000BDE8F0830123C36105F1640696E80F0061
:10D2800005F1540787E80F0023692A6DB3F8C070D1
:10D29000DB6A526893F8A0306421022B17FB012748
:10D2A00040F0B68007EE907A3246B8EEE70AA5F570
:10D2B000C04106A8FBF788F806A9304615F0A4FD82
:10D2C0002046F0EE408AFFF79DFF2369B3F9C020A6
:10D2D000D3ED310A01EE102AB3F9C220B0EE409A24
:10D2E00000EE102AB8EEC11A1A20B8EEC00A26F0D5
:10D2F000C7FC2369B3F9C030F4EEC98A07EE903A4F
:10D30000F1EE10FA54BFF0EE686AF0EE496AB8EE3A
:10D31000E77AC8EEA67A236820465B68B0EE408ABA
:10D3200067EE877AB4EE670AF1EE10FA48BFB0EE06
:10D33000678A98470146A5F5C040FAF71FFB082108
:10D3400002468046A5F5C040FAF79CF9DFED457A24
:10D3500038EE408AB4EEE78AF1EE10FA31DBC4F819
:10D360001C9096E80F0005F1740484E80F009FED0F
:10D370003E9AB8F1000F14D005AA0321304615F0EB
:10D380001DFA70B1DDED057AF8EEE77A0322E8EEDA
:10D39000097A2046FDEEE77A17EE901A15F0D8F9D3
:10D3A00062E7D5ED1A8A3148F8EEE88A15F0FAF905
:10D3B000E8EE098A02462E48FDEEE87A17EE901A4A
:10D3C000ECE7F4EEC98AF1EE10FA21D505AA494638
:10D3D000304615F0F3F918B1059B9F42A8BF1F46D0
:10D3E00059F0E8FF064619EE100AF3F78DF8CDE97B
:10D3F000020118EE900AF3F787F81E4ACDE9000102
:10D400000621304653F04EF96069032103F0E6F936
:10D4100039461948FAF78EFF206903F067FC134874
:10D4200005AA002115F0CAF968B96269AB6EA96F47
:10D430008B4292F82010D4BF0023012363F3000134
:10D4400082F8201010E70A4806AA002115F0B6F964
:10D450000028EAD0DDE905316269E9E7488B002060
:10D460005C790020000000340000C842AC8B002032
:10D47000BC8B00206CB60D08482B0020014800F042
:10D4800091BA00BF04790020F0B52DED028B99B060
:10D49000044688F059F90146206900F50E700AF03B
:10D4A00059FC054638B1204619B0BDEC028BBDE8E9
:10D4B000F040FDF717BEE36983B1012B00F01E8138
:10D4C0009F48F5F731FE9E48F5F728FF9C4819B0B4
:10D4D000BDEC028BBDE8F040F6F786BA9FED998A65
:10D4E00060688DED098A8DED0A8A8DED0B8A8DEDD0
:10D4F0000C8A0BAA09A901230068934D7FF0D8FD7F
:10D500002069B0EE480A03F0B3F863688F481B68DF
:10D51000D3EDCF7AFDEEE77A17EE903AC5F8F03505
:10D5200063681B68D3EDD07AFDEEE77A17EE903A88
:10D53000C5F8F43504F0B4F92369D3F83C01036865
:10D5400005F2F4525B6B05F5BE61984748B163681C
:10D550001B68D3F88823C3F89423D3F88C23C3F82B
:10D560009823206904F0B2F8A36820691E68336824
:10D57000DF6AD5F8F03507EE903A05F2F453D3EDB3
:10D58000000AF8EEE00AF8EEE78ACDED050A05F0AC
:10D5900071F8DDED050AB0EE401A3046B0EE680ACB
:10D5A000B8472069C36B93ED070A02F0A1FC20691C
:10D5B00003F0D0FC63688DED0D8A8DED0E8A8DED44
:10D5C0000F8A18680FA980F0C5F80D9B14930E9B65
:10D5D000159302220F9B169314A910A815F08AFC2C
:10D5E0005B4907AA10A815F09BF948B1DFED597AFD
:10D5F0009DED077AB4EEE77AF1EE10FAFFF660AF30
:10D60000554D0123E36105F1640797E80F0005F12B
:10D61000540686E80F002B6D22695B68B2F8C06083
:10D62000642216FB023607EE906A3A46B8EEE70A25
:10D63000A5F5C04114A8FAF7C7FE384614A915F09D
:10D64000E3FB2046B0EE408AFFF7DCFDB4EEC08A73
:10D65000F1EE10FAF0EE408A22D508AA002105F179
:10D66000740015F0ABF818B1089B9E42A8BF1E4687
:10D6700059F0A0FE074618EE900AF2F745FFCDE9F3
:10D68000020118EE100AF2F73FFF344ACDE900011B
:10D690000621384653F006F86069032103F09EF82E
:10D6A00031462748FAF746FE206903F01FFB284958
:10D6B00007AAA1F1100015F033F9636988B19DED57
:10D6C000077ADFED247A93F82020B4EEE77AF1EEC2
:10D6D00010FAACBF0121002161F3000283F8202081
:10D6E000EEE6AA6EA96F8A4293F82010D4BF0022FA
:10D6F000012262F3000183F82010E1E6206906F0C0
:10D7000015F8636993F86430042B06D91248036D49
:10D710002A465968743015F01BF8636993F8643031
:10D72000032B02D9206907F0EBFA236993F8D4316F
:10D73000013B012B3FF6C4AE0148F5F72FFEBFE6D3
:10D74000482B002000000000487B0020808C002037
:10D75000BC8B002000000034488B00206CB60D0804
:10D7600030B5C369012B85B004D1404C94F80C331B
:10D77000012B04D005B0BDE83040FDF727BCA4F56F
:10D780008043DFED3B6AB3F952229FED3A0A07EE80
:10D79000102AB3F9842207EE902AB8EEC77AF8EE81
:10D7A000E77AB4F9F821B0EEC77AF0EEE77AB4EE92
:10D7B000677A00EE902AF1EE10FAC8BFF0EE477AD1
:10D7C000B8EEE07AD3EDB00A03F6885270EEC70ADD
:10D7D00092ED007A27EE267AF5EEC00AF7EE006A9F
:10D7E000F1EE10FAB4EEE67A48BFDFED220AF1EE70
:10D7F00010FAD8BFB0EE667AF3EE046A77EEA71A95
:10D8000067EEA67AC0EE876A74346D4693ED8B7A24
:10D81000194BB0EE612AA6EE872A93ED001AF4EEBA
:10D82000427AF1EE10FA48BFB0EE672AF4EE421ADF
:10D83000F1EE10FAC8BFB0EE612A26F053F994E871
:10D840000F0007EE901A9FED0D7AF8EEE77A85E863
:10D850000F00E0EE077A0A482946FDEEE77ACDEDA3
:10D86000017AFAF7F7F805B030BD00BF488B002009
:10D870009A99193F00000000C08000200000C842B3
:10D88000482B00201120704700487047FCB60D0857
:10D890000048704708B70D08012070470120704705
:10D8A00001207047012070470369002283F840215E
:10D8B00001207047174B184993EDE87AB3F94021DE
:10D8C000D3F87402B5EEC07AF1EE10FA07EE902AA2
:10D8D000C8BFDFED126AF8EEE77ACABF27EE267AF4
:10D8E00020EE270A27EE000A67EEA07ABDEEC00AF6
:10D8F000FDEEE77A10EE102AC1F8F02517EE902A17
:10D90000C1F8F425036801F2F4525B6B01F5BE61C6
:10D91000184700BF488B0020487B00200000C84209
:10D920001E4BDFED1F6AB3F94011A3F58050A3F53C
:10D930008043F5EEC00AD3F8C02C8A42A8BF0A463D
:10D9400007EE902AF1EE10FAF8EEE77AD6BF03F66A
:10D95000C44393ED907A93ED007A27EE800A07EEA8
:10D96000901ACCBF27EE267A27EE667AF8EEE77A91
:10D97000BDEEC00AB4EEE77AF1EE10FA58BFB0EE91
:10D98000677A60EE870A10EE102AFDEEE00AC0F812
:10D99000F02510EE903AC0F8F4357047488B00201F
:10D9A0000000C84237B52C4CD4F8A83CB3F9082085
:10D9B0001B8B07EE102A07EE903AD4F8AC3CB8EE79
:10D9C000C77AB3F908201B8BF8EEE77A054687EE95
:10D9D000270A224807EE102A07EE903AB8EEC77AD7
:10D9E000F8EEE77A8DED010AC7EE270ACDED000AC1
:10D9F00009F060FFDDED000A9DED010A28B128461F
:10DA000003B0BDE83040FFF755BF04F58043D3F8BD
:10DA1000FC23520405D4284603B0BDE83040FFF78C
:10DA20007FBFB3F9403107EE903AF8EEE77A04F59C
:10DA3000405427EE800A67EEA00ABDEEC00AFDEE54
:10DA4000E00A10EE103AC4F8F03510EE903AC4F83F
:10DA5000F43503B030BD00BF484B0020B88E002025
:10DA600010B5044687F070FE0146206900F50E707F
:10DA70000AF070F920B12046BDE81040FDF732BB36
:10DA8000114803F00DFF206990F9D0304BB102F03E
:10DA9000C9F90E48F5F748FBBDE810400B48F5F70B
:10DAA0003DBC02F035FA206905F090FB0748F5F718
:10DAB0003BFB0648F5F732FC20469FED050ABDE822
:10DAC0001040FDF7EFBC00BF808C0020482B0020E9
:10DAD000000000000B2070470048704722BA0D0874
:10DAE0000048704780B70D0801207047012070473B
:10DAF000012070470020704738B52F48F6F704F929
:10DB00002D48F5F7E1FF2C48F5F7C2FD2A48102112
:10DB1000F4F7A0FFD0B1294A936E926F9342D4BF1D
:10DB200000230123254C94F8E82072B963B304F173
:10DB300064030FCB04F1540585E80F00A4F5C04041
:10DB4000F9F7F0FC012384F8E83038BD1C4AB2F93B
:10DB50008C1C0029F9DD02F580429FED1A7A936E44
:10DB6000926D9B1A07EE903AF8EEE77A67EE877AA5
:10DB700007EE101AB8EEC77AF4EEC77AF1EE10FA93
:10DB8000CCBF01230023CDE7A4F58043642193F9A2
:10DB9000F02212FB01F2D3F8C01CA4F580548A4293
:10DBA000A8BF0A46D4F8F005C3F8C02C514226F0AD
:10DBB00007F9C4F8F005C8E7482B0020488B00207F
:10DBC000484B00200AD7233CF0B52F4C2DED028B9B
:10DBD00004F16405074695E80F0004F1540686E851
